:020000040800F2
:10000000000001106D25040871A80308359F000841
:1000100071260408712604087126040800000000F7
:10002000000000000000000000000000BDAE03085A
:10003000B9AE030800000000B5AE0308E19A00085D
:100040007126040871260408712604087126040824
:1000500071260408712604084D41010879420108FF
:100060003D42010801420108C541010895160408F6
:100070008516040875160408651604085516040844
:10008000411604082D160408712604087126040878
:1000900071260408712604087126040889410108A4
:1000A000119100088191000871260408A9910008A7
:1000B0007191000861910008519100084D170408E2
:1000C000551704083D17040845170408712604084D
:1000D000712604084D9D0008AD9C00080D9C000889
:1000E0001341010871260408D5AF030871260408DE
:1000F000219100087126040831910008191604089E
:10010000712604087126040841910008712604082C
:100110007126040871260408A52A0208892A020803
:1001200005160408F1150408DD150408C9150408AE
:10013000B515040871260408712604087126040800
:1001400071260408712604087126040875A803089E
:10015000A11504088D150408791504086D9B000885
:100160002D170408351704087126040871260408A1
:1001700071260408712604087126040871260408F3
:08018000712604087126040831
:08018800042104000100000045
:1001900016000800742500208C25002000000000B7
:1001A000680600081D000100C03000204C3100200E
:1001B000000000007006000827000400E030002066
:1001C0005031002000000000720600082C001000D2
:1001D0001C3600200C3600200000000081EC0108D5
:1001E0002B002400503600202C3600200000000098
:1001F00051EC0108290050004435002074360020DD
:1002000000000000000000000A020A00F036002092
:100210000037002000000000760600081E000400E1
:10022000D83C00201040002000000000800600089C
:1002300022000C00783F0020144000200000000045
:10024000840600081B00F400AC4000203C4F002056
:1002500000000000E55102080E0202005642002094
:100260003050002000000000900600082F00110010
:100270000A4F0020345000200000000092060008C1
:1002800005100600304F00204850002000000000FC
:10029000A4060008F5216C002040002050500020EA
:1002A00000000000096A020803010A00185100203A
:1002B0002451002000000000AA06000803000100ED
:1002C000E4520020EC52002000000000000000007A
:1002D00004008000C86200205C6300200000000071
:1002E00000000000F9010400AC570020DC6300208E
:1002F0000000000041820008FD0124008457002016
:10030000E063002000000000D18100080600160014
:10031000FC530020046400200000000045CA0208CD
:10032000FB010100385300201C6400200000000085
:100330006980000801200800206A0020406A00202F
:1003400000000000B40600081A000800046A00203B
:10035000486A002000000000BC060008FA01020004
:10036000486C0020806C00200000000085800008A0
:1003700002020300306C0020846C002000000000AA
:10038000000000000C020100206C0020886C00209E
:1003900000000000C4060008FE010900046C0020F3
:1003A0008C6C0020000000007180000803123300F4
:1003B0004B6F0020186F002000000000C8060008E6
:1003C00025005A00646E0020BE6E00200000000070
:1003D00000000000F6110C00586E00204C6E00204A
:1003E00000000000FC060008150070006C6D002085
:1003F000DC6D002000000000000000002A0060000A
:10040000AC6C00200C6D002000000000B9C902088F
:100410000101040018700020A083002000000000EB
:100420000000000008020900C8820020A483002008
:10043000000000008533010806020C004083002004
:10044000B083002000000000AF370108070202005F
:1004500064830020BC83002000000000080700081F
:1004600002000C004C830020C0830020000000002C
:1004700000000000F7010600BC820020CC830020B1
:10048000000000000A070008090201008D84002016
:10049000BC8400200000000010070008FC010900D7
:1004A0005895002044960020000000003580000888
:1004B0000A101200508D002050960020000000000D
:1004C00012070008340010007C8C00206496002085
:1004D00000000000E1C9020812200C006C8C002012
:1004E00074960020000000002407000818102C005B
:1004F000F48B002080960020000000001DF301080E
:100500000D003C00208C0020AC9600200000000074
:100510007DC1030814000200709900207499002026
:100520000000000030070008100003006099002060
:100530007899002000000000320700082800100011
:10054000509900207C99002000000000212B020817
:1005500023001000409900208C990020000000002A
:100560003D2B020819000500389900209C990020B5
:100570000000000036070008F8110100349900203F
:10058000A4990020000000003C07000800010400BE
:1005900030990020A8990020000000003E070008C4
:1005A0000E20EA00C49900202C9C002000000000CE
:1005B00025CA020813000400F49A0020189D0020A8
:1005C000000000004407000802010300AF9900206A
:1005D0001C9D002000000000312103080C002400B5
:1005E00070B000201CB100200000000009210308A9
:1005F0000102050050B0002040B1002000000000C2
:1006000069B20308000205003CAE002048B100209A
:10061000000000000000000026000E0048B9002085
:1006200038B9002000000000EDD103080B201000B5
:1006300014B7002058B90020000000004807000847
:100640001F000E0098BA00206CBC002000000000C3
:10065000580700080502010080BA00207CBC002079
:0806600000000000660700081D
:10066800C409000019012828000020030000000028
:100678004A01B400D601000000000100C800141EA1
:10068800010064002C0128000000000000000000A8
:100698000000000000000000000000002000010130
:1006A8000000040101006C1600000000E80364006B
:1006B800040A00017E05EA05B405320001000000C5
:1006C8000000000000000000000000000000000022
:1006D8000000000000000000000000000000000012
:1006E8000000000000000000000000000000000002
:1006F80000000100000000000000000000000000F1
:10070800013C240100000000280000300100005ACC
:100718000000000090012C01C800640000000001E6
:1007280000054246463400000300000105000000B1
:1007380028010000040090010000000008040400E3
:100748002B21231E64000200000001000A01290079
:0F0758000000000000000100000000050000008C
:1007670001010000F87604080C9904080000000055
:100777000000000008770408107704080000000054
:1007870001200000147704081C770408000000000B
:100797000140000020770408EC8C040800000000EA
:1007A700012000002C7704083877040800000000B7
:1007B700040000003C770408689B04080000000060
:1007C700040000004877040858AB04080000000044
:1007D7000100000002010100685E0C00FF0000003C
:1007E7000000803F0000803F000000000000000084
:1007F700000000000000803FFFFFFFFF0101D6015E
:100807004DE60108000000000000000000010101A2
:1008170001000000000001FFFF00000001010000CF
:10082700FFFFFFFF2D202D2D202D2D2D2D202D2DD0
:100837002D2D000000000000000000000000000057
:10084700000000000000000001020304010203048D
:1008570006070809010000000000803F0000803FF4
:100867000000000000000000000000000000803FC2
:100877000000000000000000000000000000000071
:100887000000000000000000000000000000000061
:10089700000000000000803F000000000000000092
:1008A70000000000006002401060024000000000ED
:1008B700000B000000002000000000000000000006
:1008C700006002402860024000000000060C0000A3
:1008D700000020000000000000000000006002404F
:1008E7004060024000000000100D000000002000E2
:1008F7000000000000000000006002405860024055
:1009070000000000160E000000002000000000009C
:10091700000000000060024070600240000000001C
:10092700200F000000002000000000000000000071
:1009370000600240886002400000000026100000AE
:1009470000002000000000000000000000600240DE
:10095700A0600240000000003011000000002000ED
:10096700000000000000000000600240B860024084
:1009770000000000362F00000000200000000000EB
:100987000000000000640240106402400000000004
:1009970000380000000040000000000000000000D8
:1009A700006402402864024000000000063900008D
:1009B700000040000000000000000000006402404A
:1009C7004064024000000000103A000000004000B0
:1009D700000000000000000000640240586402406C
:1009E70000000000163B000000004000000000006F
:1009F7000000000000640240706402400000000034
:100A0700203C000000004000000000000000000043
:100A17000064024088640240000000002644000091
:100A270000004000000000000000000000640240D9
:100A3700A0640240000000003045000000004000B4
:100A4700000000000000000000640240B86402409B
:100A570000000000364600000000400000000000D3
:100A67000000000008000000000000010000000076
:100A77000000000000000000C86D0408050804001D
:100A8700000000004C710408245B04083871040856
:100A970000000000F46D040805080A0000000000CB
:100AA7004C710408245B0408B071040800000000BE
:100AB70001010100793A030800000000C804002082
:100AC7004CAD04080000000000000000000000001A
:100AD700000000000C99040800000000000000005E
:100AE7002C05002004000000F8AC04080D000000ED
:100AF700E143030810090020000000000CB30408BC
:100B07000D0000000944030804090020000000004C
:100B17006CAD04080800000000000000F808002081
:100B2700040000005CAD04080D000000213B030831
:100B3700EC0800200000000008AC040803000000D7
:100B4700B98F0308E00800200000000064AD040826
:100B570003000000B98F0308D4080020000000003C
:100B67000CAC0408010000000000000000000000B9
:100B770000000000000000000E0000000000000060
:100B870000000000000000004CAD04080000000059
:100B97000000000000000000000000000C9904089D
:100BA70000000000000000002C05002004000000E9
:100BB70090AC040803000000F5410308C8080020B2
:100BC700080000005CAD04080D000000213B03088D
:100BD700EC0800200000000008AC04080300000037
:100BE700B98F0308E00800200000000064AD040886
:100BF70003000000B98F0308D4080020000000009C
:100C07000CAC040801000000000000000000000018
:100C170000000000000000000E00000000000000BF
:100C2700000000000000000074AD04080000000090
:100C37000000000000000000000000000C990408FC
:100C470000000000000000002C0500200400000048
:100C570098AC040803000000B98F03081C090020A2
:100C6700000000000CAC04080100000000000000B8
:100C77000000000000000000000000000E0000005F
:100C87000000000000000000000000002D202D2DB6
:100C9700202D2D2D2D202D2D2D00000000000000D2
:100CA700000000000000000000000000DA830020C0
:100CB70088136F1701000000DC83002088136F176B
:100CC70000000000E0AB0408000000000000000086
:100CD7000000000000000000F0AB0408080000005E
:100CE700000000005805002004000000FCAB0408C9
:100CF70008000000000000004C0500200000000074
:100D070008AC040804000000354203080000000096
:100D1700000000000CAC0408010000000000000007
:100D27000000000000000000000000000E000000AE
:100D3700000000000000000000000000D883002031
:100D470088136F170100000078BA002088136F1707
:100D570000000000D93A03080000000064050020E5
:100D67008C840020010000000C7104087ABA00206E
:100D7700010000001871040870BA0020020000008A
:100D87002071040832AE00200000000000000000BF
:100D970030AE002000000000000000002EAE002052
:100DA70000000000000000002CAE00200000000042
:100DB700000000002AAE0020000000000000000034
:100DC70028AE0020000000000000000030230020B3
:100DD7000000000000000000D78300200200000090
:100DE7002C71040848AC0408000000000000000053
:100DF7000000000000000000F0AB0408080000003D
:100E070000000000E805002004000000FCAB040817
:100E17000800000000000000DC05002000000000C2
:100E270008AC040804000000AD3A03080000000005
:100E3700000000000CAC04080100000000000000E6
:100E47000000000000000000000000000E0000008D
:100E570000000000000000000000000058AC04087B
:100E6700000000000000000000000000000000007B
:100E770068AC04080D00000085430308180600202D
:100E87000400000074AC04080D000000FD3A0308DC
:100E97000C0600200400000080AC04080D000000D0
:100EA7004943030800060020000000008CAC04083A
:100EB7000300000015420308F405002008000000A5
:100EC70098AC040803000000B98F03081C09002030
:100ED700000000000CAC0408010000000000000046
:100EE7000000000000000000000000000E000000ED
:100EF700000000000000000000000000A0AC040893
:100F070000000000000000000000000000000000DA
:100F1700A8AC0408040000005142030800000000C8
:100F2700000000000CAC04080100000000000000F5
:100F37000000000000000000000000000E0000009C
:100F470000000000000000000000000000AD0408E1
:100F5700000000000000000000000000000000008A
:100F67008CA404080D000000000000007806002093
:100F77000400000010AD0408080000000000000095
:100F87006C060020040000001CAD040808000000E7
:100F970000000000600600200400000024AD0408E3
:100FA70008000000000000005406002004000000B4
:100FB7002CAD0408080000000000000048060020CF
:100FC7000400000034AD0408080000000000000021
:100FD7003C060020040000003CAD040808000000A7
:100FE70000000000300600200400000044AD0408A3
:100FF7000800000000000000240600200400000094
:101007000CAC040801000000000000000000000014
:1010170000000000000000000E00000000000000BB
:101027000000000000000000C53A030800000000AF
:10103700840600200000000000000000FC060020DD
:1010470000000000000000009C07002076BA002086
:10105700040000003871040874BA0020E0150C176A
:101067000000000073BA002008000000245B040899
:1010770072BA0020050000004C710408000000004F
:1010870000000000EC07002071A5030829A503084C
:1010970001AF0308000000004DA1030891A3030856
:1010A70019A40308F1A203080000000000000000D3
:1010B70041A10308C1A00308BDA00308B9A0030804
:1010C700ADA00308A9A00308B5A00308B1A00308B1
:1010D70035A1030829A1030801A1030815A10308E5
:1010E700EDA00308D9A00308C5A0030820700020BD
:1010F700702D72000000000000000000D01C0020CE
:10110700FFFFFFFFFA0000000100000001000000E0
:1011170084B004088CB00408A0AC040800000000E8
:101127000000000000000000000000007CB0040880
:10113700040000006F4103080000000000000000E9
:101147000CAC0408010000000000000000000000D3
:1011570000000000000000000E000000000000007A
:101167000000000000000000EAAD00200100C409F3
:1011770000000000E8AD00200100C40900000000E5
:10118700E6AD00200100C40900000000E4AD002026
:101197000100C40900000000E0AD00200100C409FF
:1011A70000000000E2AD00200100C40900000000BB
:1011B700DEAD00200100C40900000000DCAD002006
:1011C7000100C40900000000EA8300200100C800F4
:1011D70001000000E8830020320030753200000073
:1011E700E7830020055A0500E283002000FF010085
:1011F700E683002001000000B0090020E4830020FE
:1012070002000000B45A0408E183002000FF010037
:10121700E583002001000000B0090020E3830020DF
:1012270002000000B45A040800000000000000009B
:10123700B8090020F25000209CFF2C01000000009C
:10124700500300200A000000B0710408D483002076
:10125700E0150C17000000005203002008000000F2
:10126700245B040851030020050000004C710408AA
:10127700D683002002000000C8710408E49A002009
:101287000100FF7F01000000E39A00200200000038
:10129700D4710408B899002003000000E471040821
:1012A700B799002003000000E4710408B69A0020F3
:1012B7000000F40101000000B49A00200000F401CE
:1012C70001000000B29A00200000F40101000000B4
:1012D700B09A00200000F40101000000AE9A00203F
:1012E70000FF0100CE9A0020E803D0070A000000A3
:1012F700CC9A0020006401000A000000C89A002070
:1013070000640100C79A002000640100CD9A002004
:10131700006401000A000000C69A00200064010072
:101327000A000000CB9A0020006401000A000000B8
:10133700CA9A0020006401000A000000C99A002030
:10134700006401000A000000C59A002000FF0100A8
:101357000A000000C49A002000FF01000A000000F4
:10136700C09900200000F40101000000BE99002090
:101377000000F40101000000BC9900200000F40106
:1013870001000000BA9900200000F40101000000EC
:10139700C09A00201400E80301000000BE9A002054
:1013A700E803307501000000BD9A002000C8010065
:1013B700BC9A002000C80100BB9A002000C80100A9
:1013C700BA9A0020006401000A000000B99A0020C0
:1013D70000FF01000A000000D99A002000C80100A0
:1013E700D89A002000C80100D79A002000C8010041
:1013F700D69A002000C80100D59A002000C8010035
:10140700D49A002000C80100D39A002000C8010028
:10141700D29A002000C80100D19A002000C801001C
:10142700ACB004080000000000000000000000004D
:1014370000000000BCB00408090000000000000024
:101447005C0A002004000000C4B004080900000082
:1014570000000000500A00200400000048B60408FD
:101467000900000000000000440A002004000000FA
:10147700287804080900000000000000380A00204E
:1014870004000000CCB004080900000000000000C0
:101497002C0A002004000000D4B004080900000052
:1014A70000000000200A002004000000DCB004084F
:1014B7000900000000000000140A002004000000DA
:1014C700E4B004080900000000000000080A00203A
:1014D700040000000CAC040801000000000000003C
:1014E7000000000000000000000000000E000000E7
:1014F700000000000000000000000000F8B1040830
:1015070000000000000000000000000000000000D4
:10151700B4A104080700000000000000800A0020B2
:101527000000000008B204080800000000000000E6
:10153700740A00200000000014B20408080000002C
:1015470000000000680A0020000000000CAC04083E
:101557000100000000000000000000000000000083
:10156700000000000E000000000000000000000066
:10157700000000001CB2040800000000000000008A
:1015870000000000000000002CB204080D0000005D
:1015970000000000BC0A00200000000034B204086C
:1015A7000D00000000000000B00A0020000000004D
:1015B7003CB204080700000000000000A80A002051
:1015C7000000000044B204080D0000000000000005
:1015D7009C0A0020000000004CB204080D00000027
:1015E70000000000900A00200000000054B2040828
:1015F7000700000000000000880A0020000000002B
:101607000CAC04080100000000000000000000000E
:1016170000000000000000000E00000000000000B5
:1016270000000000000000005CB204080000000099
:10163700000000000000000000000000B4A1040842
:101647000C00000000000000EC83002000000000F8
:1016570070B204080C00000000000000EE830020B8
:101667000000000080B204080C0000000000000029
:10167700248400200000000090B204080C00000041
:10168700000000001884002000000000A4B2040835
:101697000C00000000000000F083002000000000A4
:1016A700B0B204080C00000000000000F283002024
:1016B70000000000B8B204080C00000000000000A1
:1016C700F483002000000000CCB204080C000000E6
:1016D70000000000F683002000000000D4B20408D8
:1016E7000C00000000000000F8830020000000004C
:1016F700DCB204080C000000000000003684002063
:1017070000000000F4B204080C0000000000000014
:10171700FA8300200000000000B304080C0000005A
:1017270000000000FC83002000000000089B040864
:101737000C00000000000000FE83002000000000F5
:1017470008B304080C00000000000000008400201B
:101757000000000014B304080C00000000000000A3
:10176700028400200000000020B304080C000000E1
:101777000000000004840020000000002CB30408CF
:101787000C0000000000000006840020000000009C
:1017970038B304080C000000000000000884002093
:1017A7000000000044B304080C0000000000000023
:1017B7001C840020000000004CB304080C0000004B
:1017C700000000001A8400200000000054B3040841
:1017D7000C0000000000000028840020000000002A
:1017E70060B304080C000000000000002A840020F9
:1017F700000000006CB304080C00000000000000AB
:10180700308400200000000090B104080C000000A4
:10181700000000000A840020000000005CAD0408FE
:101827000C000000000000001284002000000000EF
:1018370078B304080C000000000000000C840020AE
:101847000000000084B304080C0000000000000042
:101857000E8400200000000090B304080C00000074
:1018670000000000108400200000000098B3040866
:101877000C0000000000000014840020000000009D
:10188700D4A104080C000000000000001E84002002
:1018970000000000A4B304080C00000000000000D2
:1018A7001684002000000000B0B304080C000000FC
:1018B700000000002684002000000000BCB30408DC
:1018C7000C00000000000000208400200000000041
:1018D700C4B304080C0000000000000022840020AC
:1018E70000000000CCB304080C000000000000005A
:1018F7002C84002000000000D4B304080C00000072
:10190700000000002E840020000000000CAC04083A
:1019170001000000000000000000000000000000BF
:10192700000000000E0000000000000000000000A2
:1019370000000000DCB30408000000000000000005
:101947000000000000000000ECB3040805000000E0
:1019570000000000B6990020000000000CAC04084D
:10196700010000000000000000000000000000006F
:10197700000000000E000000000000000000000052
:1019870000000000F4B3040800000000000000009D
:1019970000000000000000000C990408000000008F
:1019A70000000000C40000200400000000B4040888
:1019B7000D000000D1410308100B002000000000BB
:1019C700F8AC04080D000000313A0308040B0020AE
:1019D700000000000CB304080D000000153A0308CE
:1019E700F80A0020000000006CAD040808000000A1
:1019F70000000000EC0A0020040000005CAD0408B1
:101A07000D00000061390308E00A00200000000013
:101A170004B404080900000000000000D40A0020F4
:101A27000400000008AC040803000000B98F030895
:101A3700C80A0020000000000CAC040801000000E8
:101A4700000000000000000000000000000000008F
:101A57000E00000000000000000000000000000071
:101A67000CB40408000000000000000000000000A3
:101A7700000000001CB404080D0000000000000076
:101A8700280B00200000000024B404080A0000000E
:101A970000000000509B00200000000030B4040844
:101AA7000A00000000000000589B00200000000012
:101AB70038B404080A00000000000000609B002002
:101AC7000000000040B40408080000000000000007
:101AD7001C0B00200000000048B4040804000000AC
:101AE700ED90030800000000000000000CAC0408A3
:101AF70001000000000000000000000000000000DE
:101B0700000000000E0000000000000000000000C0
:101B17000000000054B404080000000000000000AA
:101B2700000000000000000068B404080D00000079
:101B370000000000400B00200000000078B40408FB
:101B470004000000018E03080000000000000000F0
:101B570080B404080D00000000000000340B0020D2
:101B67000000000094B4040804000000E18D03089D
:101B770000000000000000000CAC04080100000099
:101B8700000000000000000000000000000000004E
:101B97000E00000000000000000000000000000030
:101BA7009CB40408000000000000000000000000D2
:101BB70000000000B0B404080700000000000000A7
:101BC7007C0B002000000000BCB4040808000000E3
:101BD70000000000700B002000000000C8B40408DB
:101BE7000800000000000000640B00200000000057
:101BF700D4B404080800000000000000580B0020BF
:101C070000000000E0B40408080000000000000025
:101C17004C0B0020000000000CAC04080100000081
:101C270000000000000000000000000000000000AD
:101C37000E0000000000000000000000000000008F
:101C4700ECB4040800000000000000008F09002029
:101C570000000000547704080B000000000000009B
:101C6700F40B002000000000F8B404080B0000008B
:101C770000000000E80B00200000000004B5040885
:101C87000B00000000000000DC0B0020000000003B
:101C970010B504080B00000000000000D00B002066
:101CA700000000001CB504080B0000000000000045
:101CB700C40B0020000000005C7704080B00000044
:101CC70000000000B80B00200000000028B5040841
:101CD7000B00000000000000AC0B0020000000001B
:101CE70034B504080700000000000000A40B002022
:101CF700000000003CB504080700000000000000D9
:101D07009C0B00200000000048B504080B000000F1
:101D170000000000900B00200000000054B50408EC
:101D27000800000000000000840B002000000000F5
:101D37000CAC0408010000000000000000000000D7
:101D470000000000000000000E000000000000007E
:101D5700000000000000000060B50408000000005B
:101D670000000000000000000000000074B5040837
:101D77000800000000000000240C00200000000004
:101D870080B504080800000000000000180C0020BF
:101D9700000000008CB504080800000000000000E7
:101DA7000C0C00200000000098B504080800000093
:101DB70000000000000C0020000000000CAC04082C
:101DC700010000000000000000000000000000000B
:101DD700000000000E0000000000000000000000EE
:101DE70000000000A0B5040800000000000000008B
:101DF7008C09002000000000B0B504080B000000AB
:101E0700000000006C0C002000000000BCB50408B6
:101E17000B00000000000000600C00200000000024
:101E2700C8B504080700000000000000580C002097
:101E370000000000D4B504080700000000000000FF
:101E4700500C002000000000E0B504080700000067
:101E570000000000480C002000000000ECB504085A
:101E670008000000000000003C0C002000000000FB
:101E7700F4B504080800000000000000300C002042
:101E8700000000000CAC0408010000000000000086
:101E97000000000000000000000000000E0000002D
:101EA700000000000000000000000000FCB504086E
:101EB70000000000000000008C0900200000000066
:101EC70008B604080700000000000000B80C002056
:101ED7000000000010B60408070000000000000022
:101EE700B00C00200000000018B60408070000002E
:101EF70000000000A80C002000000000F077040894
:101F07000700000000000000A00C002000000000F7
:101F1700F87704080700000000000000980C002074
:101F2700000000000078040807000000000000001F
:101F3700900C00200000000020B6040807000000F5
:101F470000000000880C00200000000028B60408EC
:101F57000700000000000000800C002000000000C7
:101F670030B604080700000000000000780C0020CD
:101F7700000000000CAC0408010000000000000095
:101F87000000000000000000000000000E0000003C
:101F9700000000000000000000000000000000003A
:101FA700D58A0308C00C0020B49900201B0000004C
:101FB700F4710408B39900200A320100B299002095
:101FC70001FA0100AE99002000C80100AC99002079
:101FD700E803D0070100000042455441464C4947F9
:101FE7004854463400000000E0830020000301004D
:101FF700DF83002000030100193C0308F53B0308B9
:102007009C0D0020BD3B03087D3B0308140E0020F8
:102017004D8A03083D3C0308C80E0020EB8A0308DD
:10202700B58D0308D41100209D3903080000000076
:1020370024120020C9900308318D030800130020E3
:102047000D8B030800000000B4130020958B0308D4
:10205700658B0308401400201D8C0308618C03085E
:10206700E0140020C29A002001030100418B0308FD
:102077001D8B0308F8150020C58B0308218E030864
:1020870084160020918C0308798E03084C170020D2
:10209700B89A00200103010038B6040800000000C8
:1020A70000000000000000000000000044B6040823
:1020B70008000000000000006C180020000000006D
:1020C7004CB6040807000000000000006418002058
:1020D700000000005CB604080700000000000000D4
:1020E7005C1800200000000068B604080700000024
:1020F70000000000541800200000000074B6040817
:102107000D0000000000000048180020000000003B
:1021170080B6040803000000B98F03083C180020AC
:10212700000000000CAC04080100000000000000E3
:102137000000000000000000000000000E0000008A
:1021470000000000000000000000000088B604083E
:102157000000000000000000000000000000000078
:1021670098B604080A0000000000000090760408F2
:1021770000000000A0B604080A00000000000000EC
:10218700D876040800000000A8B604080A0000007A
:1021970000000000DA9A002000000000B0B6040832
:1021A7000A0000000000000078180020000000006E
:1021B7000CAC040801000000000000000000000053
:1021C70000000000000000000E00000000000000FA
:1021D7000000000000000000B8B60408000000007E
:1021E700000000000000000000000000C4B6040862
:1021F70003000000B98F0308B0180020000000009A
:10220700D0B6040803000000B98F0308A418002003
:1022170000000000D8B6040803000000B98F0308C7
:102227009818002000000000E0B604080500000030
:1022370000000000DE83002000000000E8B604086C
:1022470007000000000000009018002000000000B8
:10225700F4B60408070000000000000088180020FA
:10226700000000000CAC04080100000000000000A2
:102277000000000000000000000000000E00000049
:1022870000000000000000000000000000B7040884
:102297000000000000000000000000000000000037
:1022A70014B7040803000000B98F0308D4180020EE
:1022B7000000000020B7040803000000B98F0308DE
:1022C700540300200000000028B7040803000000A2
:1022D700B98F0308C81800200000000030B70408B1
:1022E70003000000B98F0308BC180020000000009D
:1022F7000CAC040801000000000000000000000012
:1023070000000000000000000E00000000000000B8
:1023170000000000000000003CB7040800000000B7
:1023270000000000000000000000000048B704089B
:1023370007000000C58E03083019002000000000C8
:1023470094B3040803000000B98F03082419002080
:102357000000000054B7040803000000B98F030809
:1023670018190020000000005CB7040803000000F3
:10237700B98F03080C1900200000000064B7040897
:1023870007000000A98E03080419002000000000C0
:102397008477040803000000B98F0308F8180020A9
:1023A7000000000070B7040803000000B98F03089D
:1023B700EC180020000000007CB7040803000000B0
:1023C700B98F0308E0180020000000000CAC0408D7
:1023D70001000000000000000000000000000000F5
:1023E700000000000E0000000000000000000000D8
:1023F700000000009D8A0308658A03083819002039
:10240700FD8C030800000000EC190020613B030865
:10241700453B0308781A0020000000000000000078
:102427002C1B0020D58C0308E18E0308B81B002065
:1024370088B704080000000000000000000000004A
:102447000000000094B7040803000000B98F0308D8
:10245700C41C0020000000009CB704080300000013
:10246700B98F0308B81C0020000000004C9B04082B
:1024770003000000B98F0308AC1C00200000000017
:10248700A8B7040803000000B98F0308A01C0020A8
:1024970000000000B4B7040803000000B98F030868
:1024A700941C002000000000BCB7040802000000D4
:1024B7009D9103080000000000000000C4B7040855
:1024C700020000009D9103080100000000000000C9
:1024D700D0B70408020000009D9103080200000025
:1024E70000000000000000000E00000000000000D7
:1024F70000000000000000000403090412010002AC
:102507000202004083044057000201020301000059
:1025170009024300020100C032090400000102025F
:102527000100052400100105240100010424020212
:102537000524060001070582030800FF09040100BE
:10254700020A00000007050102400000070581029A
:1025570040000000FF0000000990020845A403089E
:10256700BD8A020895A1030805A60308A5A10308CB
:10257700C1A1030885A1030875A103080000000095
:1025870000000000E001080000A2040800000000AD
:102597000000000045210308A08601000400000098
:1025A7000000000000000000000000000000000024
:1025B70000000000000000000000000094B30408C1
:1025C700C8970408000000008D5C01087D0000002A
:1025D70006000000000000000000000000000000EE
:1025E70000000000000000000000000000000000E4
:1025F70024BB04080000000000000000210C0108B3
:10260700E8030000030000000000000000000000D5
:1026170000000000000000000000000000000000B3
:10262700000000002CBB04080000000000000000B0
:102637007DCB020810270000030000000000000007
:102647000000000000000000000000000000000083
:1026570000000000000000008CB904080000000022
:10266700D9EA010811100108204E000005000000FA
:102677000000000000000000000000000000000053
:102687000000000000000000000000008CA3040808
:102697000000000000000000899F000810270000CC
:1026A7000100000000000000000000000000000022
:1026B7000000000000000000000000000000000013
:1026C70038BB04080000000000000000018000087B
:1026D700E803000005000000000000000000000003
:1026E70000000000000000000000000000000000E3
:1026F7000000000044BB04080000000000000000C8
:102707006D230308204E00000300000000000000B6
:1027170000000000000000000000000000000000B2
:10272700000000000000000054BB04080000000087
:102737000000000075210308204E00000300000080
:102747000000000000000000000000000000000082
:1027570000000000000000000000000064BB040847
:10276700000000000000000015310108400D0300C3
:10277700030000000000000000000000000000004F
:102787000000000000000000000000000000000042
:10279700C4A20408000000000000000039CD0308AF
:1027A70010270000010000000000000000000000EA
:1027B7000000000000000000000000000000000012
:1027C70000000000E497040800000000000000007B
:1027D7003964020810270000030000000000000011
:1027E70000000000000000000000000000000000E2
:1027F700000000000000000074BB04080000000097
:1028070000000000AD0A0108A086010001000000D9
:1028170000000000000000000000000000000000B1
:10282700000000000000000000000000D49704082A
:102837000000000000000000CD09010850C300009F
:102847000100000000000000000000000000000080
:102857000000000000000000000000000000000071
:1028670090B10408000000000000000035050108D1
:10287700A861000001000000000000000000000047
:102887000000000000000000000000000000000041
:10289700000000007CBB04080000000000000000EE
:1028A70099BE0308A0860100010000000000000097
:1028B7000000000000000000000000000000000011
:1028C700000000000000000094A3040800000000BE
:1028D70000000000F5C30008A00F00000100000081
:1028E70000000000000000000000000000000000E1
:1028F70000000000000000000000000088BB040882
:1029070000000000000000005D6C020810270000B6
:1029170001000000000000000000000000000000AF
:1029270000000000000000000000000000000000A0
:102937004C9B04080000000000000000F97C02081E
:102947001A41000001000000000000000000000024
:102957000000000000000000000000000000000070
:1029670000000000F8A304080000000000000000B9
:1029770081E40308102700000100000000000000A8
:102987000000000000000000000000000000000040
:102997000000000000000000489B04080000000041
:1029A70000000000319303081A41000001000000F5
:1029B7000000000000000000000000000000000010
:1029C70000000000000000000000000094BB0408A5
:1029D700000000000000000061020408400D030031
:1029E70000000000000000000000000000000000E0
:1029F70000000000000000000000000000000000D0
:102A07009CBB04080000000000000000F5AB0108B3
:102A1700400D03000000000000000000000000005F
:102A2700000000000000000000000000000000009F
:102A370000000000A4BB0408000000000000000024
:102A4700C5BB0308A08601000300000000000000CA
:102A5700000000000000000000000000000000006F
:102A6700000000000000000000FFFF000000000061
:102A7700AA550501000001AA550B010000AA550738
:102A8700010000AA55090200000000000100000033
:102A9700C012AA5503009F01500100000700000063
:102AA7000200000048230020000000000000000092
:102AB700000000000000000000000000000000000F
:102AC70000000000000000000000000000000000FF
:102AD70000000000000000000000000000000000EF
:102AE70000000000000000000000000000000000DF
:102AF70000000000000000000000000000000000CF
:102B0700000000000000000043000000000000007B
:102B170000000000000000000000000000000000AE
:102B2700000000000000000043000000000000005B
:102B3700000000000000000000000000000000008E
:102B4700000000000000000043000000000000003B
:102B5700000000000000000000000000000000006E
:102B6700000000000000000043000000000000001B
:102B7700000000000000000000000000000000004E
:102B870000000000000000004300000000000000FB
:102B9700000000000000000000000000000000002E
:102BA70000000000000000004300000000000000DB
:102BB700000000000000000000000000000000000E
:102BC70000000000000000004300000000000000BB
:102BD70000000000000000000000000000000000EE
:102BE7000000000000000000B32804088F28040834
:102BF70000000000B3BB040878B00408007D040897
:102C0700007D0408007D0408007D0408007D040899
:102C1700007D0408007D0408007D0408007D040889
:102C2700FFFFFFFFFFFFFFFFFFFFFFFFFFFF0000AB
:102C37000100415343494900000000000000000023
:102C4700000000000000000000000000000000007D
:102C57000000415343494900000000000000000004
:102C6700000000000000000000000000000000005D
:082C7700000000000100000054
:1080000038B50B4C23688BB15A68821A002A054692
:1080100004DA0CE05A68AA1A002A07DB9A68226080
:1080200018461A6890472368002BF3D138BD38BD35
:10803000E03400200B4B002210B4027203F584746C
:10804000032102E0072A09DC9979890702D5197909
:10805000815401329C4203F11803F3D15DF8044BC3
:10806000704700BF5464040828230370704700BFA2
:108070000123322131224170427103720370037176
:10808000704700BF1F22032302704370704700BF78
:10809000436A8269D154436A0169826B01338B421E
:1080A00028BF00234362002A2FD0EFF31182502310
:1080B00083F31288836B1968C9072CD470B45E6887
:1080C0006EB9456A816A8D4217D084690C44DC60C0
:1080D0000ED9691A59608562002180F85C10196810
:1080E00041F00101D2B2196082F3118870BC70476F
:1080F0000469611A59608662EEE7012380F85C30FA
:10810000D2B282F3118870BC7047826DD36843F09D
:108110008003D3607047D2B282F31188704700BFEA
:10812000426B10B462B1C36CC2684469D11A013B9E
:10813000615C5DF8044B08BF1346C364C8B2704766
:10814000016A4369C4685B5C0131A14228BF1146E2
:1081500001625DF8044BD8B2704700BF836B13B166
:1081600090F85C007047836A406A181AB0FA80F091
:1081700040097047416A836A99420AD3CB1A816BDE
:10818000026961B14968501E0B4483420AD2C01A89
:10819000704702691144CB1A816B0029F2D1501E3D
:1081A000C01A704700207047436B43B1C26C5B68D4
:1081B00093422FBF981AC0689B1AC0187047C269B3
:1081C000036A9A422FBFD01AC0688018C01A70473D
:1081D0000A4B30B503F1180493F900205D78072AA3
:1081E000C8BF143A811804330D7313F8025C855428
:1081F00013F8012C0A76A342EED130BDF03A040800
:1082000003682DE9F041DF691FB13B46BDE8F0414D
:108210001847002A164611DD04460D460E4400E0BC
:1082200023689B68204698470028F9D0236815F8F2
:10823000011B1B6820469847AE42F1D1BDE8F08192
:1082400000232522027043708370C370704700BF03
:10825000038A2DE9F0478589ADB21D4029D00F462C
:1082600006464FF000484FF00009B5FA85F328FAAA
:1082700003F2D24391B21B3B15403182042B16D836
:10828000DFE803F03129211903007B6A002B32D08B
:1082900003F1FF3A1FFA8AFAC7F824903C6A34B116
:1082A00023682046514698476468002CF8D1002D79
:1082B000DBD1BDE8F0873868716B036889B29847F5
:1082C000002DD2D1F5E77868B16B036889B2984781
:1082D000002DCAD1EDE7B868F16B036889B2984701
:1082E000002DC2D1E5E7F868316C036889B2984780
:1082F000002DBAD1DDE7F36A1FFA83FACEE700BF9B
:1083000030B50446806D61718389A26823F40053FF
:108310001B041B0C838185B0A379009213F0040227
:1083200030D04FF4805213F00203ADF804205CD13A
:10833000ADF806304FF480630022ADF8083011F03C
:108340000103ADF80C2028D1ADF80A3008238D07C1
:10835000694648BFADF80A3020F0B2FFA279A36D9C
:10836000D10724D412F0080F9A8A1BD122F00802F8
:108370001204120C9A829A8992B242F400529A81A3
:1083800005B030BD13F00203ADF804202AD04FF43D
:1083900000551346ADF80650CEE70423ADF80A3079
:1083A0000C23D4E792B242F008029A82E3E7104924
:1083B0008B4215D0A1F54C418B420FD001F5806165
:1083C0008B4209D00B498B42CCD10520012139F0D9
:1083D00081F8A279A36DC5E70220F7E70120F5E750
:1083E0000020F3E7ADF80630A6E74FF400539FE70F
:1083F000001001400014014010B50446806DA160DA
:10840000838923F400531B041B0C8381A37984B05C
:1084100013F00402009135D04FF4805213F00203A0
:10842000ADF804205CD1ADF806304FF4806362797A
:10843000ADF80830D1074FF00003ADF80A30ADF8C1
:108440000C3045BF0423ADF80A3008230C236946DD
:10845000920748BFADF80A3020F032FFA279A36D31
:10846000D1071FD412F0080F9A8A16D122F0080201
:108470001204120C9A829A8992B242F400529A81A2
:1084800004B010BD13F00203ADF8042025D04FF462
:1084900000511346ADF80610C9E792B242F0080247
:1084A0009A82E8E710498B4215D0A1F54C418B42E6
:1084B0000FD001F580618B4209D00C498B42D1D19C
:1084C0000520012139F006F8A279A36DCAE7022040
:1084D000F7E70120F5E70020F3E7ADF80630A6E75F
:1084E0004FF400539FE700BF00100140001401400B
:1084F000022828BF022010B4084C094B207000EB62
:108500008002C0EBC20207495DF8044B013003EB67
:108510004203C0B20B6034F0EFBC00BF6C8C002093
:10852000C499002084B7002008B517F0A5F90CF015
:108530005DF9BDE8084017F087B900BF2DE9804814
:10854000013085B0C3B203938B4D8C4F8C4C8D4E54
:108550000A2302933220DFF8309227F0D3F84FF449
:10856000FA7A4FF0100C4FF47A70D9F80430C3F354
:108570000803002B40F0C180EFF31183002B40F083
:10858000BC802968A26800BF2B689942F9D1D7F84E
:1085900000E000FB0EF39B1AB3FBFEF300FB01317E
:1085A0004FF0010E0191D9F80430C3F30803002BFA
:1085B00040F08780EFF31183002B40F082802B681E
:1085C000A16800BF2A689342F9D1D7F800B000FB38
:1085D0000BF2521AB2FBFBF200FB0323019A9B1A27
:1085E000B3F57A7FDFD3BAF1010ABED1039B002B2A
:1085F00040F0BD804FF47A7ADFF88C9150464FF00E
:10860000100CD9F80430C3F30803002B40F092801B
:10861000EFF31183002B40F08D802968A26800BF22
:108620002B689942F9D1D7F800E000FB0EF39B1AB2
:10863000B3FBFEF300FB01314FF0010E0191D9F8BD
:108640000430C3F3080303BBEFF31183EBB92B68CA
:10865000A16800BF2A689342F9D1D7F800B000FBA7
:108660000BF2521AB2FBFBF200FB0323019A9B1A96
:10867000B3F57A7FE3D3BAF1010AC2D1029B013B81
:1086800002937FF467AF38F05BFFEFF311888CF350
:108690001288A1682368DB0344BFC6F800E0A16824
:1086A0002B6832685FFA88F888F31188D7F8008061
:1086B0001A4400FB08F35B1AB3FBF8F300FB023328
:1086C000D4E7EFF311888CF31288A1682368DB03E9
:1086D00044BFC6F800E0A1682B6832685FFA88F8EA
:1086E00088F31188D7F800801A4400FB08F35B1A5E
:1086F000B3FBF8F300FB023370E7EFF311828CF366
:108700001288D4F808E02368D90303D50123336025
:10871000D4F808E02B683168D2B282F311883A6845
:10872000194400FB02F3A3EB0E03B3FBF2F300FBCF
:10873000013135E7EFF311828CF31288D4F808E0A9
:108740002368D90303D501233360D4F808E02B68EC
:108750003168D2B282F311883A68194400FB02F3FF
:10876000A3EB0E03B3FBF2F300FB013164E7184601
:1087700026F02AFE3EE700BFE86B0020EC6B0020ED
:1087800010E000E0E46B002000ED00E038B5484B5D
:108790005A899989914224BF00225A81198ADA891B
:1087A000914224BF0022DA81DA78CAB1072A41490E
:1087B0006AD091F85300404D012400210A282C7002
:1087C0009C70D9715DD00C2807D0002A6CD0DFEDE9
:1087D0003B7A072A0ED00A2862D0DFED397A09E009
:1087E000344A92F853000A2856D00C285BD1D97924
:1087F000DFED347A344C9FED350AA278002918BF9A
:10880000F0EE407A062A04D8314901EB820191ED5D
:10881000060A217979B1013A032A0BD8F7EE007ADA
:1088200087EE800A3AF038F92388984228BF184624
:10883000208038BD38BD9B781F4A07EE103A11786A
:10884000B8EEC77A67EE277A07EE101AB8EEC77A45
:1088500027EE277AB4EEC70AF1EE10FAEADD80EED1
:10886000277AFDEEC77A17EE903A102BA8BF102397
:10887000012BB8BF0123DBB28B4238BF0B4613700C
:1088800038BDDFED147AA4E791F853000A2803D02D
:108890000C28ACD0D9799AE7D979DFED0E7AA9E71F
:1088A000DFED0D7AA6E7D979DFED047AA2E700BF04
:1088B000508D0020648D0020349900206F12033900
:1088C0006F12833A0AD7A339FC5300206F12033882
:1088D000F03A04085304E9380F506E3A2DE9F04796
:1088E000AA4FAB4E16F0C8FFBE421ED2DFF824835B
:1088F000DFF824934446258862197DB14A450DD29C
:10890000052D0BD933886188C3F30B03994200F01E
:10891000E080144625886219002DEFD17168304639
:1089200014360BF0EFFEBE42E4D39A4A1378A3F15B
:10893000170102290FD9984911F83300002840F097
:10894000F780D8000144497829B1944911F83330AF
:108950000BB918231370924B5A78022A00F2D9806F
:108960009049914802EB420201EB82011A780160C2
:10897000022A00F2D78002EB82018C4BC2EBC102CB
:1089800003EB4203998C5A8C894C9142236001D3AA
:1089900000225A84874B9A78042A00F0EA8032B980
:1089A0001A88B2F5F07F84BF4FF4F0721A80824DBE
:1089B000FFF7ECFE2B68814A1A40002A00F0E280A3
:1089C000D80700F1D180590400F1C9801A0700F1DD
:1089D000B8809B0400F1BC802CF072FF10B978487D
:1089E00033F0CCFB4FF400700BF0C2FE4FF40010DC
:1089F0000BF0BEFE4FF000700BF0BAFE4FF080603F
:108A00000BF0B6FE26F06EFA002130226D483BF0E6
:108A100000F8206825F0B6F96B4B256803F150018A
:108A200003E00433994200F081801A78002AF8D1DB
:108A30009C78D8788442F4D26449654B0A70284601
:108A40001D602BF071FD634A63491079634A644BE2
:108A50001160C822642111FB0021002259609A6034
:108A6000DA601A615A619A61DA6183F8202083F82A
:108A700021201BF067FE5B4B9FED5B5A1B885B4A16
:108A80009FED5B6A55795B4C5B495C48086006EE7C
:108A9000903AF8EEE66A1388C5EE265A07EE103AC9
:108AA00053881279C4ED005A07EE903AB8EEC77AAF
:108AB000534BF8EEE77A1D725A7227EE067A67EE8C
:108AC000867ABDE8F04783ED017AC3ED007A16F0AF
:108AD000BBBE63799B077FF41CAF716894F804A058
:108AE00030460BF00FFE3388BAEB133F04D0143638
:108AF000BE42FFF4FFAE18E773887068AA1FC3F385
:108B00000B039A4204F10601A8BF1A4639F0EEFDA4
:108B1000EDE700225A701A78234822490160022AA0
:108B20007FF629AF00221A70204B2BE7012283E742
:108B3000D8000C186468002C7FF404AF172414705C
:108B400000E730480BF014FE2B689B047FF544AF20
:108B50002D480BF00DFE40200BF00AFE3CE72B48A1
:108B60000BF006FE2B6831E729480BF001FE2B685D
:108B700029E79A8AB2F57A7FBFF419AF4FF47A7277
:108B80009A8214E743F008032B6019E7680600088F
:108B90009001000870990020C85D0408505B04082B
:108BA0006C8C002070B0002088B70020C499002091
:108BB00084B70020FC530020F49A002009600002D2
:108BC000208C0020842E00204435002037230020F4
:108BD000B82E0020206A002046990020BC2D0020DD
:108BE000AC3C0020E0300020C0C9FB4874250020C8
:108BF00017B7D138E43000208C6400203661023D84
:108C0000686400200160000209400002092000029F
:108C100008600002024000080080000808B516F055
:108C20002BFE0BF0E3FD16F00FFEFFF757FE0120C1
:108C3000BDE8084034F060B938B50C4C0C4DAC427E
:108C400006D26168204614340BF05CFDAC42F8D3C8
:108C5000084A094B094C1460002209491A705A70DD
:108C600008480860BDE838401CF050BF900100087B
:108C70006806000884B700206C8C0020C49900208E
:108C800088B7002070B0002008B5FFF7D5FF16F0B8
:108C9000F3FD0BF0ABFDBDE8084016F0D5BD00BFFD
:108CA000F0B50C2934D8DFE801F0893333335E3373
:108CB0003333343333330700048C9689B2F802E03F
:108CC0001788734D24F480542404240C0484038CEA
:108CD0008488818B23F4005321F4E6411B040904AA
:108CE0001B0C46EA0E06090C43EA063341EA07214B
:108CF000A8429BB2A4B289B200F09E8005F58065BF
:108D0000A84200F099809268848081830264038481
:108D1000F0BD048C9589B2F802C0B2F800E05C4F57
:108D200024F480742404240C0484038C8688818BAE
:108D300023F400731B0421F073011B0C45EA0C049F
:108D4000090443EA0423090CB8429BB2B6B241EAD3
:108D50000E015CD04F4CA04259D09268868081832E
:108D6000C2630384F0BD048C9589B2F802C0B2F8E6
:108D700000E0474E24F010042404240C0484038CE7
:108D80008788018B23F0200321F4E6411B040904AA
:108D90001B0C45EA0C04090C43EA041341EA0E21BA
:108DA000B0429BB2BFB289B25DD03A4CA0425AD019
:108DB00092688780018382630384F0BD048C978965
:108DC000B2F802E01688324D24F001042404240C89
:108DD0000484038C8488018B23F002031B0421F09C
:108DE00073011B0C47EA0E0709043B43090CA84218
:108DF0009BB2A4B241EA060125D005F58065A842E0
:108E000021D092688480018342630384F0BDD589B8
:108E1000148A578A23F4006343EA05254FF6FF338B
:108E20002B40958826F440563C4343EA052346EA06
:108E300004169BB2B6B290E7158A24F4804444EA43
:108E40008514A4B25FE7D689158A578A23F00803F0
:108E5000334324F4407496883D4323F004032C43A9
:108E60003343A4B2CDE7D489158A568A23F0800310
:108E700043EA04134FF6BF741C40938827F44067FD
:108E8000354344EA031347EA85079BB2BFB28FE735
:108E900000000140000401402DE9F04F4FF4A072A2
:108EA000002183B08A488B4CDFF84C928A4D8B4E60
:108EB0008B4FDFF848823AF0ACFD8A488A49DFF8E8
:108EC00040E2DFF840C200221359834200F0D5800F
:108ED000B3F1804F00F0DC80AB4200F0E480B3429D
:108EE00000F0E380BB4200F0E280734500F0E180D7
:108EF000634500F0E080434500F0DF80DFF808A222
:108F0000534500F0DC800AF5806A534500F0D980B3
:108F10000AF5806A534500F0D680AAF5983A534581
:108F200000F0D3800AF5806A534500F085800AF589
:108F3000806A534508BF0D237FD01832B2F5907F69
:108F4000C2D1644C694E6A4F6A4D04F5907802E0D4
:108F50001834A0456DD0A379002BF9D023794FEABE
:108F6000131909F1FF39B9F1030F03F00F03EFD81B
:108F700036F8190040FA03F2D207E9D54FF0010A9A
:108F80000AFA03F3013B184039F06CF917F809307D
:108F9000184415EBC002DBD055F83000DFF86CE167
:108FA000217A00F13F4303F57E039B0A1EF803304C
:108FB00003F01F0E5B09032B0AFA0EFA5FD0042B95
:108FC00068D0022B07D1DFF820E1DEF844304AEA0E
:108FD0000303CEF8443093880093B3FA83F3C3F1CC
:108FE0001F039BB2DA0800EB820203F00703D2F8FA
:108FF00020E09B004FF00F0C0CFA03FC2EEA0C0E45
:10900000C2F820E0D2F820E001FA03F343EA0E03AD
:10901000136269460023022218348DF804208DF86B
:1090200005308DF806308DF8073020F043FBA04561
:1090300091D103B0BDE8F08F0C2309EBC3034FF0CF
:10904000010A1B7903F01F0B5B09032B0AFA0BFAC9
:1090500009D0042B0CD0022B7FF46FAF4B6C4AEA83
:1090600003034B6469E70B6C4AEA03030B6464E790
:109070000B6B4AEA03030B635FE70023DDE7DFF8CE
:1090800068E0DEF840304AEA0303CEF84030A2E759
:109090000123D2E7DFF850E0DEF830304AEA03037C
:1090A000CEF8303097E70223C7E70323C5E7042350
:1090B000C3E70523C1E70623BFE70723BDE708236E
:1090C000BBE70923B9E70A23B7E70B23B5E700BFDE
:1090D000C0840020546404080004004000080040DC
:1090E000000C004000000140003802407865040890
:1090F00074650408506A0020585D040800040140AB
:109100000010004000140040004001401C640408AE
:1091100001490248FFF79CB8B0850020004001409B
:1091200001490248FFF794B88885002000040140F7
:1091300001490248FFF78CB88885002000040140EF
:1091400001490248FFF784B860850020000C004008
:1091500001490248FFF77CB838850020000800402C
:1091600001490248FFF774B8108500200004004050
:1091700002494FF08040FFF76BB800BFE884002041
:1091800010B5064C06482146FFF762F804F58C71CD
:109190000448BDE81040FFF75BB800BFC084002062
:1091A000000001400044014001490248FFF750B867
:1091B000C084002000000140F0B50468534DA30AAC
:1091C000AB4200F083800ED9514DAB4266D076D9C8
:1091D000504DAB4266D00135AB4240F095804FF424
:1091E0009C7E072609E0023DAB4273D052D8B3F50E
:1091F000801F73D14FF0480E01264779B0004FEA27
:10920000970C00296BD063460227A5899F408319DC
:109210000CEB43032F4303F1040C3F4DBFB245F861
:10922000231045F82C20A781EFF31181502282F3FF
:109230001288821905EBC2021369002B36D0136223
:109240000433821905EBC202576917B11F605369D5
:109250000433821905EBC202976917B11F60936945
:109260000433821905EBC202D76917B11F60D369B5
:1092700004330027CAB21F6082F31188304405EB23
:10928000C000036AABB9A38923F001031B041B0CC4
:10929000A381F0BD4FF0980E0326AEE74FF0E80E25
:1092A0000526AAE74FF4887E0626A6E705EB0E03FF
:1092B000C7E7A3899BB243F00103A381F0BD013D41
:1092C000AB4220D14FF0200E002696E74FF0C00EA3
:1092D000042692E74FF0700E02268EE7F0BD0223BF
:1092E000BF0803FA07F7A3890B4D9BB223EA0703D4
:1092F00087190CEB470CA3810CF1040345F82C10E3
:1093000045F8232090E7F0BDF0BD00BF030010003A
:109310004100100050001000C084002010B5036808
:1093200082480139834282B089B200F0CA80A0F538
:109330008060834200F0C58000F58040834200F0E9
:10934000B78000F58060834200F0B28000F5806055
:10935000834200F0AD80764C188824686408B4FB22
:10936000F2F4013CA4B282B2B3F1804F0AD071484A
:10937000834207D000F58060834203D000F580600F
:10938000834202D122F0700292B26B48834200F015
:10939000A18000F58060834200F0A68022F4407234
:1093A00000F56C4092B283421A80D9621C854FD07E
:1093B0005E4A93424CD001229A821A8892B242F0BD
:1093C00001021A80B3F1804F00F09880594A93420D
:1093D00000F0968002F58062934200F0938002F5DF
:1093E0008062934200F0908002F58062934200F028
:1093F0008D8002F58062934200F08A8002F570420F
:10940000934200F0878002F57052934200F084800E
:1094100002F58062934200F0818002F580629342FF
:109420007ED0A2F5983293427CD002F580629342BE
:109430007AD002F58062934208BF0D2215D002A8AF
:109440004FF0012340F8043D1FF0A4FE02B010BD10
:109450000122002119869A821A88384892B242F075
:10946000010283421A80ADD10A46354B03EBC20399
:1094700001A85C798DF80440012300228DF80530A5
:109480008DF807308DF806201FF084FE1B2C08D0C5
:109490002E2CDBD12B4B019301A81FF07BFE02B0D9
:1094A00010BD294B019301A81FF074FE02B010BD3E
:1094B0001F4C18882468B4FBF2F4013CA4B282B2B9
:1094C00052E71B4C18882468B4FBF2F4013CA4B2A8
:1094D00082B257E701201A80D9621C8598821A88C7
:1094E00092B202431A8071E701201A80D9621C856A
:1094F00098821A8892B202431A8063E70122B4E785
:109500000222B2E70322B0E70422AEE70522ACE76D
:109510000622AAE70722A8E70822A6E70922A4E76D
:109520000A22A2E70B22A0E70C229EE700040140DA
:109530004C8D00200004004000100040000001405D
:10954000585D04082C010001190100012B4B9842C1
:109550003CD0B0F1804F3BD0A3F57C43984239D04A
:1095600003F58063984237D003F58063984235D085
:1095700003F58063984233D003F58063984231D07D
:1095800003F5704398422FD003F5705398422DD0C5
:1095900003F5806398422BD003F58063984229D06D
:1095A000A3F59833984227D003F58063984207D0FB
:1095B00003F58063984208BF0D2202D00020704757
:1095C0000C220F4B03EBC203187970470022F8E717
:1095D0000122F6E70222F4E70322F2E70422F0E791
:1095E0000522EEE70622ECE70722EAE70822E8E791
:1095F0000922E6E70A22E4E70B22E2E70000014045
:10960000585D04082DE9F04F013085B0C3B20393D3
:109610000B4602918B4C8C4E002B00F09A8032202E
:109620008A4D8B4FDFF82C9226F06CF84FF4FA7AC3
:109630004FF0100C4FF47A70D9F80430C3F30803DC
:10964000002B40F0DE80EFF31183002B40F0D98037
:109650002968A26800BF2B689942F9D1D7F800E0C9
:1096600000FB0EF39B1AB3FBFEF300FB01314FF03E
:10967000010E0191D9F80430C3F30803002B40F028
:109680008780EFF31183002B40F082802B68A16864
:1096900000BF2A689342F9D1D7F800B000FB0BF263
:1096A000521AB2FBFBF200FB0323019A9B1AB3F59B
:1096B0007A7FDFD3BAF1010ABED1039B002B40F0C1
:1096C000BD804FF47A7ADFF88C9150464FF0100C41
:1096D000D9F80430C3F30803002B75D1EFF31183DD
:1096E000002B71D12968A26800BF2B689942F9D17B
:1096F000D7F800E000FB0EF39B1AB3FBFEF300FB70
:1097000001314FF0010E0191D9F80430C3F3080381
:1097100013BBEFF31183FBB92B68A16800BF2A6864
:109720009342F9D1D7F800B000FB0BF2521AB2FB0A
:10973000FBF200FB0323019A9B1AB3F57A7FE3D374
:10974000BAF1010AC4D1029B013B0293002B7FF4C2
:1097500066AF05B0BDE8F08FEFF311888CF3128887
:10976000A1682368DB0344BFC6F800E0A1682B684A
:1097700032685FFA88F888F31188D7F800801A44B5
:1097800000FB08F35B1AB3FBF8F300FB0233D2E7EC
:10979000EFF311888CF31288A1682368DB0344BFC0
:1097A000C6F800E0A1682B6832685FFA88F888F391
:1097B0001188D7F800801A4400FB08F35B1AB3FB4A
:1097C000F8F300FB023370E7EFF311828CF3128899
:1097D000D4F808E02368D90303D501233360D4F813
:1097E00008E02B683168D2B282F311883A681944D4
:1097F00000FB02F3A3EB0E03B3FBF2F300FB01311A
:109800007FE7EFF311828CF31288D4F808E0236825
:10981000D90303D501233360D4F808E02B683168FD
:10982000D2B282F311883A68194400FB02F3A3EB29
:109830000E03B3FBF2F300FB013118E7184625F0E5
:10984000C3FD3EE710E000E0E46B0020E86B002081
:10985000EC6B002000ED00E0204B5B68C3F30803D5
:1098600030B4BBB9EFF31183A3B91D4B1D4C18687D
:10987000A16800BF1A689042F9D11B4B1C684FF4D5
:109880007A7202FB04F3591AB1FBF4F130BC02FB0B
:1098900000107047EFF31182102383F312881149EF
:1098A0008C680B6813F4803F104B02D001201860C5
:1098B0008C680B49D2B20D68186882F311880A4B84
:1098C00019684FF47A72284402FB01F31B1B30BC69
:1098D000B3FBF1F302FB0030704700BF00ED00E086
:1098E000E86B002010E000E0EC6B0020E46B00204F
:1098F0002DE9F84F8046FFF7AFFF254E2549DFF8E9
:10990000A0E0254A254D844610274FF47A740120A3
:10991000DEF80430C3F30803D3B9EFF31183BBB906
:109920000B68D2F808A000BFD1F800904B45F7D1E2
:10993000D6F800B004FB0BF9A9EB0A09B9FBFBF957
:1099400004FB0393A3EB0C034345E1D3BDE8F88F7D
:10995000EFF3118A87F31288D2F808B01368DB039B
:1099600044BF2860D2F808B00B68D5F800905FFAC1
:109970008AFA8AF31188D6F800A0994404FB0AF306
:10998000A3EB0B03B3FBFAF304FB0933DAE700BFE5
:10999000EC6B0020E86B002010E000E0E46B00209E
:1099A00000ED00E02DE9F04FDFF830C1474A4849AB
:1099B000484E494D8046102718F1FF38C0F084808A
:1099C000DCF80430C3F30803002B5CD1EFF3118300
:1099D000002B58D10B68946800BF08688342F9D106
:1099E000D6F800904FF47A7000FB09FEAEEB040E3F
:1099F000BEFBF9FE00FB03EEDCF80430C3F3080302
:109A00004FF47A740120FBB9EFF31183E3B90B68CB
:109A1000D2F808A000BFD1F800904B45F7D1D6F896
:109A200000B004FB0BF9A9EB0A09B9FBFBF904FB35
:109A30000393A3EB0E03B3F57A7FBDD2DCF80430B9
:109A4000C3F30803002BDFD0EFF3118A87F31288EA
:109A5000D2F808B01368DB0344BF2860D2F808B01E
:109A60000B68D5F800905FFA8AFA8AF31188D6F865
:109A700000A0994404FB0AF3A3EB0B03B3FBFAF336
:109A800004FB0933D5E7EFF3118487F31288D2F88A
:109A900008901368D80303D501232B60D2F80890EF
:109AA0000B682868E4B284F31188D6F800A04FF45C
:109AB0007A7400EB030E04FB0AF3A3EB0903B3FB78
:109AC000FAF304FB0E3E97E7BDE8F08F10E000E0EC
:109AD000E86B0020EC6B0020E46B002000ED00E060
:109AE00030B4EFF31183102282F312880649074C39
:109AF0000A680748013200250A602560DBB2026867
:109B000083F3118830BC7047E86B0020E46B0020C1
:109B100010E000E00F4B1B88014643B90E4B0F4A83
:109B20001B7810680BB981F001010AF0E1BA0C4B07
:109B30005A691AB118B91A68106058747047094AFE
:109B400018681188084A92FBF1F2012102605974E9
:109B5000704700BFC06B0020C26B0020C46B0020A8
:109B6000C86B0020E06B002020A1070038B5264B11
:109B70005C69636B73B1A36DA26BD2B1998A1A88C9
:109B8000C90592B201D5D20700D438BD4FF6F7729D
:109B90001A8038BDA36D99891A88890692B2EBD5CF
:109BA0009206E9D5E26AD2B19888216B80B29047DB
:109BB000E1E799891A880D0692B2DFD51006DDD546
:109BC000A26A616A8A4219D0A1692569885C988075
:109BD0000132B2FBF5F105FB1122A262CEE79B88B0
:109BE000E2696169DBB28B54E269E068A36D01321E
:109BF000B2FBF0F100FB1122E261BDE7DA6822F06E
:109C00008002DA60BAE700BFA482002038B5264B94
:109C10009C68636B73B1A36DA26BD2B1998A1A88E9
:109C2000C90592B201D5D20700D438BD4FF6F772FC
:109C30001A8038BDA36D99891A88890692B2EBD52E
:109C40009206E9D5E26AD2B19888216B80B290473A
:109C5000E1E799891A880D0692B2DFD51006DDD5A5
:109C6000A26A616A8A4219D0A1692569885C9880D4
:109C70000132B2FBF5F105FB1122A262CEE79B880F
:109C8000E2696169DBB28B54E269E068A36D01327D
:109C9000B2FBF0F100FB1122E261BDE7DA6822F0CD
:109CA0008002DA60BAE700BFA482002038B5264BF4
:109CB0005C68636B73B1A36DA26BD2B1998A1A8889
:109CC000C90592B201D5D20700D438BD4FF6F7725C
:109CD0001A8038BDA36D99891A88890692B2EBD58E
:109CE0009206E9D5E26AD2B19888216B80B290479A
:109CF000E1E799891A880D0692B2DFD51006DDD505
:109D0000A26A616A8A4219D0A1692569885C988033
:109D10000132B2FBF5F105FB1122A262CEE79B886E
:109D2000E2696169DBB28B54E269E068A36D0132DC
:109D3000B2FBF0F100FB1122E261BDE7DA6822F02C
:109D40008002DA60BAE700BFA482002038B5264B53
:109D50001C68636B73B1A36DA26BD2B1998A1A8828
:109D6000C90592B201D5D20700D438BD4FF6F772BB
:109D70001A8038BDA36D99891A88890692B2EBD5ED
:109D80009206E9D5E26AD2B19888216B80B29047F9
:109D9000E1E799891A880D0692B2DFD51006DDD564
:109DA000A26A616A8A4219D0A1692569885C988093
:109DB0000132B2FBF5F105FB1122A262CEE79B88CE
:109DC000E2696169DBB28B54E269E068A36D01323C
:109DD000B2FBF0F100FB1122E261BDE7DA6822F08C
:109DE0008002DA60BAE700BFA482002070B4EFF30B
:109DF0001186502383F31288836B1A68D20720D40C
:109E00005D686DB9446A826A944217D081691144D1
:109E1000D9600ED9A21A5A608462002280F85C20B0
:109E20001A6842F00102F1B21A6081F3118870BC25
:109E3000704701698A1A5A608562EEE7012380F84B
:109E40005C30F3B283F3118870BC704703685B6ABF
:109E500003B11847704700BF03681B6A03B1184776
:109E6000704700BF03682DE9F041DF691FB13B4631
:109E7000BDE8F0411847002A164611DD04460D469C
:109E80000E4400E023689B68204698470028F9D0DC
:109E9000236815F8011B1B6820469847AE42F1D194
:109EA000BDE8F08103689B69184700BF03685B69E0
:109EB000184700BF03681B69184700BF0368DB68C9
:109EC000184700BF03689B68184700BF03685B68BA
:109ED000184700BF03681B68184700BF38B50C4619
:109EE000097849B1054601342B6828461B68984714
:109EF00014F8011B0029F7D138BD00BF10B40B4B7B
:109F00000B4A1C7801238340234052F8200031B9CA
:109F1000B3FA83F149095DF8044B0AF0E9B8191C5A
:109F200018BF01215DF8044B0AF0E2B8B06B0020C5
:109F3000B46B002008B501210220FFF7DFFF094BB9
:109F40001B7803F00503052B08D000210120FFF743
:109F5000D5FF00210846FFF7D1FFFEE724F0DCFA29
:109F6000F3E700BFA0820020064B53F820302BB14E
:109F70001A689B8851690B4201D113837047538340
:109F8000704700BFB46B00202DE9F04FBC4B1E782A
:109F90008BB0002E40F08180BA4BBB4C1D78BB4F7C
:109FA000DFF80CB305F00105A4F10A0954F80A0C16
:109FB000B8B14FF0CC0808FB0698FFF787FF80B1D7
:109FC00054F80A0CFFF77AFF14F8023C024683B9F2
:109FD00024283BD075B354F80A0CFFF777FF00280C
:109FE000EED10136032E04F1CC04DFD10BB0BDE875
:109FF000F08F012B2ED0022B33D0032B40D0042B1B
:10A0000000F06981052B00F05781062BE3D114F88D
:10A0100001ECBEF1000F00F0D881BEF1010F00F09D
:10A020001B8201360023032E04F8023C04F1CC0409
:10A03000BCD1DBE7232A54F80A0C00F08281944B50
:10A0400093F83A309342B8D137F07AFA012304F802
:10A05000023CC0E74D2800F06781002304F8023C71
:10A06000B9E700233C2804F8023C00F057813E2861
:10A07000B1D10122032304F8012C04F8023CAAE721
:10A08000C028EAD80021042304F8050C04F8040CC5
:10A0900004F8061C04F8023C9DE77E4B1868002873
:10A0A000A4D00AF092FADFF80CA27B4DDFF8F89109
:10A0B000DAF80000FFF70AFF002897D0DAF800006E
:10A0C000FFF7FCFE09281BD03F2819D02B68002B76
:10A0D00067D1042800F0BA810C2800F0CA807F28DC
:10A0E000E6D0A0F12002D2B25E2AE1D80BB9202836
:10A0F000DED05A1C09F803002A601FF0DBFBD7E70B
:10A100002C68002C5AD1654FA34607F52078BBF187
:10A11000000F08BFBB4610374745F8D1BBF1000F11
:10A1200000F04E81103FDBF800003A68065D135DD9
:10A130009E42204402EB040140F04081661E4E44E2
:10A1400022460BB9FD2A5CD906F8013F01322A608C
:10A1500010F8013F11F801EF9E45F2D00AB15F45BA
:10A1600012D04F481FF0AEFB5F4508D35BF8100BD1
:10A170001FF0A8FB09201FF09DFBBB45F6D94948FD
:10A180001FF0A0FB2A680024944291D2661E4E4420
:10A1900016F8010F1FF08EFB2B6801349C42F7D399
:10A1A00086E70C2865D00A2834D00D2832D07F28C5
:10A1B00000F0BE80FF2B3FF67BAF92E7374E0027C3
:10A1C00006F52078BB4602E0103646450DD0224603
:10A1D000316848460AF054FD0028F5D1B346002FF7
:10A1E000F2D1374610364645F1D13B465F469B4695
:10A1F000002B98D1002F3FF45BAF29481FF062FB82
:10A20000B4E7511C202009F80200296009F8013048
:10A210000A46A4E71FF0D7FB2321234839F010FC9E
:10A22000002800F01181A0EB0900286090B1431EC6
:10A2300019F80310202940F02C8109EB030243B1E7
:10A2400012F8011D202903F1FF304FD10346002BE6
:10A25000F6D12B604FF480720021484639F0D9FBCB
:10A26000074B1B78002B3FF4C1AE0E481FF02AFBB2
:10A270001EE70E481FF026FB0A481FF023FB17E7D6
:10A280004CB00020105100206E60002018250020E6
:10A29000208C0020906F002084320020106704087A
:10A2A0001C76040824760408843100202C760408E7
:10A2B000243B04088031002014F8063C14F8051CE7
:10A2C00099426FD814F8043C83427FF4C6AE06234B
:10A2D00004F8023C9BE614F8043C04F8030C5A40D2
:10A2E000052304F8042C04F8023C74E62B606A4C45
:10A2F000002204F5207809F8032002E010344445D8
:10A300004CD02168484614F03BF90028F6D044456B
:10A3100044D2E368984700232B609BE7032204F8AC
:10A32000013C04F8022C56E6022304F8023C52E6F3
:10A33000013B002259482B6009F803201FF0C2FAA4
:10A34000B6E6574B5749DB78574ADFF888E110608B
:10A35000003318BF01230B70544B554ACEF8003020
:10A36000544B7A604FF0400E012187F80CE03860C2
:10A37000B8607D73504819701FF0B8FE4F481FF049
:10A38000A1FA4FF4006011F02BFD4D4B93F83A30D9
:10A39000232B3FF459AE14F8023C36E649481FF02F
:10A3A00091FAB8E714F8041C08EB0300514001339C
:10A3B00004F8041C04F8063C82720CE62246CDE642
:10A3C0004148103F1FF07EFAD0E69BE80F000DF1E8
:10A3D000280C0DF1080888E80F004CF824ED14F85B
:10A3E000053C14F803AC0694624623444FF0010C7C
:10A3F000414606A8ADF822E00793ADF820A08DF8FD
:10A4000024C000F069F840B1029A304B03924146F3
:10A41000A4F10A00029328F0C9FADDF804800023B1
:10A4200004F8023CB8F1000F3FF4DBAD54F80A0C1D
:10A4300028F07CFB013654F80A0CC047032E04F1C7
:10A44000CC047FF4B3ADD1E52868EFE6204813F0E3
:10A450003BF80BB0BDE8F08F14F8053C14F8032C62
:10A460000694234407936E2A4FF000030893099340
:10A47000ADF820207FF4D5AD06A80AF080FC06A830
:10A480000AF072FC06A80AF06FFC06A80AF06CFC41
:10A49000C7E503462BE700BF10670408547604089D
:10A4A0006C8C0020F0700020803100201C250020E2
:10A4B000018200084CB00020587604082476040875
:10A4C000208C0020387604081C760408ACBC0020E0
:10A4D00084310020906F00202DE9F04F9BB0B0F93F
:10A4E00008500D81EDB2442D00AF0C46904600F0AF
:10A4F000D782064643D9812D00F0108200F2998060
:10A50000542D00F0CE8040F2F5816E2D00F0968241
:10A51000802D40F02481C54B93F800A00AF1020A77
:10A520001AF0FF0A00F09980C14BDFF83C83C14E5E
:10A53000DFF838B39A4403F101090A2516E0322DF9
:10A5400000F0DD82A5F13C00C0B2132840F2DD82AC
:10A5500000232268511C216015702268D14502F148
:10A5600001012160137078D019F8015B0A2DE6D142
:10A57000BBF80030FF2BA8BFFF23DBB2E9E7052DB6
:10A5800000F07C8220D8022D00F0838040F29F8171
:10A59000032D00F04A82042D40F0E1802A46A649AE
:10A5A00020460AF0F1FB002120460AF032FC226826
:10A5B0000221531C0125236028462B466C3711705D
:10A5C0006381BD46BDE8F08F242D60D040F20F813D
:10A5D000282D00F0EC81382D40F0C1800A68974B9F
:10A5E0000125511C21601570226805215019206039
:10A5F000117022680A215019206011702268002110
:10A60000501920601170226819785019206011705B
:10A61000226859785019206011702268997853196E
:10A6200023602B46117028466C376381BD46BDE818
:10A63000F08FA02D19D040F21F81B82D00F0F381CA
:10A64000FE2D40F08C807E4D05F1080635F8021B8A
:10A6500020460AF0DEFBB542F8D101252B462846FC
:10A660006C376381BD46BDE8F08F764B08461968AC
:10A670000AF0B8FB744B204619680AF0B3FB734B21
:10A680001968204601250AF0ADFB2B46E7E7704B21
:10A69000F6E704226F49204601250AF075FB2B4698
:10A6A000C1E70B686C4ADFF8C881581C1121206093
:10A6B000197023681278591C21601A70236898F861
:10A6C0005520591C21601A70236898F85420591C91
:10A6D00021601A70B8F8501020460AF09AFB2368DF
:10A6E0000022591C21601A7023682822591C2160FD
:10A6F0001A70B8F8521020460AF08BFBA8F1020538
:10A7000008F14E0635F8021F20460AF082FBB542DA
:10A71000F8D12268514B0D21501C20605D1811703A
:10A72000226813F8011F501C9D4220601170F7D160
:10A7300023680222591C21601A70B8F8561020466E
:10A740000AF067FBB8F8581020460AF062FB0125B2
:10A75000B8F85A1020460AF05CFB2B4663E7214606
:10A76000284610F079FA034600287FF476AF742D5E
:10A7700000F0C680772D0DD13268716891421EBFFE
:10A78000531C33601178364A08BF1946204632F010
:10A7900071FC62E7F52D01F0B383762D00F088811E
:10A7A000472D00F02682392D326800F0E78200F252
:10A7B0000582212D01F08483292D40F01B83531C39
:10A7C000336013780A2B01F04784502B41F0478304
:10A7D00030460AF0C9FADFF89C80A8F8000030463D
:10A7E0000AF0C2FA0125A8F802002B461BE7202D2B
:10A7F000B5D10B681B4D591C6A7821601A7023680B
:10A800002A78591C21601A702368AA78591C216083
:10A810001A70298920460AF0FCFA23686A79591CC3
:10A8200021601A702268A979C3E600BFA1B900208F
:10A83000343B040830700020728C0020AF99002057
:10A84000246C0020107AFF1F147AFF1F187AFF1F54
:10A85000F49A002090760408306C00207D4000209F
:10A8600071C1030814B7002067666666587000203F
:10A870002040002018700020822D7FF470AF0B68FC
:10A88000BA4ABB4D1178BB4A581C20601970118917
:10A8900020460AF0BEFAB84B22681B88FF2B02F153
:10A8A0000101A8BFFF2321601370A96881F3100183
:10A8B00089B220460AF0ADFA296801F30F0189B286
:10A8C00020460AF0A6FAAD4B2268197871E6012DF0
:10A8D0007FF445AF0B680022591C21601A70236871
:10A8E0005A1C22601D7022682521531C23602B46B0
:10A8F000117098E6522D7FF432AF2268002158E69D
:10A900003268716891421EBF531C336011789C4AB3
:10A9100008BF1946204632F0ADFB9EE6994B1E78E3
:10A92000033616F0FF063FF498AE974BDFF88482AB
:10A930001E4403F1010A4FF00A0920E0B9F1500F5B
:10A9400000F0DB80B9F1320F00F0F480A9F13C0097
:10A95000C0B2132840F2F1800025294623685A1C12
:10A960002260204683F800900AF053FA29462046D8
:10A970000AF04FFAB2453FF470AE1AF8019BB9F1F4
:10A980000A0FDBD1814B9D68196805EB85054FF6F1
:10A99000FF736D009D42A8BF1D469942A8BF19468E
:10A9A00025EAE57521EAE171ADB289B2D6E70B6817
:10A9B000DFF80492764E591C022221601A70236837
:10A9C0004FF006085A1C226083F8008023680A2290
:10A9D000591C21601A70236801255A1922601D70C4
:10A9E000B9F8001020460AF014FAB9F8021020460F
:10A9F0000AF00FFA23685A19226083F8008023684E
:10AA00005022591921601A702368002259192160B7
:10AA10001A70318820460AF0FCF9718820460AF045
:10AA2000F8F92B46FFE55B4B2AE60B685A1C0A60D7
:10AA30001D700B685A1C0A601D705EE74E4B0A6859
:10AA40001B884B4DFF2BA8BFFF23511C21601370A7
:10AA5000A96881F3100189B220460AF0DAF94E4B59
:10AA6000204619880AF0D5F9296801F30F0189B247
:10AA7000204601250AF0CDF92B46D4E50B224749A3
:10AA800020460AF081F90822454920460AF07CF95F
:10AA900001250722434920460AF076F92B46C2E5F4
:10AAA000002A3FF4DAAD404B136001252B46BAE58E
:10AAB0003268511C31601278002A01F0D482102AC9
:10AAC00001F02D831D4619462368581C20601A701A
:10AAD00020460AF087F9294620460AF083F9334BCD
:10AAE000204619680AF07EF9204600210AF091F903
:10AAF000002120460AF08DF9FFE62D4B43E733880D
:10AB0000FF2BA8BFFF23DBB223E534F089F900282F
:10AB10003FF41EAD03780A2B25D8B0F9023088FB2C
:10AB20000312DB17C3EBA2039BB2FF2BA8BFFF23CB
:10AB3000DBB20EE598E8220027E734F071F900282F
:10AB40003FF40AAF03780A2B3FF606AFB0F90430A2
:10AB5000B0F9061003EB830383F3500521EAE1719A
:10AB6000ADB289B2FAE60023E2E700BFA6BA002040
:10AB7000FCB6002014B7002090BA00208C400020C2
:10AB800085C20308A1B90020443B0408E46F0020FB
:10AB900018700020586E0020544200209876040857
:10ABA000A4760408B076040839AC0108D43000203B
:10ABB0001C7000202870002030990020552D00F0D6
:10ABC000ED80572D40F01681531C336012F8370B7F
:10ABD00007F127010133336013F8015C01F8015FCD
:10ABE0009342F7D107F12801012505F06BF92B46B7
:10ABF00019E5726835687B623046551B0AF09DF88E
:10AC0000052D38627B6A01F21A828026B34601253F
:10AC100094E80600521A103AB242B8BF1FFA82FBFB
:10AC2000714A396A92683A61521A9345396A7B626D
:10AC30002046FA6088BF1FFA82FB0AF0D3F87B6ACD
:10AC4000002B01F0DB81002D41F0B7812368C7F8AC
:10AC500000D05D71C0B00533C7F804D0FB61BBF113
:10AC6000000F01F074833B6A3A69934281F06B8371
:10AC70003E6A7D62AA46A846BC608025FB68A3EBBD
:10AC80000808594BB8F5807F9B6828BF4FF480783F
:10AC900008EB06029A4288BFA3EB06080AF002FFFF
:10ACA0007C684246214630460AF082FFF969B86165
:10ACB00004EB000C0B787B6164452ED2DFF83091F9
:10ACC0000CF1FF3C04F1FF3E1EF8013F09EB83024B
:10ACD00019F823405688ECB100234FF4004204F1E8
:10ACE000FF3832424FEA520202D0087828430870F7
:10ACF0006D0806D10AF1010A4D701FFA8AFA013176
:10AD00008025D34503D8F44532D8434530DB0133A1
:10AD10009C42E6D1F445D7D1F9617B6ABA69134404
:10AD20009BB2D3457B6206D97B6A3A6A9846D618AD
:10AD30003B699E42A2D3BC68802D1CBF0AF101036F
:10AD40001FFA83FA0AF1020189B220460AF061F87B
:10AD50002368796A01255A19226020461D700AF07D
:10AD600058F82368534423602B46D7F800D05AE4A0
:10AD7000FB69BC681A463B7D1370DDE7531C3360EA
:10AD800013780A2B01F09D81304609F0F8FF304618
:10AD900009F0F5FF304609F0F2FF5EE4531C336022
:10ADA00092F80080B8F1FF0F01F0DA81B8F1FE0FE0
:10ADB00001F0A281304609F0D7FF33687268D21AD9
:10ADC000002A07DD5A1C32601B781BB9B8F10C0F42
:10ADD00041F2AA81B8F1270F00F2B782034B012597
:10ADE00023F818002B461EE4080300202040002012
:10ADF000543B040871680B3D8B1AEF2D00F2A582BD
:10AE000001A050F825F000BFC9BC00084BB30008F2
:10AE10004BB300084BB300084BB300084BB300081A
:10AE20004BB300084BB300084BB300084BB300080A
:10AE30004BB300084BB300084BB300084BB30008FA
:10AE40004BB300084BB300084BB300084BB30008EA
:10AE50004BB300084BB300084BB300084BB30008DA
:10AE60004BB300084BB300086FBC00084BB300089D
:10AE70004DBC00084BB3000823BC00084BB30008CE
:10AE80004BB300084BB30008FBBB00084BB30008F2
:10AE9000A1BB00084BB3000831BB00084BB300084E
:10AEA0000BBB00084BB3000803BE00084BB30008FF
:10AEB000ABBD00084BB300082BBD00084BB3000826
:10AEC0004BB300084BB300084BB300085BA6000867
:10AED0004BB30008FFBC00084BB300084BB300089D
:10AEE0006FBE00084BB3000815BE00084BB3000846
:10AEF0004BB300084BB300084BB3000889BE0008F1
:10AF00004BB300084BB300084BB30008CBBA0008A2
:10AF10004BB300080BBA00084BB300084BB3000852
:10AF2000A3B900084BB300084BB300084BB30008AB
:10AF30004BB300084BB300084BB300084BB30008F9
:10AF40009DB800084BB3000829B800084BB30008AF
:10AF500059BA00084BB300080BB900084BB30008FE
:10AF6000E3B90008C7B70008ABB700084BB3000847
:10AF70004BB300084BB300084BB300084BB30008B9
:10AF80004BB300084BB300084BB300084BB30008A9
:10AF90004BB300084BB300084BB300084BB3000899
:10AFA0004BB300084BB300084BB300084BB3000889
:10AFB0004BB300084BB300084BB300084BB3000879
:10AFC0004BB300084BB300084BB300084BB3000869
:10AFD0004BB300084BB300084BB300084BB3000859
:10AFE0004BB300084BB300084BB300084BB3000849
:10AFF0004BB300084BB300084BB300084BB3000839
:10B000004BB300084BB300084BB300084BB3000828
:10B010004BB300084BB300084BB300084BB3000818
:10B020004BB300084BB300084BB300084BB3000808
:10B030004BB300084BB300084BB300084BB30008F8
:10B040004BB300084BB300084BB300084BB30008E8
:10B050004BB300084BB300084BB300084BB30008D8
:10B060004BB300084BB300084BB300084BB30008C8
:10B070004BB300084BB300084BB300084BB30008B8
:10B080004BB300084BB300084BB300084BB30008A8
:10B090004BB300084BB300084BB300084BB3000898
:10B0A0004BB300084BB300084BB300084BB3000888
:10B0B0004BB300084BB3000881B700084BB300083E
:10B0C00065B700083BB700084BB300084BB3000856
:10B0D0004BB300084BB300084BB300084BB3000858
:10B0E0004BB300084BB300084BB300084BB3000848
:10B0F0004BB300084BB300084BB30008DDB60008A3
:10B100008BB6000853B600084BB30008B1B5000871
:10B110007DB5000861B500084BB3000897B500087D
:10B12000F5B4000887B4000875B4000819B4000825
:10B130004BB30008E9B300084BB300084BB3000859
:10B14000BFB3000891B300087DB3000855B30008F1
:10B150002DB3000803B30008D7B20008BFB200083F
:10B160004BB300084BB300084BB300084BB30008C7
:10B170004BB300084BB300084BB300084BB30008B7
:10B180004BB300084BB300084BB300084BB30008A7
:10B190004BB300084BB300089FB200084BB3000844
:10B1A0004BB3000847B200084BB300084BB300088C
:10B1B0004BB30008E3B100084BB300084BB30008E1
:10B1C0004BB30008C9B10008B94B1B78DB0700F18D
:10B1D000BC800125FDF7A8F9FDF780FB2B46FFF7A2
:10B1E00022BA304609F0C0FD336838851A46591C2A
:10B1F000316012F8021B326087F82A105A7887F8FB
:10B200002B20DA1C32609A7887F82C201A1D3260C5
:10B21000DA7887F82D205A1D32601B7987F82E3096
:10B2200007F1280000233B8609F0F8FCA14AA24B55
:10B230001268801A4FF0010561F10001C3E90601AF
:10B240002B46FFF7F0B9531C336013780F2B7CD8D3
:10B25000911C3160C3EBC30398495078C854D01C8B
:10B2600030600B4491785970111D3160D17899701C
:10B27000511D31601179D970911D31605179197169
:10B28000D11D31609179597102F108013160D27993
:10B290009A7101251FF070FD2B46FFF7C4B93046A7
:10B2A00009F062FDDFF82482A8F80E00304609F0AC
:10B2B0005BFD0125A8F80C002B46FFF7B4B930461A
:10B2C00009F052FD7E4A00EB800043000125138007
:10B2D0002B46FFF7A8B91146531C3360794B11F880
:10B2E000020B1870316051785970D11C316091781F
:10B2F0009970111D3160D278DA7001252B46FFF765
:10B3000092B9304609F030FDDFF8D881A8F8100076
:10B31000304609F029FDA8F81200304609F024FD56
:10B320000125A8F814002B46FFF77DB91346511CE0
:10B33000316013F8020B3360D31C5178336092787C
:10B340001BF0CCFF00287FF488A94FF0FF352B4677
:10B35000FFF769B91346511C31605B4913F8020BC2
:10B3600008703360594953788B70D31C3360544B49
:10B3700092789A7001252B46FFF755B9544B5549E1
:10B3800018684E22012537F0B1F92B46FFF74BB96B
:10B390001146531C3360504B11F8020B187031608A
:10B3A00051785970D11C316092789A70304609F00A
:10B3B000DBFC4A4B0125D8802B46FFF734B93046D9
:10B3C00009F0D2FCDFF81481A8F80000304609F03B
:10B3D000CBFCA8F80200304609F0C6FC0125A8F80D
:10B3E00004002B46FFF71FB9DFF8FC9099F80030F6
:10B3F000002B3FF432A9DFF8F4800025304609F035
:10B40000B3FC22F075FF99F80030A8EC010A013571
:10B410009D42F3DBFFF721B90D2B96D1531C33600E
:10B420001578072D91D8DFF8C89030464FF00C08FA
:10B4300009F09AFC08FB05F809EB0805A8803046DE
:10B4400009F092FCE880304609F08EFC33682881D0
:10B450001A46591C316012F8021BA97232605B78DF
:10B46000EB72304609F069FC012549F808002B46CB
:10B47000FFF7D9B8304609F077FC194B0125188041
:10B480002B46FFF7D0B8531C33601078060600F146
:10B490000387074B1B78DD073FF5DFA8032828BF8C
:10B4A00000200125FDF724F82B46FFF7BCB800BFAC
:10B4B00010510020E86B0020682500206C6D0020F2
:10B4C00050990020D83C0020508D00204099002049
:10B4D00084B70020CC63040838990020046A002057
:10B4E000F43F0020FC530020A1B90020603100206F
:10B4F000AC6C0020531C3360304692F800A009F079
:10B500001CFC8146304609F018FC0546304609F01F
:10B5100014FC8046304609F027FC304609F024FC34
:10B52000304609F02CFCBAF1000F00F09E86BAF10B
:10B53000100F7FF492A8AB4BC3F804909D60B8F154
:10B54000000F02D0A84BC3F80080A849A84B0222E4
:10B55000081F01251A7028F091FF2B46FFF763B8EA
:10B56000A44B1B78DA073FF578A8A34A1378012586
:10B5700043F0040313702B46FFF755B89D4B1B781F
:10B58000D9073FF56AA89D4B4FF4C87201251A8070
:10B590002B46FFF748B8974B1B78D8073FF55DA8B7
:10B5A0000125FDF771FBFDF799F92B46FFF73BB835
:10B5B000092B7FF7CAAEDFF868821346511CD8F812
:10B5C0000050316013F8021B297033605378AB7060
:10B5D000D31C33609378642B02F10401A8BF642369
:10B5E0006B713160D378642B02F10501A8BF64232D
:10B5F000AB7131601379EB71931D33605379642B18
:10B6000002F10701A8BF64232B7231609379EB70BC
:10B6100002F108033360D3792B71304609F0A4FBA3
:10B62000726833686881D11A00290CDD591CD8F87A
:10B6300000003160521A002A1978417203DD9A1C09
:10B6400032605B784370012523F04CFC2B46FEF7FB
:10B65000EABF6B4B1868D31C014621329D1E356032
:10B6600013F8035C0D705D1E356013F8025C4D70BD
:10B67000336013F8015C8D700333934201F10301D1
:10B68000ECD122F0DFFCFEF7E8BF531C33601378E7
:10B690005949002B00F098850B7843F00203901C69
:10B6A0000B70584D306053782B75304609F045FBD0
:10B6B0002860304609F041FB6860304609F054FBD1
:10B6C0002881304609F050FB4F4AE8811378012564
:10B6D00043F0020313702B46FEF7A5BFC3F34705E3
:10B6E000122D3FF632AEC5B107F1680307F1260A05
:10B6F00003EB4508D146A8F14208304609F034FB77
:10B7000029F8020FC845F8D1404B3AF8022F23F828
:10B71000022FD145F9D1112D09D83D4A6B00023BCA
:10B7200013440021223223F8021F9A42FBD1394AE6
:10B7300001231D461370FEF776BF531C3648336055
:10B7400001781378002940F03A8504220270334AC8
:10B750009B001380FEF780F8224B012518622B46D0
:10B76000FEF761BFDFF8BC8000233046C8F8003028
:10B7700009F0E3FA0125C8F800002B46FEF753BF95
:10B780001346511C316013F8025B3360D31C5078B0
:10B7900033609178002D00F00986012D7EF45DAFB5
:10B7A00017F08EF92B46FEF73EBF531C336013781B
:10B7B000002B00F09A854FF40040012510F010FB9B
:10B7C0002B46FEF730BF0B4B1B7813F001017FF4C3
:10B7D000BCAD531C33601078012517F0B7F82B4629
:10B7E000FEF721BF68250020D430002070250020FE
:10B7F000E83E00201051002082B7002084BC0020C9
:10B8000084B70020C0570020E63E00207E33002091
:10B8100080330020A4330020E43B00205442002069
:10B8200088B70020586E00201346511C3160DFF8A5
:10B83000648313F8021B88F802103360C9495378F7
:10B840000B70D31C3360C84D93782B71131D33607C
:10B85000D378092BA8BF09233046AB7009F084FACE
:10B86000336872682880D11A012905DD304609F055
:10B870007BFA33687268E8819A4240F09D85FCF754
:10B8800085FF336872689A423EF4E7AE5A1C326014
:10B890001B78EB7001252B46FEF7C5BEB34B1B682A
:10B8A000002B3EF4DAAE28F0E1FEFF283EF4D5AEE0
:10B8B000304609F059FA3F2840F20785DFF8D88270
:10B8C000002588F8005033687268A8F80400D21A7E
:10B8D000012A7EF7C2AE1A46591C316012F8021BCB
:10B8E00088F8021007F16800326000225D7800F8E5
:10B8F000402D28F08DFE97F82830AB423EF4ADAED7
:10B90000284628F0A9FEFEF7A8BE304609F02CFA1A
:10B91000304609F029FA304609F026FA304609F097
:10B920002EFA3368924D1946581C2A68306011F877
:10B93000020B82F82C003160597882F83610D91C3D
:10B9400031609B7882F83730304609F018FA30467B
:10B9500009F015FA304609F012FA3046D5F80080A1
:10B9600009F002FAA8F83A003046D5F8008009F04C
:10B97000FBF933687268A8F83800D11A01290ADD8A
:10B98000591C2A6831601B7882F82E30304609F045
:10B99000F6F933687268D31A032B00F38884286899
:10B9A0006FE6744B1B78012B3EF657AE1046531CC6
:10B9B0003360DFF8E88110F8023B88F8023030602D
:10B9C000D31C50783360CB1A012B917840F39684C6
:10B9D000304609F0C9F90125A8F800002B46FEF70A
:10B9E00022BE1346511C3160634913F8020BC87024
:10B9F0003360624953784B71D31C3360604B92784B
:10BA0000DA7001252B46FEF70EBE531C336092F808
:10BA10000080B8F1110F3FF698AC931C3360594D7C
:10BA2000537805F81830304609F09EF940F6CA03FD
:10BA30009842A8BF184640F2EE23984205EB480111
:10BA4000B8BF18460125A0F2EE222B46192092FB22
:10BA5000F0F24A70FEF7E7BD531C3360444DDFF847
:10BA60003481137888F805303046D5F8009009F015
:10BA70007BF9A9F820003046D5F8009009F074F958
:10BA800072683368A9F81E00D11A072900F372847E
:10BA9000D11A032900F36084D21A002A05DD591C4B
:10BAA0002A6831601B7882F82630FCF76FFE2AF096
:10BAB000CFFC354B1B68002B00F02C842868012537
:10BAC00021F0F0FE2B46FEF7AEBD1346511C2F4D64
:10BAD000316013F8021B2971336053786B71304663
:10BAE00009F042F9336828805A1C32601B78AB7128
:10BAF000304609F039F9336868805A1C32601B7887
:10BB0000EB7101252B46FEF78EBD511C3160157877
:10BB10001F2D3FF61AAC052B7FF417AC304609F009
:10BB20000CF91B4B43F8250019F0F0FFFEF795BD0B
:10BB3000174D05F14008304609F016F93368A5F8AD
:10BB40008000591C1A46316012F8021B85F88210D9
:10BB500032605B7885F883300435A845EBD1FEF779
:10BB60007CBD00BF34990020FC53002014510020FC
:10BB700084B70020E29A00204099002048B90020B4
:10BB8000509900205036002068990020206A00203B
:10BB9000AC400020508D002018510020304F002074
:10BBA000531CBC4D336013782B72304609F0DCF81F
:10BBB000A883304609F0D8F82883304609F0D4F835
:10BBC00032686883531C33601278EA747268D31A3F
:10BBD000032B00F32B833368D11A052900F3168356
:10BBE000D21A002A7EF739AD5A1C32601B7885F8CC
:10BBF000213001252B46FEF716BD531C3360A648A5
:10BC000015780570C91A00297EF727AD931C33609B
:10BC10005378003318BF0123012543702B46FEF7EC
:10BC200002BD304609F0A0F8DFF88882C8F80000AD
:10BC3000304609F099F8C8F80400304609F094F845
:10BC40000125C8F808002B46FEF7EDBCDFF86C8232
:10BC50000023C8F80030304609F06FF8D8F80030FB
:10BC600001250343C8F800302B46FEF7DCBC531C0B
:10BC700033601578132D3FF668AB931C3360507812
:10BC80007A6231F031FA00283FF45FAB7A6A834B75
:10BC9000017803F82510D11C316003EB85039178FE
:10BCA0005970111D3160D1789970511D3160127930
:10BCB000DA70002023F056F8794B80F0010001255E
:10BCC00018702B46FEF7AFBC764A102B4FF00001E0
:10BCD00028BF1023116051609160D1601174002B56
:10BCE0003EF4BBAC3168013A0B440131316011F8CC
:10BCF000010C02F8010F9942F7D1FEF7AEBC1346D2
:10BD0000501C3060684813F8025B857033605578CA
:10BD100045708B423EF4A1ACD31C3360634B9278E8
:10BD20001A7401252B46FEF77EBC0721B3FBF1F107
:10BD3000C1EBC1055B1B7FF408ABC9B201F1FF3950
:10BD40005FFA89F900293EF488AC09F101091D4622
:10BD5000531C336092F900A0504630F075FE013557
:10BD6000804600283FF4F1AA80F802A0304608F08F
:10BD7000FBFF3368A8F800001A46591C316012F81E
:10BD8000021B88F8031032605A7888F80420DA1C05
:10BD900032609A7888F806201A1D3260DB7888F8BD
:10BDA00005304D45D4D1FEF758BC531C3360137891
:10BDB0000E2B3FF6CAAA911C31605578032D3FF631
:10BDC000C4AA3B48062101FB03F1431802F1030E0C
:10BDD0005D71C6F800E095784554111D3160D17849
:10BDE0005970511D316011799970911D31605179EF
:10BDF000D970D11D316092791A7101252B46FEF759
:10BE000012BC531C3360234B12785A7501252B4604
:10BE1000FEF709BC531C33601F4B1278DFF89C807F
:10BE20001A700023C8F80030304608F086FF3368E7
:10BE3000D8F8002017491F4D10435A1CC8F80000BD
:10BE400032601B780B72304608F08EFF2860304657
:10BE500008F08AFF6860304608F086FFA860304628
:10BE600008F082FF304608F07FFFFEF7F6BB124B6A
:10BE700002F108010132326012F8010C03F8010FDF
:10BE80008A42F7D1FEF7E9BB012509F06DFE2B468A
:10BE9000FEF7C9BBF48B00207099002044350020C8
:10BEA000372300200A4F00206099002068250020D9
:10BEB000646E00204C830020F38B0020F49A002055
:10BEC0001346511C3160C34D13F8021B6970336077
:10BED00053782B70D31C33609378AB70304608F0E6
:10BEE00043FF33682881591C1A46316012F8021B3F
:10BEF000697132605B78AB7101252B46FEF793BB0D
:10BF0000336872689A4240F0B380B34BFF221A70D4
:10BF10004FF0000AB14D15F0A1FB51462022B04868
:10BF200085F800A037F075FD87F828A097F828302D
:10BF3000072B00F24281DFF8CC92A94E524697F8C7
:10BF4000283003EB430309EBC3035B7CE3B197F8B1
:10BF5000283003EB430309EBC30320215B699BB14A
:10BF600097F8283003EB430309EBC303586946F8FD
:10BF7000220007F0FBFF2B7856F8230008F0B3F8F7
:10BF80002A780132D2B22A7097F828300133DBB216
:10BF900087F8283097F82830072BD0D92368591C08
:10BFA00021601A70B8F1000F3EF457AB8D4BC8F802
:10BFB000003001252B46FEF736BB8B4B3A6A9B6857
:10BFC000D4F800905A449A4200F2B98009F06AFD10
:10BFD0005A464946386A09F0EBFD2368034423605A
:10BFE000B042BEF63AAB002100E0236801305A1C93
:10BFF000B04222601970F8D1FEF72FBB002DDCD1C2
:10C000005946204608F005FF23685A1C22601D701F
:10C01000754B26689D683B6A0BEB0302AA4240F20F
:10C0200084813B6AED1A09F03DFD2A463146386AA3
:10C0300009F0BEFD236803442360FEF70EBB3046C3
:10C0400008F092FE326871687B6A9142834649D15A
:10C0500006461D46FEF7DCBD304608F085FEDFF8DB
:10C06000A881FEF7BABB614B93E82200FEF72CBD16
:10C070005A1C19463260584811F8022B0270316080
:10C080005B784370042A03D9FF2A7EF436AC3FE77D
:10C0900057490978994205D8022A7EF42EACFF2B25
:10C0A0007EF42BAC236801255A1922601D70B8F16B
:10C0B000000F3EF4D2AA4F4BC8F800302B46FEF7D3
:10C0C000B2BA931C33604C4B51781970D11C31605B
:10C0D00091785970111D3160D2789A7001252B46E4
:10C0E000FEF7A1BA511C316012781D46131C06469A
:10C0F00018BF0123FEF78CBD931C33605578022DC9
:10C100003FF623A9304608F02FFE3C4B03EB4503D6
:10C110004FF0FF35A3F856002B46FEF784BA2E4B9E
:10C1200059689D68FEF7D0BC344B0030984418BF66
:10C130000120012588F85E002B46FEF774BA3A6AA2
:10C14000A3EB020809F0AEFC42464946386A09F002
:10C150002FFD236803442360002D3EF47EAA3FE7B1
:10C16000931C3360264B51781970D31C3360DFF871
:10C170008C80937888F85530131D3360D37888F815
:10C180005430304608F0F0FDA8F85000304608F072
:10C19000EBFD304608F0E8FD96E80C009B1A012BF9
:10C1A000A8F852007EF759AA304608F0DDFD0125B7
:10C1B000A8F85A002B46FEF736BA5246EEE6042996
:10C1C0007EF44BAAFFF7C3BA0B7803F0FD03FFF729
:10C1D00066BA00BF14B70020682500208D6F0020CC
:10C1E000A8340020B517030808030020DC3E002017
:10C1F000A1B9002045AC0108AF99002020400020E3
:10C20000306C00203C530020309900205A1C3260D2
:10C210001B78EB72304608F090FD3368E8605A1CDA
:10C2200032601B782B7433687268D9E4304608F0AA
:10C230009BFDA884304608F097FD33687268E88457
:10C24000D11A03297FF7C8AC1A46591C316012F87D
:10C25000021BA97732605B7885F82030304608F001
:10C2600083FD336872686884B6E4584B1020C3F8C5
:10C2700000905D600FF084FD554A137843F0010390
:10C280001370B8F1000F3EF4E8A9524B0125C3F832
:10C2900000802B46FEF7C7B900F07F00032828BFB7
:10C2A0000020012516F028FC2B46FEF7BCB93046CD
:10C2B000D5F8008008F058FDA8F8320030462E6806
:10C2C00008F052FDB086FFF76ABBC50800F007030F
:10C2D00001350133EDB2DFF818812846194688F898
:10C2E000013032F009FDFFF7ECBA3B4A1368012533
:10C2F00023F4004313602B46FEF795B9374B1A8899
:10C30000012512FB00F22B4692FBF1F2A8F8002067
:10C31000FEF789B932483349334A344B036001256B
:10C320000B6013602B46FEF77EB909F0BBFB5A4643
:10C330003146386A09F03CFC236801250344236038
:10C340002B46FEF770B97D62AA46FEF7FBBCDA46C3
:10C35000C7F824B0FEF7F6BC304608F005FDA8F893
:10C360000E00304608F000FD33687268A8F810002F
:10C37000FFF792BB304608F0F7FCA8F80A003046F9
:10C3800008F0F2FCA8F80C003046D5F8009008F050
:10C39000EBFCA9F822003046D5F8009008F0E4FC48
:10C3A00033687268A9F82400FFF772BB012521F0F9
:10C3B000CDFC2B46FEF737B95A1C32601B78003390
:10C3C00018BF012388F80730FFF759BADC3E002078
:10C3D00082B70020D43000207CB70020AE97002028
:10C3E000A8640020FC640020FC6800207B37010862
:10C3F000185100202DE9F04F2DED028B95B0064627
:10C4000031F0D8FC9E4B1D7825B115B0BDEC028BE8
:10C41000BDE8F08F9B4B1B685805F6D5DFF8B0924E
:10C42000D9F80020002A00F02781974CD4F8283151
:10C4300003F5F43348339E42C0F01E81934F94F8C5
:10C440002C113B68C4F82861013184F82C1199073C
:10C4500001F1798713F0140F41F0178713F0080FDB
:10C4600094F82C3140F0C28113F0070801F0BA852E
:10C47000282B874B029302F0B1805E209047854BBA
:10C480001B78002B6BD0804C834AD4F83431F31ADC
:10C49000934201F24384DFF83CA29AF80080B8F19D
:10C4A000000F33D1DFF80092D9F80000FDF70EFD40
:10C4B000C0B201280ED90228784F42F04F813B7854
:10C4C000002B42F02A82D4F83C31F31AB3F57A6F8C
:10C4D00082F0D58272480768002F40D09AF8003069
:10C4E000BBB9704BD9F800001B689B781E3B012B31
:10C4F0004FF0020142F26882043031F013FB012256
:10C5000000238AF8002084F8483126E06448076850
:10C510002FB3D4F8443140F6B732F31A93421ED900
:10C5200094F84031002B02F00F81013BDBB284F81C
:10C530004031002B01F0978717F8011B94F8482130
:10C54000076094F8493158480A440133006884F878
:10C55000482184F84931FDF7BDFCC4F84461534AD1
:10C56000029B12781B68012A03F101030C9301F06E
:10C57000FF824F4B1B787BB1DFF85C91D9F800301C
:10C5800053B1414C029BD4F85C21D3F800B0ABEB23
:10C590000202632A01F21A82DFF8408198F800A0B3
:10C5A000BAF1020F01F03A873C4F97F87430032B31
:10C5B00001F0DC843F4B1B7873B13F4D2B685BB1BE
:10C5C000314CFDF749F9D4F86831039044F61F6205
:10C5D000C31A934200F26081384B1B78002B7FD145
:10C5E000374B1B7843B1284CD4F8B83203F50043DD
:10C5F000E8339E4281F03283324B1B78002B3FF4AC
:10C6000004AF214E304C314D06F2C1272068FDF7B2
:10C610005DFC00283FF4F9AE2068FDF74FFC2B7855
:10C6200080465A1E33B120682A70FDF74FFC00285F
:10C63000F2D1EAE603223946781E37F0D0F996F8AF
:10C64000C03296F8C12286F8C38283F47F4383F018
:10C65000FF039B1A1FFA88F89BB2B8EB132FD5D1B2
:10C6600096F8C222DBB29A42D0D1781E32F058FC42
:10C670002B7818442870C9E7054B0293FFE600BFEA
:10C680004CB00020509500209825002024B70020B1
:10C69000E86B002036B800203F0D030000000020AA
:10C6A0009CB7002098B7002094B7002037B800202E
:10C6B00044B800204CB8002050B80020BCB800207E
:10C6C000CDB8002056B800205CB8002060B800202B
:10C6D000A4B70020A0B7002064BC00209E34002036
:10C6E000604C2278002A41F03A82DFF8A49199F850
:10C6F0000040002C40F0AB805B4D2878002842F0D1
:10C700008C805A4C5A4DD4F8B0222978594B93FB5F
:10C71000F1F313449E42FFF463AF94F8B432564AE7
:10C72000C4F8B062D75CFB0702F17482B80702F16B
:10C73000E981790702F12A823A074CD54F4BDFF89D
:10C7400054810D930DF15009A3F13D0249F8202DBC
:10C750000021A3F1400203F8401C02231121517073
:10C7600093704846D8F8001008F018FB4846D8F8EF
:10C77000041008F013FBB8F80E30414903EBC30373
:10C780009B00053381FB0321DB17C3EBA10189B2B9
:10C79000484608F01AFBB8F8103003EB8303590041
:10C7A00089B2484608F011FB364B1B789B0743BF04
:10C7B000B8F8081001F57A7189B24FF47A714846D9
:10C7C00008F003FB0C9B98F81420591C0C91484668
:10C7D0001A7031F095FA94F8B4322978013393FB4A
:10C7E000F1F201FB123384F8B432F9E613F0030AD4
:10C7F0007FF43AAE5E209047D9F800301420984775
:10C80000214B1F4AB3F9043082FB03124FEAE3784D
:10C81000C8EBA2080FFA88F85FFA88F031F0D6F971
:10C82000C8F3072031F0D2F9D9F800305E209847DC
:10C83000D9F800301C209847504631F0C7F95046CF
:10C8400031F0C4F994F82C31D9F800200CE60F4DE2
:10C850002F6E002F41F09D86044B89F80070C3F8BD
:10C86000B062BDE628B80020C4B80020982500209A
:10C87000CCB80020A0860100C8B80020E8B700208E
:10C880006766666682B7002030B70020D4B8002003
:10C89000C5B80020C057002094F86E31002B41F03D
:10C8A000EA85DF4B1B6803F00802002A48F60341C3
:10C8B0004AF60B404BF60F4249F6074704BF0246C3
:10C8C0000F4613F0040F4FF0190118BF17469B06CF
:10C8D00084F86E1103D547F4804747F0200725F010
:10C8E00049FEC7F30909002842F0D282CD4B9B795B
:10C8F000002B42F09F82984664204FF0FF3A4FF0A1
:10C90000000C0C970D97ADF83CC0CDF842C0CDF8A7
:10C9100046C0CDF84AC0CDF83890ADF83E80ADF8AD
:10C9200040A08DF84E000CAF0FCFDFF808E384F87D
:10C9300005C0AEE80F0097E80F00AEE807002EF83C
:10C94000023B71464FF0010C1B0CFE271F20C82232
:10C9500001F81E39A770A27184F807C0E07094F83E
:10C960007E01207180F0F10383EA0313DAB2130928
:10C9700083F0E70343EA022383EAC2031BB283EA9C
:10C980000312D2B2C3F3072383EA121343EA02234A
:10C9900083EAC2031BB283F0C80282EA0212D2B257
:10C9A000C3F3072383EA121343EA022383EAC20391
:10C9B0001BB283EA0C0787EA0717FFB2C3F307220B
:10C9C00082EA171242EA072200EB0C0382EAC70749
:10C9D0000EEB0C0084F87E31278011F8013B7B4080
:10C9E00083EA0313DBB21A0982EA172242EA03221E
:10C9F00082EAC3031BB29FB281422780EDD183F04C
:10CA00007C0383EA0313DBB24FEA131E8EEA172E70
:10CA10008EEA032E8EEAC30E0FFA8EFE1FFA8EF9EF
:10CA2000DFF814C2A4F800905FFA8EFE4FEA1929CD
:10CA300084F8289084F827E00CF5D37804F1220AD2
:10CA4000DCF80000DCF80410DCF80820DCF80C301E
:10CA500047460FC70CF1100CD445B846F0D1DCF8AE
:10CA600000003860704F9CF8043088F8043007F1FB
:10CA7000270884F8CDE184F8CE9117F8011F2868C3
:10CA8000FDF728FAB845F8D194F86F21002A41F053
:10CA90005E856649029B08781B680A2184F86F113D
:10CAA000002801F09A86DFF894E10128BEF8001012
:10CAB000059142F2EE820228BEF8028002F0008266
:10CAC000BEF804100491032802F0DD820428BEF8A9
:10CAD00006A002F0D3820528BEF8087002F0C782D3
:10CAE0000628BEF80AC002F0BF820728BEF80C1064
:10CAF00001D0BEF80E2094F87EB10C938BF0300379
:10CB000083EA0313DBB24FEA131E494884F804B0EA
:10CB10008EF07A0E4EEA032E00888EEAC303DFF809
:10CB200020E1C0EB00208EFB009E8644C0171BB2A4
:10CB3000C0EB6E200690C3F3072E83EA0310059B1B
:10CB4000C0B24FF0000963F30F098EEA101305938A
:10CB50004FF0000E049B68F31F4967F30F0E4FF070
:10CB60000008002763F30F0861F30F07059BCDF85A
:10CB700034906CF31F4E62F31F474FF0000C9DF88A
:10CB80001820CDF83CE06AF31F48CDF838801097A4
:10CB90008DF844C08DF8452043EA00230DF130089C
:10CBA00083EAC007B8E80F003FB287F0C80989EAF6
:10CBB0000919DFF880E084F805C05FFA89F9C7F346
:10CBC0000727AEE80F0087EA191747EA092398E814
:10CBD000030083EAC9031BB283F023074EF8040B5A
:10CBE00087EA0717FFB2C3F3072282EA17127046DB
:10CBF00042EA072282EAC70720F814190BF1010B59
:10CC00004FF0230CFE211622C82384F87EB1278022
:10CC100084F807C00EF1020EA170E270A37111E05A
:10CC200024B7002014B700203F270020ACB000201C
:10CC300054420020A02500209A250020DCAD0020D1
:10CC40000308208010F8013B7B4083EA0313DBB22A
:10CC50001A0982EA172242EA032282EAC3031BB2BC
:10CC60009FB270452780EDD183F0F40383EA03136C
:10CC7000DBB24FEA131E8EEA172E8EEA032E8EEADF
:10CC8000C30E0FFA8EFE1FFA8EFCD64FA4F800C01A
:10CC90004FEA1C295FFA8EFE84F81EE084F81F908C
:10CCA0007968BA683868FB6807F5D37CACE80F0090
:10CCB00038697969BA6904F2C518ACE8070004F26A
:10CCC000A71784F8C59184F8C4E117F8011F2868F4
:10CCD000FDF700F9B845F8D194F87231002B41F016
:10CCE0004684C14F3B681922980684F8722140F1AE
:10CCF0000E83BE4BDFF800831B78990741F18687CE
:10CD000098F81430042B8CBF4FF003094FF0020940
:10CD1000FCF7A2FDB8F81030B8F808200C9003EB2F
:10CD200083035B00ADF84A304FF47A70D8F80030D6
:10CD30008DF84C900E93B8F80E1098F814E0D8F8CF
:10CD400004308DF84DE000FB02F24FF0000A4FF086
:10CD5000FF300DF13009CDF834A010920F93ADF8EB
:10CD600048101190CC46BCE80F00DFF890E2AEE826
:10CD70000F009CE80F00AEE807007246182122F869
:10CD80001C39E17194F87E1184F805A081F07803D4
:10CD900083EA0313D8B2030983F0F60343EA0023BE
:10CDA00083EAC0031BB283EA0310C0B2C3F30723B4
:10CDB00083EA101343EA002383EAC0031BB283F023
:10CDC000C80080EA001C5FFA8CFCC3F3072080EAED
:10CDD0001C1040EA0C2080EACC0000B280F018035E
:10CDE00083EA0313DBB2C0F3072080EA131040EAA2
:10CDF000032080EAC30301F1010CFE204FF01E0A5C
:10CE00004FF0C80BA0700EF1020E217184F87EC1A4
:10CE1000238084F803A084F806B0184612F8011B9A
:10CE2000414081EA0111C9B20B0983EA102343EAA8
:10CE3000012383EAC10109B288B272452080EDD195
:10CE400081F0180181EA0111C9B20A0982EA1023AE
:10CE500083EA012383EAC1031BB29AB261492280AB
:10CE6000DBB2120A04910692059384F8272084F815
:10CE700026308E4601F5D37B04F1220ADEF800004D
:10CE8000DEF80410DEF80820DEF80C30DC46ACE8F2
:10CE90000F000EF1100ED645E346EFD1DEF800008C
:10CEA000CCF800009DF81430DFF854A184F8CC31A0
:10CEB0009DF8183084F8CD31D3461BF8011F28683F
:10CEC000FDF708F84A4B5B45F7D1FCF7C5FCD8F8ED
:10CED00000103B68B8F808200591D8F804100691B6
:10CEE00013F0140F4FF47A7101FB02F141F07485D5
:10CEF0000F4694F87EB10C908BF06A003D4BDFF842
:10CF000004E1B3F90420109780EA0010C0B20309CD
:10CF100083F0D50343EA002383EAC0031BB283EA0C
:10CF20000310C0B2C3F3072383EA101343EA0023BC
:10CF300083EAC0031BB28EFB020E05980D90D21738
:10CF40004FF00008C2EBAE0206980E9083F0C80CBA
:10CF50000F91ADF84A20ADF84480ADF84680ADF8A9
:10CF600048808CEA0C1CCE465FFA8CFCC3F3072782
:10CF7000BEE80F0087EA1C1747EA0C2787EACC07B0
:10CF8000DFF878C084F804B03FB2ACE80F0087F057
:10CF900021039EE8070083EA0313DBB2C7F30727E8
:10CFA00087EA13170BF1010E47EA03278CE8070005
:10CFB00087EAC30384F87EE14FF0210B4FF0FE0EA9
:10CFC0001C27C8220CF10C0C84F8058084F807B0EB
:10CFD00084F802E0ACF11C01E7701846A2712380CE
:10CFE00012E000BF9A25002024B7002082B700205D
:10CFF0006527002030B70020C0570020A025002062
:10D000003F2700206766666611F8012B424082EADE
:10D010000212D2B2130983EA102343EA022383EAFD
:10D02000C20212B290B261452080EDD182F0680256
:10D0300082EA0212D2B24FEA121B8BEA102383EA71
:10D04000022B8BEAC20B0FFA8BFB1FFA8BF3DB4F21
:10D0500023805FFA8BFB1B0A059384F8253084F844
:10D0600024B007F5D37C04F1220838687968BA68DF
:10D07000FB68E646AEE80F0010374745F446F4D1AA
:10D080003B88AEF800309DF81430CD4F84F8CAB11B
:10D09000D04684F8CB3118F8011F2868FCF71AFF36
:10D0A0004745F8D194F87EC1C64A84F804C08CF094
:10D0B000EB0383EA0313D9B20B0983F0C50343EAF8
:10D0C000012383EAC1031BB283EA0310C0B2C3F396
:10D0D000072181EA101141EA002181EAC00109B269
:10D0E0000CCA81F0C80787EA0717FFB24FF0000E9D
:10D0F000C1F307210D93CDF838E081EA17130C92A4
:10D1000099E8070043EA072383EAC7030FFA83F885
:10D11000AD4B84F805E088F0310783E8070087EA23
:10D120000717FFB2C8F3072383EA171343EA07235D
:10D1300083EAC703277A607AA27AE17A94F80CE04E
:10D1400094F811801BB25F4087EA0717FFB2C3F360
:10D15000072383EA171343EA072383EAC7031BB2B3
:10D16000584080EA0010C0B2C3F3072383EA1013CB
:10D1700043EA002383EAC0031BB25A4082EA02104A
:10D18000C0B2C3F3072282EA101242EA002282EA06
:10D19000C00212B2514081EA0111C9B2C2F30723A1
:10D1A00083EA111343EA012383EAC1031BB28EEA27
:10D1B000030E8EEA0E1E5FFA8EFEC3F3072383EA88
:10D1C0001E1343EA0E23677BA07BE17B227C83EA6C
:10D1D000CE031BB25F4087EA0717FFB2C3F30723F2
:10D1E00083EA171343EA072383EAC7031BB25840B5
:10D1F00080EA0010C0B2C3F3072383EA101343EAA6
:10D20000002383EAC0031BB2594081EA0111C9B26D
:10D21000C3F3072383EA111343EA012383EAC1031B
:10D220001BB25A4082EA0212D2B2C3F3072383EA46
:10D23000121343EA022383EAC2031BB288EA0308FB
:10D2400088EA08185FFA88F8C3F3072383EA1813FB
:10D2500043EA082383EAC803A17CE27CDFF87481F7
:10D260001BB2594081EA0111C9B2C3F3072383EA13
:10D27000111343EA012383EAC1031BB25A4082EA35
:10D280000212D2B2C3F3072383EA121343EA022342
:10D2900083EAC2031BB283F0270787EA0712D2B2E0
:10D2A000C3F3072787EA121747EA022787EAC2076C
:10D2B0003FB20CF10103BAB25FFA87F94FF0310CBB
:10D2C000FE200C2184F87E31C8234FEA122E2280E2
:10D2D00084F807C0A070E170A37184F81490049FD3
:10D2E00084F815E07968BA68FB683868B7F810C048
:10D2F000A8E80F0028F803CB84F8BBE184F8BA91C2
:10D300001AF8011F2868FCF7E5FDD045F8D194F81C
:10D310007671002F41F026812C4B94F87E81B3F971
:10D320000010B3F90220B3F904309FED296A677148
:10D3300007EE103A029B1B680C9388F06A0383EA9D
:10D34000031306EE901AD9B20B0983F0D50343EA12
:10D35000012383EAC1031BB283EA03115242C9B21B
:10D3600007EE902AC3F3072383EA111343EA01234C
:10D37000F8EEE77AF8EEE66AB8EEC77A83EAC10318
:10D380001BB267EE867A66EE866A27EE067A002082
:10D3900083F0C80ECDED0E7ACDED0D6A8DED0F7ACE
:10D3A0001090119012908EEA0E1C0DF130095FFA68
:10D3B0008CFCC3F3072EB9E80F000DE09A2500207E
:10D3C00063270020DC3E0020A025002030B700208D
:10D3D00088C3E43A402700208EEA1C1E4EEA0C2E39
:10D3E0008EEACC0EDFF888C40FFA8EFEACE80F0090
:10D3F0008EF01E0799E8070087EA071A5FFA8AFA93
:10D40000CEF3072787EA1A1747EA0A278CE80700AE
:10D4100087EACA071C214FF0050A4FF01E094FF09A
:10D42000FE0EC82208F10103E17084F876A184F8A9
:10D43000079084F802E0ACF11001A2710CF10C0C21
:10D4400084F80480278084F87E3111F8013B7B400A
:10D4500083EA0313DBB21A0982EA172242EA0322A3
:10D4600082EAC3031BB29FB261452780EDD183F0EE
:10D47000270383EA0313DBB21A0982EA172282EA3E
:10D48000032282EAC3031BB21FFA83FCDFF8E483A2
:10D49000A4F800C05FFA83FE4FEA1C2C84F825C074
:10D4A00084F824E008F5D37904F1220AD8F80000C2
:10D4B000D8F80410D8F80820D8F80C304F460FC719
:10D4C00008F11008D045B946F0D1E04FB8F8003067
:10D4D000A9F8003007F1240884F8CAE184F8CBC128
:10D4E00017F8011F2868FCF7F5FCB845F8D194F847
:10D4F00077A1BAF1000F41F02F80D54B1B680522B0
:10D5000084F877219A0641F17281D24ADFEDD27A0E
:10D51000D18907EE101AB8EEC77A13F0140F27EE70
:10D52000277A01F0F984CD4BDFEDCB6AD3ED007A99
:10D53000F8EEE77A67EEA67A94F87EC1C84BC94A3E
:10D54000B3F90410B2F90620C74FC8488DED0D7A23
:10D550008CF0220383EA03135FFA83FE4FEA1E1363
:10D5600083F0590343EA0E23B2F5FA6F83EACE0340
:10D570001BB2A8BF4FF4FA6283EA0318B2F57A7FB0
:10D580005FFA88F8C3F3072EB8BF4FF47A72A2F59A
:10D590007A728EEA181E642303FB02F34EEA082E09
:10D5A00087FB03278EEAC80EDA17C2EBA71280FBAF
:10D5B00001300FFA8EF7CB174FF0000BC3EBA0032F
:10D5C00087F0C8080DF13009CDED0E7AADF8422094
:10D5D000ADF84030CDF830B0CDF83CB0CE4688EA5A
:10D5E0000818BEE80F005FFA88F8C7F3072787EA34
:10D5F000181747EA082787EAC8089D4FDEF800E0B9
:10D6000084F804C00FC70FFA88F888F04A0383EA49
:10D610000310C0B2C8F3072383EA10133A460CF193
:10D62000010143EA002383EAC00342F810E9002025
:10D630004FF04A084FF0FE0C4FF0140E84F87E11A4
:10D64000C82160712380043784F8078084F802C001
:10D6500084F803E0A171184612F8011B414081EAE9
:10D660000111C9B20B0983EA102343EA012383EABB
:10D67000C10109B288B2BA422080EDD181F0140113
:10D6800081EA0111C9B24FEA111E8EEA102E8EEA0C
:10D69000012E8EEAC10E774B0FFA8EFE1FFA8EFC1A
:10D6A0001F464FEA1C2B5FFA8EFE84F81DB084F8EB
:10D6B0001CE0596838689A68DB68A4F800C007F570
:10D6C000D37CACE80F0038697969B7F81880049703
:10D6D000ACE8030004F2A717ACF8008084F8C3B1EB
:10D6E000B84684F8C2E104F2C31B18F8011F286889
:10D6F000FCF7F0FBC345F8D15F4B604A1B7812780A
:10D70000013B12F00100DBB214BFC0214021172BF6
:10D7100003D85B4A134493F814A05A4B1A88930712
:10D720001ABF002341F01001012312F4027F18BF39
:10D73000022312F0100F18BF062312F0200F18BF9B
:10D740001023002841F091814FF0030894F87EC126
:10D750000C938CF0460383EA0313DAB2130983F0C7
:10D76000920343EA022383EAC2031BB283EA031053
:10D77000C0B2C3F3072282EA101242EA002282EA10
:10D78000C00212B282F0C80E8EEA0E1E00235FFAAB
:10D790008EFE0320C2F307228DF834A08DF8378067
:10D7A00082EA1E128DF835308DF836108DF838006B
:10D7B00042EA0E2899E8070088EACE0E0FFA8EF8A2
:10D7C000DFF8ACA0E37188EA0819AAE803005FFA61
:10D7D00089F9C8F3072888EA191848EA092181EA73
:10D7E000C90994F808808AF800200FFA89F988EAB4
:10D7F000090282EA02185FFA88F8C9F3072282EA6E
:10D80000181242EA0822607AA17A94F80B906371A8
:10D8100082EAC80212B2504080EA0010C0B2C2F3DD
:10D82000072282EA101242EA002282EAC00212B201
:10D83000514081EA0111C9B2C2F3072282EA1112F2
:10D8400042EA012282EAC1021EE000BF3F27002017
:10D8500024B70020C05700200AD7233C28B7002057
:10D8600030B70020DCAD0020D34D621067666666DD
:10D87000A02500209A25002070990020105100203A
:10D88000583F040880B7002012B289EA020989EAE9
:10D8900009195FFA89F9C2F3072282EA191242EAEA
:10D8A000092294F80C80607BA17B84F804C082EA92
:10D8B000C90212B288EA020888EA08185FFA88F8F2
:10D8C000C2F3072282EA181242EA082282EAC80258
:10D8D00012B2504080EA0010C0B2C2F3072282EABE
:10D8E000101242EA002282EAC00212B2514081EADA
:10D8F0000111C9B2C2F3072282EA111242EA0122DF
:10D9000082EAC102E17B94F8109013B281EA03022B
:10D9100082EA0212D2B2C3F3072383EA121343EA64
:10D92000022383EAC2031BB289EA030282EA0212DB
:10D93000D2B2C3F3072383EA121343EA022383EA32
:10D94000C2031BB283F0320282EA0212D2B2C3F3E4
:10D95000072383EA121343EA022383EAC2031BB2BA
:10D960009AB24FF0FE085FFA83FE0920C8210CF13D
:10D97000010C84F802804FEA1228E070A17184F84B
:10D980007EC1228084F8128084F811E0049B18681C
:10D9900059689A68B3F80CB00AF5CC7CACE807007B
:10D9A0000AF5D47A8CF80290ACF800B084F8B8810B
:10D9B00084F8B7E117F8011F2868FCF78BFABA451D
:10D9C000F8D1039BC4F86831FEF706BEDFF83C834C
:10D9D000BF4FDFF83CA3412031F022FDB8F902200F
:10D9E00087FB0230D217C2EBA00080B231F0FCFC02
:10D9F000B8F9002087FB0230D217C2EBA00080B23A
:10DA000031F0F2FCB8F9042087FB0230D217C2EBE8
:10DA1000A00080B231F0E8FC9AF80010D9F80000BC
:10DA2000FCF758FA94F8608118F0010700F0288597
:10DA3000A84F3A68910640F18180A74ADFF8D48266
:10DA40001278920740F1C48798F81420042A8CBFFA
:10DA5000032302230393472031F0E2FCD8F80000AF
:10DA600031F08EFCD8F8040031F08AFCB8F80E20B2
:10DA70009A49D9F80000A1FB0232C2F347121146BD
:10DA80000492FCF727FA9AF800003968049A11F01A
:10DA9000140F82EA00028AF8002040F0BA86B8F833
:10DAA0000820642000FB02F031F06AFC98F8147042
:10DAB000039BD9F8000043EA8707FFB23946FCF719
:10DAC00009FA9AF80020D9F80000574039468AF838
:10DAD0000070FCF7FFF994F86081B8F1000F2DD1C8
:10DAE0007F4F4F2031F09CFC386831F049FC78685A
:10DAF00031F046FC404631F043FC0121D9F80000EA
:10DB0000FCF7E8F9744A9AF800701278D9F8000026
:10DB100002F00108414687F001078AF80070FCF71F
:10DB2000D9F99AF80020D9F8000088EA02021146D3
:10DB30008AF80020FCF7CEF994F86081694AC4F8AD
:10DB40005CB108F10103DBB2A2FB0312D20802EBC5
:10DB50008202A3EB420384F86031FEF71DBD624BE5
:10DB600062491868FCF77EF900232370FEF7BDBDFB
:10DB70005F4F386800283EF4FCAC4FF0000ADFF835
:10DB800098815C4CAB465546FCF7A0F9F8B1F5B965
:10DB90004FF00109AA463868FCF790F983B27E2B52
:10DBA00000F0518498F80120002A49D194F84C11D2
:10DBB000B1B11B2B84F84C2100F01E840D2B45D0F5
:10DBC000386888F80190FCF781F90028E3D1AA466B
:10DBD00050460CAA48495D462FF04CFCFEF7C9BCE4
:10DBE0007D2B00F0F08594F8502122B180F02003C5
:10DBF000DBB284F8501194F84B21062A10D8B4F8FF
:10DC00004E1138681944A4F84E11A118013281F858
:10DC1000543184F84B21FCF759F90028BBD1D6E7E1
:10DC2000B4F84E2188F8019013449BB21A0A52FAB4
:10DC300083F3FF2BA4F84E31386802D12F4DA3E7B0
:10DC40003868FCF743F90028A5D1C0E73868A4F884
:10DC50004E21FCF73BF900289DD1B8E794F8BC327F
:10DC6000C4F8B862012B40F2738594F8BD222449B0
:10DC7000981801EB8001013202F00102CF6A84F8AA
:10DC8000BD22BFB11F4D0D950DF15009123DA523C9
:10DC900049F8205D802284F810311523314648462A
:10DCA00084F8112184F81231B847002840F0D1845B
:10DCB00094F8BC32144A013382FB0312A2EBE372E4
:10DCC00002EB42029B1A84F8BC32FEF795BC00BFFF
:10DCD0006766666624B7002082B700201F85EB5177
:10DCE000DC3E0020CDCCCCCCC0B80020E8B7002072
:10DCF00090B7002098250020E2260020EC26002086
:10DD0000583F0408BD2600205655555530B7002011
:10DD100068BC0020C0570020000000209E4A9F4B96
:10DD200092F80BE0029AD4F8381110681B889C4ACC
:10DD3000401A4FF47A71DFB201FB0EF11B0A97779C
:10DD4000177588424FF00007D37753759770177196
:10DD500080F0EA84934BDFF870C21B689249934FBE
:10DD60000868DFF8689289683F688CFB038EDB17D0
:10DD7000C3EB6E1303F5FA739BB293761B0AD3764B
:10DD800089FB00A389FB01A9C017C917C0EBA30039
:10DD9000C1EBA90107F5EA43DFF834E2107730332D
:10DDA000001282F8201009121B12DFF828829EF858
:10DDB00000E0507782F821108CFB0790F917C1EB37
:10DDC000601182F823307A4B98F814A083F81AA0D7
:10DDD000783130371EF0020F82F8241082F822705A
:10DDE00000F09F84D8F800E0724AD8F80400DFF809
:10DDF000E8B182FB0E714FEAEE77C7EBA1510391B8
:10DE000082FB0092C117C1EBA25203990BFB01E107
:10DE100001EB410149000F460BFB020B0497B94689
:10DE20000BEB4B0B644F4FEA4B01059187FB099BB2
:10DE300087FB01194FEAA949CDF81C90B8F80E905C
:10DE40000399B8F8088002EB820209EBC90902EBDA
:10DE50008202089201EB81074FEA89020599039239
:10DE600007EB8707049A0697CF17C10F099104980B
:10DE700052494FEAAB4BD2174FEADE7E83F809E0F6
:10DE8000ABEB020E01FB1E020798069908F5FA7823
:10DE9000BAF1050F1FFA88FAA0EB0708059F47485B
:10DEA00083F815A04FFA8EF909EB8109414600FB72
:10DEB00018789DF8240098730898414FDFF81CE10A
:10DEC00049B201EB80018CFB020B4FEAE272049233
:10DED000039ABEF800E08CFB08C087FB02C74FEA3C
:10DEE000E27C049AC2EB6B120392364A1FFA89F95C
:10DEF0001288ADF8102083F80A90039A83F813E093
:10DF000089B24FEAE8784FEA112BC8EB6010CCEBEE
:10DF1000A7174FEA1A284FEA192C4FEA222A9DF830
:10DF20000C2083F810B04FEA202983F80BC0D97376
:10DF3000C7F3072C4FEA1E2134BF4FF0320B4FF0CE
:10DF4000330B1A739DF8102083F80DA0587483F8D2
:10DF5000129083F81680DF7183F808C0197583F872
:10DF60001BB01A77C4F83461FEF795BADFF87090E9
:10DF7000D9F80000FBF79AFF00283EF41BABD9F854
:10DF800000000121FBF78EFF0222002387F8742096
:10DF900088F80030FEF70EBB98BA002090BA002037
:10DFA00064B8002028B70020FCB600202CB7002061
:10DFB00090B800206BCA5F6B83DE1B4340420F00AA
:10DFC000D34D6210084F00201F85EB5167666666CF
:10DFD00082B70020C0570020806967FF8CB70020FF
:10DFE000E03500205E209047D9F8003002209847A5
:10DFF000FF2030F015FF0378FF2B00F0998490F993
:10E0000001304FEAE3785FFA88F8D8B22FF0DEFDEE
:10E0100040462FF0DBFDD9F800305E209847D9F854
:10E02000003003209847FF2030F0FAFE0378FF2BE2
:10E0300000F07984B0F90830D8B2C3F307282FF084
:10E04000C5FD40462FF0C2FDDA4B1B78042B7DD076
:10E05000DFF88CB3B4F82E119BF80020DFF884A30E
:10E0600091FBF2F302FB13139BB2BAF80010A4F871
:10E070002E314FEA03181FFA88F8642303FB0123AB
:10E080005200B3FBF2F348EA0328C3F303225E20F5
:10E09000D9F800301FFA88F848EA02089847D9F8FA
:10E0A0000030062098475FFA88F02FF08FFD4FEA86
:10E0B00018202FF08BFDC049B4F82E214B7ABAF806
:10E0C00000A00132012BA4F82E2100F00C874A7B1E
:10E0D0000AEB8A031FFA83FA002A40F0C084D9F8B9
:10E0E00000305E209847D9F800303A209847B34B6B
:10E0F000A3FB0A384FEA58181FFA88FB5FFA8BF027
:10E100002FF064FD4FEA1B202FF060FDD9F800309E
:10E110005E209847D9F800303B209847642303FBE2
:10E1200018A39BB2A648053380FB0320DB17C3EB83
:10E13000A000C0B22FF04AFD00202FF047FDDFF80D
:10E14000A88298F80630002B40F051843B689F0667
:10E1500040F11282DFF894A29AF80030980700F19B
:10E16000EA83DFF88C820027BB46D9F800305E20B6
:10E170009847D9F800300120984758462FF026FDDF
:10E1800038462FF023FDD9F800305E209847D9F8A3
:10E1900000300920984700202FF018FD00202FF0B4
:10E1A00015FDB8F8123098F814B0B3F5967F0AD977
:10E1B00094F82C2102F00F02072A04D842F20F7BB8
:10E1C0009B4528BF9B46D9F800307B4F5E2098477F
:10E1D000D9F80030052098473B7A002B00F066857F
:10E1E000ABF1200307EE903A9FED767AF8EEE77AEE
:10E1F000F6EE006A67EE877ABEEE007AF5EEC07A38
:10E20000F1EE10FA58BFB0EE667A77EE877AFDEE3F
:10E21000E77ACDED027ABDF908B05FFA8BF02FF006
:10E22000D5FCCBF307202FF0D1FC9AF80020002377
:10E2300092070A930B9300F1658394F83031012B18
:10E2400000F06083B7F90030DFED5F6A07EE103A47
:10E25000B7F9023007EE903AB8EEC77AF8EEE77AEF
:10E2600027EE267A67EEA67ABDEEC77AFDEEE77A4C
:10E270000CA88DED0C7ACDED0D7A2FF0C9FC94F839
:10E280002C31D9F80020FEF7F3B85E209047D9F87A
:10E290000030302098474D4BD3F800805FFA88F06B
:10E2A0002FF094FCC8F307202FF090FC94F82C3149
:10E2B00013F003087EF4C8AA454AD4F82811454B48
:10E2C0009142186840F28F8380EAE073A3EBE07319
:10E2D0003A4A1BB282FB03124FEAE37ACAEB621A94
:10E2E0004FF0640808FB1A380FFA88F80FFA8AFA18
:10E2F0005FFA88FB5FFA8AF2C8F30728CAF3072A95
:10E30000D9F8003002925E209847D9F800301020EA
:10E310009847029A10462FF059FC50462FF056FCB1
:10E32000D9F800305E209847D9F80030212098476E
:10E3300058462FF04BFC40462FF048FC3B68D9F87C
:10E340000020FEF78BB8DFF8AC809FED238A4FF0FA
:10E35000240A5E2090475046D9F8003098471F4B5A
:10E36000F8EC016A9B8A07EE103AF8EEE66AB8EE1E
:10E37000C77A0AF1010AC6EE877A5FFA8AFA67EE6F
:10E38000887AFDEEE77ACDED027ABDF908B05FFA42
:10E390008BF02FF01BFCCBF307202FF017FCBAF10A
:10E3A000270F02D0D9F80020D3E73B68D9F8002026
:10E3B000FEF750B88C40002098BA00201F85EB5122
:10E3C00067666666E4380E3F0050C3472CB70020EE
:10E3D0003F4B4C0028B7002000007A4438B700209B
:10E3E000A6BA002090BA002014B7002082B70020FF
:10E3F000C057002068B700203868FBF767FD002889
:10E400007FF4DEAB386884F84A9188F80190FBF716
:10E410005DFD00287FF4BFABFFF7D9BBFBF71CFA0B
:10E42000D14B1B68A0EB030B40F6B8339B4500F2C1
:10E43000BF81CE4B1A793A2A00F04284002388F833
:10E440000030FEF7B7B8386884F84AA184F84BA1C9
:10E4500084F84C9188F801A0FBF738FD00287FF480
:10E460009AABFFF7B4BB94F8481194F84931C0480F
:10E470004A1CFEF76AB8013B84F86E31FEF704BB14
:10E48000BC4A1288D30513D4D00600F1E682910667
:10E4900000F11D85530600F13C85100700F15485FD
:10E4A000D10700F1588512F0020F0CBF04270C278A
:10E4B000B149B24A0B78D27803F001030AB143F0B4
:10E4C00002035320039330F0ABFFAD4A128802EBF6
:10E4D000820202EB8202900080B230F085FF0020C1
:10E4E00030F082FFA74AA8491288D9F80000C2EB91
:10E4F000C212520081FB023111444FEAE278C8EBAC
:10E5000061285FFA88F84146FBF7E4FC9AF800209E
:10E51000039BD9F800001F4388EA020800218AF80B
:10E520000080FBF7D7FC3946D9F80000FBF7D2FC96
:10E530009AF80020D9F800007A40D2B211468AF841
:10E540000020FBF7C7FC94F86081FFF7C6BA013AD8
:10E5500084F86F21FEF7C0BB0AF1FF3A84F877A177
:10E56000FFF72FBA013F84F87671FEF7C0BF013B79
:10E5700084F87231FEF7CBBE1B077FF580AE834B6C
:10E5800093E803000CAB83E8030018462FF040FB30
:10E5900075E60024DFF8108227464FF0500A02E0AB
:10E5A000DBB283F3118815F804B0601C5946284487
:10E5B00030F0E4FD002840F025810BF101031C44FC
:10E5C000EFF311838AF312882A6E9442E8DB00226B
:10E5D000DBB22A6683F31188FEF73EB94FF0000ADA
:10E5E0005E201F6884F82CA19047D9F80030DFF82E
:10E5F000BC811720984750462FF0E8FA644BA3FBE4
:10E6000007239B0BA8FB03125209C2EB0212A3EBD8
:10E610008203D8B22FF0DAFAD9F800305E2098479A
:10E62000D9F80030182098475A4BA3FB07239B09C1
:10E63000A8FB03125209C2EB0212A3EB8203D8B269
:10E640002FF0C4FA50462FF0C1FAD9F80020FDF798
:10E6500014BF0C9EAE424FF000014FD941F2210091
:10E6600015F8013B81EA03235A0013F4004F80EAB6
:10E67000020192B289B208BF11464A0080EA020341
:10E6800011F4004F99B293B218BF0B46590013F41E
:10E69000004F80EA010289B292B208BF0A465300D5
:10E6A00012F4004F80EA03019BB289B208BF1946F9
:10E6B0004A0080EA020311F4004F99B293B218BFE6
:10E6C0000B465A0013F4004F80EA020192B289B25D
:10E6D00008BF11464B0011F4004F80EA03029BB2C1
:10E6E00092B208BF1A46530080EA030112F4004FA9
:10E6F0009BB289B208BF1946B542B1D1484606F06F
:10E7000088FB25490C9D25486D1A152DA8BF152598
:10E710002A4633F0EBFF224A94F8BC321570FFF71B
:10E72000C9BA2D22DA761DE41E4B02991B780968BE
:10E73000C4F83811013B012B3FF60CAB102102232A
:10E7400091701371FFF706BB2FF022FAFDF705BF9A
:10E750000E4A02EB8302D76AFFF793BA2FF008FA4A
:10E7600001233B70FDF7B6BEA43400208C3400209A
:10E7700094B7002080B7002010510020AC3C00204E
:10E7800090BA00205442002003082080583F04081B
:10E7900073B2E745D34D6210A826002088320020CE
:10E7A0009D3200208C40002035DD03088988888850
:10E7B000C44AB2F8623100210133A2F8623188F80C
:10E7C0000010FDF7F7BE386884F85091FBF77EFB28
:10E7D00000287FF4E0A9FFF7FAB90146844607460E
:10E7E00082460490804605900246FEF784B99FED6C
:10E7F000B67A13F0140F08BFF0EE477A7EF493AEAA
:10E80000FEF79ABE41463A2030F014FC0743FFB2AF
:10E81000D3E6AE4A1068FFF747B9AD49AD4B009358
:10E82000A1F13F07AC4BAD4A0B9101F8404C0CA84D
:10E83000AB490A9706F0C4FB0A9F7B1C0A933C7005
:10E840000A9B2922591C0A911A700A9BEA22591C18
:10E850000A911A700A9BC822591C0A910CA81A70B6
:10E8600032F0E5FF00F101080CA942460A9833F0A6
:10E870003DFF0A9A02EB080301330A9302F80840AD
:10E880000A9B5A1C0A921C700A9B5A1C0A921C7002
:10E890000A9B5A1C0A921C700A9B5A1C0A921C70F2
:10E8A0000A9B5A1C0A921C700A9B5A1C0A921C70E2
:10E8B0000A9B5A1C0A921C700A9B5A1C0A921C70D2
:10E8C0000A9B5A1C0A921C700A9B5A1C0A921C70C2
:10E8D0000A9B5A1C0A921C700A9B5A1C0A921C70B2
:10E8E0000A9B0122991814A80A911A7050F8283D21
:10E8F000DB1B3B702FF004FA724B2C70C3F8B06234
:10E90000FDF76EBE98E80C0001210AA884F83011CA
:10E910000A920B932FF07CF9B1E4C4F83C6187F8BC
:10E920000080FDF7D7BD4FF000084046FFF787BBDA
:10E930004046FFF76BBBDFF8C081D9F80030694F64
:10E940005E209847D9F8003011209847B8F80E207B
:10E950004FF4F36B0BFB02F287FB0237D217C2EBCB
:10E960006737F8B22FF032F9C7F307202FF02EF9EE
:10E97000D9F800305E2098471920D9F80030984720
:10E98000B8F80E30584A0BFB03F382FB0301DB1788
:10E99000C3EB611382FB0321DA17C2EB611264211E
:10E9A00001FB1233D8B22FF011F900202FF00EF92D
:10E9B0009AF80030B8F8087099077FF5D4AB5FFA81
:10E9C00087FB3F0AFFF7D1BBFBF76CFAFDF797BD5A
:10E9D00001230393FFF73FB83C4B1F6807EB870702
:10E9E0007F00FEF786BAC346C246424688E4D9F89D
:10E9F0000030DFF808B1DFF808A15E209847D9F8A9
:10EA0000003028209847DBF800308AFB032ADB1708
:10EA1000C3EBAA0A5FFA8AF02FF0D8F8CAF30720EE
:10EA20002FF0D4F8D9F800305E209847D9F800309C
:10EA300004209847B8F80830002B40F04B82DBF8F0
:10EA4000083083F310085FFA88F02FF0BFF8C8F39E
:10EA500007202FF0BBF8FFF779BB342728E59BF898
:10EA600000309AFBF3FAFFF73ABB204AD278002A2B
:10EA70000CBF4FF004084FF00508FEF767BE0123F6
:10EA8000D9F800003B70FBF719FA0746D9F80000E7
:10EA9000FBF714FA7F067DF41DAD8A2800F043824F
:10EAA0008E287DF417AD9AF80030002B7DF42EAD42
:10EAB0000F48104B03602D2384F840310768FDF7A1
:10EAC0000DBD00BF982500200000000028B70020E1
:10EAD000E8B70020728C0020D8760408E07604089D
:10EAE000EC76040889B5F8141F85EB51AC3C002086
:10EAF0009CB7002064B80020C0570020FCB600205E
:10EB000067666666CF4AD04B0D920DF15008A2F1B0
:10EB10003D0048F8200D1988DFF85493A2F1400316
:10EB200000204FF00A0E02F8400C082283F801E0A2
:10EB300040469A7006F049F9D9F80030C349DA170F
:10EB400081FB0313C2EBA30399B2404606F03DF9E3
:10EB500023F01EFDD9F808900C9B4FEA1942591C6E
:10EB60000C911A700C9B4FEA1922591C0C911A70C7
:10EB70000C9B5A1C0C9283F800900C9B5A1C0C9214
:10EB8000187040462FF0BCF8FDF7D3BDAD4B0D9388
:10EB9000A3F1400900222121A3F13D0A03F8402CF2
:10EBA00089F8021089F80120CDF830A020F028F96A
:10EBB000A74BA84A1B88A84900280ABF11464FF056
:10EBC00003084FF004085A0500F19F81D80700F1AF
:10EBD000BE8103F00203A14A002B1CBF4FF00308C3
:10EBE000114642469E4833F081FD0AEB080314A803
:10EBF0009C4A013340F8203D9B1A00220AF8082065
:10EC000089F801302FF07CF8FDF796BD4FF001092F
:10EC1000FEF77EB8DFF86C929FED938AB9F9023067
:10EC2000884A0D9207EE903AF8EEE77A0DF1500817
:10EC300067EE887AA2F14003FDEEE77AA2F13D018A
:10EC400048F8201D02F8400C0822CDED027A5A70D7
:10EC50001E229A70BDF80810404606F0B6F8B9F9C1
:10EC6000003007EE903AF8EEE77A404667EE887A91
:10EC7000FDEEE77ACDED027ABDF8081006F0A5F8B2
:10EC8000B9F9043007EE903AF8EEE77A404667EEBD
:10EC9000887AFDEEE77ACDED027ABDF8081006F02D
:10ECA00094F840462FF02CF8FDF740BD5FFA8BF04A
:10ECB0002EF08CFF4FEA1B202EF088FFFFF7B5BA2D
:10ECC00099780393184611F0CBFD00287FF4B6AB7A
:10ECD0005D49664F664A09886648674CF961DFF806
:10ECE000A891116803689268F962B4F86211C7F8D4
:10ECF0006CB0FB63FA64D9F80000F965F9F754FACF
:10ED0000834600287DF451AC5146D9F80000FBF74A
:10ED1000C9F8039B94F86421DB780493642A4FF0CC
:10ED2000040387F8743040F0198194F86531072B9B
:10ED300008BF84F865B194F86521504B079207EB42
:10ED4000021A0393DAF804100691084632F06FFDB8
:10ED5000DAF8083005935FFA80FA184632F067FD5A
:10ED60005FFA80FB454B079A06990AEB0B000830C7
:10ED7000D87122F00F00987202F00F020BEBCA005C
:10ED80005A739873524603F10F0033F0AFFC059BA2
:10ED900019463B4B0AF1090018445A4633F0A6FCC9
:10EDA0003648C37903F1010ACBB1013B5FFA83FC1A
:10EDB0000CF1080CDFF8D4E084440023073010F88D
:10EDC000012B5A409300D10883EA420301F0180155
:10EDD00053404EFA01F253408445DBB2EFD1284A4A
:10EDE00004980AF8023033F04BFC94F865310022A5
:10EDF000013384F8653184F86421039BDDF80CA0AD
:10EE00009B785BB11AF80510D9F80000FBF762F89F
:10EE100001359AF80230EDB2AB42F3D894F8643180
:10EE20000322013384F8643187F8742088F80020C5
:10EE3000FFF79EB80E4B8046B3F900A06420FDF7A3
:10EE40005EBD00BFE8B7002090BA00206766666626
:10EE500080B70020BC760408C4760408D476040881
:10EE6000ABB70020A9B7002058A08B4100000020BC
:10EE7000FCB6002028B7002098250020D857002095
:10EE8000DE57002030B70020E03500200007090ED3
:10EE9000854B864A1B88927903EB830303EB83033C
:10EEA0004FEA83081FFA88F8002A40F0FA804FF0F2
:10EEB000FF330FFA83FA23F06BFB40B2FDF71FBD5F
:10EEC00011469446174692460492FDF714BE242735
:10EED000FFF7EEBA23F05CFB2EF078FE00202EF058
:10EEE00075FEFFF733B9D9F800305E209847D9F89E
:10EEF0000030392098475FFA8AF02EF067FE4FEA1B
:10EF00001A202EF063FEFFF71AB94FF00308684984
:10EF100067E61027FFF7CCBA138907EE903AF8EEB0
:10EF2000677AFEF709BB634B1B6898067DF5D2AA8A
:10EF30009AF80030002B7DF4E9AA5F485F4B03602C
:10EF40002D2384F84031B9E52027FFF7B1BA5C4999
:10EF50004FF0040845E60827FFF7AABA97F875307E
:10EF600058481A0704BF0133DBB2072B28BF01231F
:10EF70004FEA031B07EB0B025FFA8BFA92F810E0E3
:10EF8000514A039200EB0E010022087A4E498A7220
:10EF900001F10D0207EB0B014AEA0E0E012882F87F
:10EFA00000E0C96802F1010C0DD90238C0B200F1CD
:10EFB000020E9644624602F8011B72454FEA112187
:10EFC000F9D101308444BB4421F0600201339BF845
:10EFD0001110DBB20A43082B8CF800200CF101025F
:10EFE00049D04FEA031B07EB0B00384990F810E0BB
:10EFF00034487044511A007A01EB000C0AF1100AEF
:10F00000BCF1130F5FFA8AFAC4DDC9B28A1DD2B20D
:10F01000039842F0400E80F807E002F1010ADFF8A1
:10F02000B8E0CAB105315FFA81FB0BF1080B8344EC
:10F030000EF1010C00221CF8010B5040820082EA04
:10F040004002C1084240224801F0180140FA01F193
:10F050004A40E345D2B2EED104980AF80E2087F870
:10F06000753033F00DFBC8E61146FDF744BD11467F
:10F070009446FDF740BD1549511AC6E7114694461E
:10F080001746FDF738BD1146944617469246FDF7E0
:10F0900032BD114694461746924604929046FDF7BB
:10F0A0002ABD0C4B1B6804E790BA002014B700205F
:10F0B000C876040824B700209CB7002090B8002030
:10F0C000CC760408583F0408D8570020E5570020A4
:10F0D0000007090EFCB60020DE5700202DE9F04F96
:10F0E0004FF4807385B043838383C38300F10C05A1
:10F0F00004463220FAF756FC11220021284605F07A
:10F1000009FA60220121284605F004FA6420FAF782
:10F1100049FC02A92046002732F038F90123B946FC
:10F12000B8463E460193012E14BF1122122200213F
:10F13000284605F0EFF9002E0CBF4FF0010B4FF001
:10F14000FF3B4FF00A0A01220221284605F0E2F9AE
:10F150001420FAF727FC02A9204632F017F9BDF96E
:10F160000A20BDF90C00BDF90810234B82420BFBAD
:10F170000299A8BF02468A42A8BF0A469A4201FBEA
:10F180000B880BFB007733DB0120FAF7EDFEBAF1B9
:10F19000010AD8D10136022EC5D1184B93FBF8F8DD
:10F1A00093FBF9F97022A3F58423002193FBF7F771
:10F1B000A4F81A80A4F81C90E783284605F0AAF961
:10F1C00020220121284605F0A5F9002231462846D3
:10F1D00005F0A0F96420FAF7E5FB019B23B94FF491
:10F1E00080736383A383E383012005B0BDE8F08FC0
:10F1F00000230193CEE700BF01F0FFFF00D03B00EA
:10F2000038B504460D4600BF806804F067FF294604
:10F21000606831F0F3FEA06804F065FF00BF38BD00
:10F22000F0B55FEA930E33D000F1100601F110053E
:10F2300002F11004774616ED046A55ED044A56EDC6
:10F24000026A15ED025A16ED037A55ED035A56ED92
:10F25000017A26EE246A66EE856A04ED046A15EDED
:10F26000016A44ED026A27EE257A67EE867A013F4D
:10F2700004ED037A44ED017A06F1100605F110055C
:10F2800004F11004D7D14FEA0E1420442144224443
:10F2900013F003030BD000EB8303F0EC017AB1EC25
:10F2A000017A67EE877A8342E2EC017AF5D1F0BD0C
:10F2B000A849A948A94A2DE9F84F012303700B88F2
:10F2C000128823F040031B041B0C0B800B8823F0D7
:10F2D00038031B0452084FEA13430BD042F48072E8
:10F2E000002A92FAA2F1B1FA81F208BF4FF0FF3280
:10F2F000013AD2001343974A9BB2138013889BB202
:10F3000043F040031380964B1B6813B11A689B8827
:10F310005383904940F2E93302E0002B00F09E81D4
:10F320000A89013B12F0020F9BB2F6D005238B81B4
:10F3300040F2E933874902E0002B00F08F810A890F
:10F34000013B12F0010F9BB2F6D08B89814940F24C
:10F35000E93302E0002B00F0A5810A89013B12F09D
:10F36000020F9BB2F6D000238B8140F2E93379493A
:10F3700002E0002B00F096810A89013B12F0010F98
:10F380009BB2F6D08B89734940F2E93302E0002B3F
:10F3900000F084810A89013B12F0020F9BB2F6D083
:10F3A00006238B8140F2E9336A4902E0002B00F02A
:10F3B00075810A89013B12F0010F9BB2F6D08B894F
:10F3C000644940F2E93302E0002B00F063810A89CE
:10F3D000013B12F0020F9BB2F6D000238B8140F26A
:10F3E000E9335C4902E0002B00F054810A89013BBB
:10F3F00012F0010F9BB2F6D08B89DFF86CA1554952
:10F400009AF8004040F2E93344F0010402E0002B96
:10F4100000F03C810A89013B12F0020F9BB2F6D04A
:10F4200004238B8140F2E9334A4902E0002B00F0CB
:10F430002D810A89013B12F0010F9BB2F6D08B8916
:10F44000444940F2E93302E0002B00F01B810A89B5
:10F45000013B12F0020F9BB2F6D0A4B28C8140F2B5
:10F46000E9333C4902E0002B00F00C810A89013BA2
:10F4700012F0010F9BB2F6D08B893A4F3B88002BDC
:10F4800047D0DFF8E890DFF8E880324C4FF0000B0F
:10F49000072699F8015040F2E93302E0002B00F012
:10F4A000D5802089013B10F0020F9BB2F6D0A681D7
:10F4B00040F2E93302E0002B00F0C8802089013BD4
:10F4C00010F0010F9BB2F6D0A38940F2E93302E0BD
:10F4D000002B00F0BF802089013B10F0020F9BB28F
:10F4E000F6D0ADB2A58140F2E93302E0002B00F086
:10F4F000B1802089013B10F0010F9BB2F6D0A389A7
:10F500003B8819F8010F08F8010F0BF1010B9B451F
:10F51000BFDB104840F2E93302E0002B00F0AE8080
:10F520000289013B12F0020F9BB2F6D007238381C0
:10F53000084940F2E93302E0002B00F09F800A897D
:10F54000013B12F0010F9BB2F6D08B89014840F2CB
:10F55000E93311E0003800404DB0002004030020E2
:10F56000186C0020241E00205C28002043AE0020E0
:10F570005F280020002B7DD00289013B12F0020F92
:10F580009BB2F7D0FF238381484940F2E93301E081
:10F59000002B6FD00A89013B12F0010F9BB2F7D00C
:10F5A0008B899AF80040414840F2E93301E0002B92
:10F5B0005CD00289013B12F0020F9BB2F7D004230A
:10F5C00083813A4940F2E93301E0002B4ED00A89A9
:10F5D000013B12F0010F9BB2F7D08B89334840F208
:10F5E000E93301E0002B3DD00289013B12F0020F0C
:10F5F0009BB2F7D0A4B22D49848140F2E93301E0F7
:10F60000002B2FD00A89013B12F0010F9BB2F7D0DB
:10F610008B89274B1B6813B11A689B881383234A75
:10F62000138823F040031B041B0C1380138823F062
:10F6300038031B041B0C138013889BB243F0400358
:10F6400013801C4B00211970BDE8F88F204604F090
:10F650009FFE3AE7204604F09BFE51E7134804F072
:10F6600097FE73E6114804F093FED2E70F4804F0CA
:10F670008FFEB3E70D4804F08BFE92E70B4804F0D1
:10F6800087FE63E7094804F083FEF6E6074804F0C6
:10F690007FFED5E6054804F07BFEAEE6034804F0A5
:10F6A00077FE8DE6014804F073FE6CE600380040FA
:10F6B000186C00204DB00020AA490A8822F04002B0
:10F6C0002DE9F0471204A84F120C3B880A800A88E3
:10F6D00022F0380212045B084FEA124200F00C825A
:10F6E00043F4807090FAA0F10028B1FA81F108BFCC
:10F6F0004FF0FF310139C9000A439A499B4D92B23C
:10F700000A800A8892B242F040020A80296811B148
:10F710000A6888885083964A1278012A00F0258268
:10F72000C0F00C82022A40F0D381924E082232703F
:10F730004FF4C372DFF844828A48A8F80020028898
:10F7400022F040021204120C0280028822F03802D9
:10F750001204120C5BB143F4807090FAA0F30028FD
:10F76000B3FA83F308BF4FF0FF33013BDB001343D1
:10F770007C4A9BB2138013889BB243F040031380F2
:10F7800011B10B688A885A83764C4FF010094FF0FC
:10F79000010A40F2E93302E0002B00F0A381228944
:10F7A000013B12F0020F9BB2F6D01FFA89F3A3813E
:10F7B00040F2E93302E0002B00F094812289013B02
:10F7C00012F0010F9BB2F6D0A38940F2E93302E0B8
:10F7D000002B00F08B812289013B12F0020F9BB2BB
:10F7E000F6D0A4F80CA040F2E93302E0002B00F0C0
:10F7F0007D812289013B12F0010F9BB2F6D0A389D3
:10F8000009F10109B9F1200FC3D1296811B10B68C1
:10F810008A881A83534B1A8822F040021204120C71
:10F820001A801A8822F038021204120C1A801A88E0
:10F8300092B242F040021A8018883A8820F04000C4
:10F840000004000C18801B8823F038031B045208A6
:10F850004FEA13430BD042F48072002A92FAA2F0CE
:10F86000B0FA80F208BF4FF0FF32013AD2001343E2
:10F870003C4A9BB2138013889BB243F04003138031
:10F8800011B10B688A885A833478364940F2E933DB
:10F8900002E0002B00F04A810A89013B12F0020FBE
:10F8A0009BB2F6D000238B8140F2E9332D4902E070
:10F8B000002B00F03B810A89013B12F0010F9BB243
:10F8C000F6D08B89274940F2E93302E0002B00F0A3
:10F8D00031810A89013B12F0020F9BB2F6D0A4B22B
:10F8E0008C8140F2E9331F4902E0002B00F02281B5
:10F8F0000A89013B12F0010F9BB2F6D08B891E4B97
:10F9000018491C7840F2E93302E0002B00F0F68041
:10F910000A89013B12F0020F9BB2F6D002238B81C1
:10F9200040F2E9330F4902E0002B00F0E7800A893A
:10F93000013B12F0010F9BB2F6D08B89094940F2CE
:10F94000E93302E0002B00F0DD800A89013B12F070
:10F95000020F9BB2F6D0A4B28C8140F2E933014988
:10F9600011E000BF0038004004030020186C0020A4
:10F970002C6C0020261E0020336C0020241E00204A
:10F98000002B00F0BF800A89013B12F0010F9BB2EF
:10F99000F6D08B897E4B7F491C7840F2E93302E038
:10F9A000002B00F0B3800A89013B12F0020F9BB2DA
:10F9B000F6D003238B8140F2E933764902E0002B35
:10F9C00000F0A4800A89013B12F0010F9BB2F6D02F
:10F9D0008B89704840F2E93302E0002B00F09A80F6
:10F9E0000289013B12F0020F9BB2F6D0A4B2694922
:10F9F000848140F2E93302E0002B00F08B800A8919
:10FA0000013B12F0010F9BB2F6D08B89624B61482B
:10FA10001C7840F2E93344F0040401E0002B7DD06F
:10FA20000289013B12F0020F9BB2F7D004238381BD
:10FA3000584940F2E93301E0002B6FD00A89013BBD
:10FA400012F0010F9BB2F7D08B89524840F2E93394
:10FA500001E0002B66D00289013B12F0020F9BB23D
:10FA6000F7D0A4B24B49848140F2E93301E0002B86
:10FA700058D00A89013B12F0010F9BB2F7D08B8955
:10FA80002B6813B11A689B881383424A434C13882E
:10FA9000434823F040031B041B0C1380138823F0FE
:10FAA00038031B041B0C138013889BB243F04003E4
:10FAB0001380B8F80020002133F0ABFF2378CBB1DE
:10FAC000384B1B78002B56D000232370BDE8F087FD
:10FAD000354E327812F0400F0CBF4FF4C3724FF422
:10FAE000F07227E6204604F053FC6EE6204604F050
:10FAF0004FFC85E6BDE8F0871946FDE5254804F092
:10FB000047FC1BE7234804F043FC43E7214804F08B
:10FB10003FFC5EE71F4804F03BFC77E71D4804F01C
:10FB200037FC92E71B4804F033FCA9E7194804F0BE
:10FB30002FFCC7E6174804F02BFCE0E6A02115488F
:10FB400031F05CFA0021134831F058FA00F0060356
:10FB5000022B03D000F00500012812D0124E3B8882
:10FB60002968082232705B08E2E50F4E48223270A5
:10FB70004FF4F072DEE5FFF79BFB00232370BDE836
:10FB8000F087094E3B882968482232705B08EFE70E
:10FB9000346C0020003800405C28002076000020F3
:10FBA000602800204DB00020261E0020A649A74A4C
:10FBB0002DE9F84F012313700A88A54B22F040026B
:10FBC0001204120C1B880A800A8822F038021204E0
:10FBD0005B084FEA12420BD043F48073002B93FA78
:10FBE000A3F1B1FA81F308BF4FF0FF33013BDB0013
:10FBF0001343954A9BB2138013889BB243F0400392
:10FC00001380944B1B6813B11A689B8853838E49E9
:10FC100040F2E93302E0002B00F009810A89013B40
:10FC200012F0020F9BB2F6D080238B8140F2E933B1
:10FC3000854902E0002B00F0FA800A89013B12F0AE
:10FC4000010F9BB2F6D08B897F4940F2E93302E085
:10FC5000002B00F0F0800A89013B12F0020F9BB2EA
:10FC6000F6D000238B8140F2E933774902E0002B84
:10FC700000F0E1800A89013B12F0010F9BB2F6D03F
:10FC80008889C0B2734B1B6813B11A689B881383B1
:10FC90006D4A714C1388714D23F040031B041B0CFB
:10FCA0001380138823F038031B041B0C1380138864
:10FCB0009BB243F04003138023782F6883423ED0E9
:10FCC000FFF7FAFC664E674BB6F8EE21B3F80080FA
:10FCD000DFF89CC100210D464FF0050B4FF0060ADE
:10FCE0004FF00709B4181CF802002379834202F18F
:10FCF000010705F1050312D006EB030E73192071FD
:10FD0000140A83F8F0B183F8F2A183F8F32183F8A1
:10FD1000F49183F8F141013106358EF8F001BAB261
:10FD2000424501F101014FD26329DBDDA6F8EE2146
:10FD3000002D4ED1454A00231370BDE8F88F4A4B81
:10FD4000474E1B78002BBED1D6F8E431FB1AB3F531
:10FD50007A7FB8D93E4B1046198831F071FA3D4B85
:10FD60001B6813B11A689B885383A021364831F071
:10FD700045F90021344831F041F9364B1B68814682
:10FD800013B11A689B881383DFF8E8802E4804219A
:10FD900031F056FA98F80030182B6DD019F0040F96
:10FDA0004ED109F00503012B74D053B923785B06BB
:10FDB00007D5D6F8E8212B68002A6FD09B1A642B50
:10FDC0006FD8C6F8E4717EE70023A6F8EE31002D67
:10FDD000B0D01F4B1C48198831F032FA1D4B1B68FC
:10FDE00013B11A689B8853832B4600221F4916487B
:10FDF00031F0D4F8174B1B6813B11A689B88138332
:10FE0000114A138823F040031B041B0C1380138832
:10FE100023F038031B041B0C138013889BB243F0A0
:10FE200040031380094A00231370BDE8F88F064889
:10FE300004F0AEFA08E7044804F0AAFAC0B221E7D9
:10FE40000023C6F8E831BCE7003800404DB0002080
:10FE500004030020186C0020261E0020E86B002000
:10FE60005C280020241E00202C6C00204C2A00203E
:10FE700044AE0020216C00202378114A03F0400397
:10FE8000002B09F007010CBF0D20102013805180BA
:10FE9000D08083E723785A068BD592E7C6F8E831FD
:10FEA0008FE7FFF709FC98F80030182B89D1B6F8D6
:10FEB000EC31034A01339BB2A6F8EC31938080E722
:10FEC000246C00202DE9F84FA94F3B7803B1FEE7E1
:10FED000A84CA94A01233B702388128823F04003D1
:10FEE0001B041B0C2380238823F038031B045208B7
:10FEF0004FEA13430BD042F48072002A92FAA2F424
:10FF0000B4FA84F208BF4FF0FF32013AD200134333
:10FF1000984ADFF870829BB2138013889BB243F03B
:10FF200040031380D8F8003013B11A689B885383BC
:10FF3000924B01220D461A7004468E4940F2E93375
:10FF400002E0002B00F0A3810A89013B12F0020FAE
:10FF50009BB2F6D000238B8140F2E933854902E061
:10FF6000002B00F094810A89013B12F0010F9BB233
:10FF7000F6D08B897F4940F2E93302E0002B00F094
:10FF80009A810A89013B12F0020F9BB2F6D000233E
:10FF90008B8140F2E933774902E0002B00F08B813E
:10FFA0000A89013B12F0010F9BB2F6D08B8971498F
:10FFB00040F2E93302E0002B00F079810A89013B2D
:10FFC00012F0020F9BB2F6D009238B8140F2E93385
:10FFD000684902E0002B00F06A810A89013B12F0B7
:10FFE000010F9BB2F6D08B89624940F2E93302E0FF
:10FFF000002B00F058810A89013B12F0020F9BB2DE
:020000040801F1
:10000000F6D0A4B28C8140F2E9335A4902E0002BC9
:1000100000F049810A89013B12F0010F9BB2F6D032
:100020008B89574E534C013D4FF0000A4FF00A0B9D
:1000300040F2E93302E0002B00F010812289013BFD
:1000400012F0020F9BB2F6D0A4F80CB040F2E933E4
:1000500002E0002B00F002812289013B12F0010F27
:100060009BB2F6D0A38940F2E93302E0002B00F006
:10007000F9802289013B12F0020F9BB2F6D01FFAE1
:100080008AF3A38140F2E93302E0002B00F0EA801A
:100090002289013B12F0010F9BB2F6D0A38915F81B
:1000A000019F40F2E93302E0002B00F0DF8022895B
:1000B000013B12F0020F9BB2F6D00B23A38140F25A
:1000C000E93302E0002B00F0D1802289013B12F0DD
:1000D000010F9BB2F6D0A38940F2E93302E0002B76
:1000E00000F0C8802289013B12F0020F9BB2F6D0CB
:1000F0001FFA89F9A4F80C9040F2E93302E0002BD2
:1001000000F0B8802289013B12F0010F9BB2F6D0BB
:10011000A389336833B11A689B8851690B4214BFB5
:10012000538313830AF1010ABAF1360F80D140F2EA
:10013000E933104802E0002B00F0B1800289013B56
:1001400012F0020F9BB2F6D008238381094940F2D6
:10015000E93302E0002B00F0A2800A89013B12F093
:10016000010F9BB2F6D08B89024840F2E9330EE0D2
:100170004DB00020003800400403002055B000209E
:10018000B46B0020186C0020002B00F084800289E2
:10019000013B12F0020F9BB2F6D0A02383814849A5
:1001A00040F2E93301E0002B75D00A89013B12F0DF
:1001B000010F9BB2F7D08B89414CA02540F2E93367
:1001C00001E0002B5AD02289013B12F0020F9BB2B2
:1001D000F7D0A58140F2E93301E0002B4ED022890F
:1001E000013B12F0010F9BB2F7D0A38940F2E93333
:1001F00001E0002B46D02289013B12F0020F9BB296
:10020000F7D00023A38140F2E93301E0002B39D07D
:100210002289013B12F0010F9BB2F7D0A089C0B236
:100220008306CBD4D8F8003013B11A689B881383A7
:10023000234A138823F040031B041B0C13801388EC
:1002400023F038031B041B0C138013889BB243F06C
:100250004003002113803970BDE8F88F204604F078
:1002600097F800E7204604F093F818E7204604F0DA
:100270008FF831E7204604F08BF84AE7204604F077
:1002800087F8B3E7204604F083F8C0B2C8E70C480B
:1002900004F07EF86EE60A4804F07AF88CE7084825
:1002A00004F076F860E7064804F072F8B9E604480E
:1002B00004F06EF898E6024804F06AF877E600BFAA
:1002C0000038004030B4147874B11E23074D13FB7E
:1002D00001012944801A83181D2BD8BF0C7012F815
:1002E000014F0131002CF6D130BC704744AE0020E4
:1002F000F8B5434C434A2388128823F040031B047B
:100300001B0C23802388C1F1030123F0380341EA49
:1003100080071B045208FFB24FEA13430BD042F48C
:100320008072002A92FAA2F1B1FA81F208BF4FF06E
:10033000FF32013AD2001343314A334D9BB213804E
:1003400013889BB243F0400313802B6813B11A68E3
:100350009B8853832A4CBFB2102640F2E93301E058
:10036000002B45D02289013B12F0020F9BB2F7D03F
:10037000B3B2A38140F2E93301E0002B38D02289E7
:10038000013B12F0010F9BB2F7D0A38940F2E93391
:1003900001E0002B30D02289013B12F0020F9BB20A
:1003A000F7D0A78140F2E93300E02BB32289013B6B
:1003B00012F0010F9BB2F8D0A3890136202ECCD1C8
:1003C0002B6813B11A689B8813830D4A138823F096
:1003D00040031B041B0C1380138823F038031B04F9
:1003E0001B0C138013889BB243F040031380F8BDAD
:1003F000204603F0CDFFC9E7204603F0C9FFDCE744
:100400000038004004030020186C002038B5454B2C
:100410001D7800287BD105F0F70543491D700B8836
:10042000424A23F040031B041B0C12880B800B88EC
:1004300023F038031B0452084FEA13430BD042F455
:100440008072002A92FAA2F1B1FA81F208BF4FF04D
:10045000FF32013AD2001343334A354C9BB213802A
:1004600013889BB243F040031380236813B11A68CA
:100470009B88538340F2E9332B4901E0002B49D09C
:100480000A89013B12F0020F9BB2F7D004238B8143
:1004900040F2E933244901E0002B3BD00A89013BBB
:1004A00012F0010F9BB2F7D08B891F4940F2E9335C
:1004B00001E0002B32D00A89013B12F0020F9BB2FF
:1004C000F7D0ADB28D8140F2E933174900E02BB38C
:1004D0000A89013B12F0010F9BB2F8D08B89236887
:1004E00013B11A689B8813830F4A138823F04003C3
:1004F0001B041B0C1380138823F038031B041B0CF4
:10050000138013889BB243F04003138038BD45F03D
:10051000080582E7044803F03BFFC6E7024803F002
:1005200037FFDCE75C28002000380040040300208F
:10053000186C00202DE9F047C44B1C6862072DEDB4
:10054000028B03D4BDEC028BBDE8F087C04D2B7845
:10055000002BF7D06E6846F2A713861B9E42F1D996
:10056000DFF850936860B9F80070DFF84C83002F13
:1005700040F0A68198F80620AB689FEDB60ADFED43
:10058000B60ADFF8F492013AB3FBF2F307EE903AC1
:10059000F8EE677AB7EE008A27EE800A32F044FB65
:1005A000DFEDAE7A38EE400A20EE270A32F074FA18
:1005B000B8F80830DFEDAA6A07EE103AEB68C01A07
:1005C000B8EEC77A07EE900AA7EE668AB8EEE70A99
:1005D000D9ED097AF8EEE77A20EE080A67EEA67AF6
:1005E000A7EE270A32F058FA9E4BC9F824000246BB
:1005F0001860A30740F1AA81DFF8C0E29A4CDEED53
:10060000007A9FED9A5A2168F8EE677A27EE855AAC
:10061000002900F0BB81964B07EE101AD3ED026A59
:10062000B8EEC77AF8EEE66A86EE878A914991EDD0
:10063000004AB8F80C10D5ED054ADFED895A95ED62
:10064000066A67EE847A06EE901A67EE887A8A491F
:10065000B6EE004AF8EEE66AF0EE643AE7EE843A67
:1006600066EEA56A91ED097A7E49F7EE005A75EEBD
:10067000E65AB8EEC77AA3EE856A77EEA47A27EE3B
:10068000257AC5ED057AF0EE477AE6EE267ABDEEDC
:10069000E77AC5ED067A81ED007A78490978122962
:1006A00000F05B8100211960596099602160CEF8EB
:1006B0000010002F7FF446AFE869EA61121A07EED6
:1006C000102ADFED6F6A6F4B07EE906AB8EEC77ABB
:1006D000F8EE677A27EE267A40F2DC52C7EE276AF8
:1006E0000A21FDEEE67A17EE900A9042A8BF104666
:1006F0009842B8BF184604F0ADFDB8F80A309FED37
:10070000586AD5ED056A07EE103AB8EEC77AF7EEEB
:10071000007AE7EE467A05EE900AF8EEE55A66EEC4
:10072000866A67EEA57AE7EE267AB0EE670AC5ED2F
:10073000057A32F0B1F90521064604F08BFD524AE4
:100740005249B2F90040086084EAE473A3EBE47311
:10075000B3F5487F74DAB2F9022082EAE273A3EBC0
:10076000E273B3F5487F6BDA494B1B78002B40F0FE
:100770001181484B3B4A1B68126847489B1AB3F5E6
:10078000FA7FA8BF4FF4FA739842B8BF18460A21FF
:1007900004F060FD414B1C68637A00FB03F0002805
:1007A000B8BF7F30C211B2F5967F3D4BA8BF4FF462
:1007B00096729A42B8BF1A463A48E37E076895EDAA
:1007C000087ADFED396A911B01FB03F3227F344E77
:1007D000002B01FB0272B8BF1F335B11B2F5C81FBB
:1007E0003249A8BF4FF4C812B3F5967FA8BF4FF4A3
:1007F00096738A42B8BF0A46617F026007EE901A7C
:1008000037EE087AF8EEE77A27EE267AB34267EEFB
:10081000877AB8BF3346002AB8BF02F5FF52FDEE13
:10082000E77AB8BF1F3203EB623317EE902A962A9D
:100830006FF09501A8BF96228A42ACBF9F1A5F1A3B
:100840001B4A85ED088A17607CE600BF24B70020AC
:10085000A42C002008942537B1DC423ED048874ABA
:100860006F12833A28B70020A0640020BD37863578
:10087000906400201C6A002018970020216C002042
:100880000024744924FAFFFF30B700202CB7002061
:10089000DC300020D43000200CFEFFFF84B70020A5
:1008A000D4FEFFFFCC3000200000003B0000E7FF3B
:1008B000C430002082BC002048B900209C64002085
:1008C000374998F806A00A68AB689FED360ADFED55
:1008D000360A002A0AF1FF3AB3FBFAF39246B8BF90
:1008E00002F1070AA2EBEA0203EB020ABAF1000FD7
:1008F0005346B8BF0AF10703DB1007EE903AF8EE53
:10090000E77AC1F800A027EE800A32F08DF9F7EE01
:10091000007A77EEC07A9FED257A2B6967EE877AA9
:100920009A4518BF07F1FF33FDEEE77A14BF9FB277
:1009300000274FF00003C5ED037A18BFC5F810A0DB
:10094000A9F800706B61AB61002252E69FED188A36
:10095000DFF870E0174C184B9FE695ED057AD5ED62
:10096000067ADFF864C02068996891FBF0F1BDEE6B
:10097000C77AFDEEE77A17EE100A17EE909AACF8F8
:100980000200ACF80010ACF804908BE69FED088AEA
:10099000094B4BE6094A0A4B12681C680CE700BF7A
:1009A0007800002008942537B1DC423ED048874AC1
:1009B00000000000A064002090640020D8300020D7
:1009C00084B700209C640020246C00202DE9F843AB
:1009D000304B1B685B0701D4BDE8F8832E4C2F4DCC
:1009E00094F82490B9F1010F48D1EB692846984753
:1009F0002B69284698472B6A04F12C0004F1280142
:100A00009847274B276B9B79A668E06A07F1010896
:100A10009845636B08BF84F8009003F1010208BF9A
:100A20004FF00008032A1FD01E49626394F8382053
:100A300041F82300FAB904EB870704EB8803F86355
:100A4000DA6BAB89C4F83080B61A30440022A0605B
:100A500084F82420002BBFD0134A0A2B1268B8BF99
:100A60000A231361BDE8F8830E4B0122986000232E
:100A700084F8382063631BF095FBDCE76B6928463C
:100A80009847AB69284698470122EB8984F82420CF
:100A9000E0E700BF24B70020A42C00201897002016
:100AA00048B90020B057002068B90020F8B5534B72
:100AB0001B681C0700D4F8BD514C524E524D736850
:100AC00004F1FC01074630469847B4F9FC00B4F93C
:100AD000FE20B4F90031317E286028466A60AB60A0
:100AE00013F0B2FD494A137859073ED4D4F80401F3
:100AF000474B1B7883B1474B2968B3F90AC0B3F958
:100B00000CE0B3F90E606A68AB68A1EB0C01A2EBD4
:100B10000E029B1B85E80E000028CCD03E4B381AF5
:100B200098423FD9B4F91451B4F91011B4F90871CD
:100B3000B4F90A21B4F91261B4F90C3135483944D9
:100B400032442B4401EBD17102EBD27203EBD3732D
:100B50005B1049105210002541818281C381C4F885
:100B60000451BDE8F840F8F759B82C4EB5F900002B
:100B7000B5F90410A4F8080123F00403137000224F
:100B8000B5F90830A4F81001C4F804713260B280DD
:100B9000A4F80A11A4F81211A4F80C31A4F8143125
:100BA0003846A5E70020F9F7DFF92B68B4F90821EA
:100BB0009342B4F91021B8BFA4F808319342C8BFDA
:100BC000A4F81031B4F90A216B689342B4F91221E8
:100BD000B8BFA4F80A319342C8BFA4F81231B4F9DF
:100BE0000C21AB689A42B4F91421C8BFA4F80C31A7
:100BF0009A42BFF660AFA4F81431F8BD24B70020C4
:100C0000A42C0020243C002094B0002082B70020B7
:100C1000443C0020509900207FC3C9015A9900200C
:100C20002DE9F047C74C636820469847002800F03C
:100C3000C380C54B1B780122042B84F83C2000F0B4
:100C4000BD80B4F91610B4F91820B4F91A30216334
:100C50006263A363BD4B1B88002B69D0BC4DD4EDF0
:100C60000C7AD5ED004A95ED050A95ED015A95ED02
:100C7000067AD5ED035A95ED026AF8EEE76AD5EDEE
:100C8000047AA4EEA60AA5EE267A67EEC07AA5EE4F
:100C9000C07AE6EE267A85ED057AC5ED067A31F062
:100CA000FBFED4ED0D6AD5ED094A95ED0E0A95EDE2
:100CB0000A5A95ED0F7AD5ED0D7AD5ED0C5A95EDD2
:100CC0000B6A2063F8EEE66AA4EEA60AA5EE267A81
:100CD00067EEC07AA5EEC07AE6EE267A85ED0E7A4A
:100CE000C5ED0F7A31F0D8FED4ED0E6AD5ED124A7B
:100CF00095ED170A95ED135A95ED187AD5ED167AFC
:100D0000D5ED155A95ED146A6063F8EEE66AA6EE25
:100D1000A40AA6EE857A67EEC07AA0EE657AE6EEC2
:100D2000867A85ED177AC5ED187A31F0B5FEA063A5
:100D3000884FA17F884813F087FC3B88002B40F048
:100D40008480864ED6F81851854B1B685B0743D4C8
:100D5000B5F90070216B636BA06B824A824E92EDF5
:100D6000026AD2ED006AD2ED015AC91B2163B5F9BE
:100D70000270DB1B6363B5F904703568C01B07EEB6
:100D8000900AB8EEE75A07EE901AB8EEE77A07EE47
:100D9000903AF8EEE77A36EE056A36EE877A77EE25
:100DA000A57A0135A06382ED026A82ED007AC2ED78
:100DB000017A3560BDE8F087BDE8F0876B4BB4F988
:100DC0001600B4F91810B4F91A201880206359805D
:100DD00061639A80A2633DE7B6F82821322A00F0C9
:100DE0008880002A66D196F84631002BB0D0604842
:100DF000D6F838215F4980FB0273D217C2EB231269
:100E00002A80D6F83C2180FB0273D217C2EB231252
:100E10006A80D6F84031A78A80FB0302DB17C3EB58
:100E20002213DB1BAB800023CB6086F846310EF02B
:100E300023FD03F0DBFC0EF007FDF7F74FFD01206B
:100E40002CF05AF8D6F8185182E7444E226BD6F8A7
:100E50001851B3F5C87F4FF0000323632B80398806
:100E600018BFD6F81C01B7F8008008BF0020B1F504
:100E7000C87F18BFD6F82031616B02440B440020B4
:100E8000B8F5C87F6063C6F81C21C6F820316880B9
:100E900052D0D4F838E0D6F82411A0637144B8F1E8
:100EA000010FA880C6F8241168D008F1FF38A7F810
:100EB000008049E7D6F83801236B00210344C6F8C7
:100EC000383121632980D6F83C01636B61630344A8
:100ED000C6F83C316980A36BD6F84001A163034496
:100EE000012AC6F84031A98075D0013AA6F8282118
:100EF00079E72B8820491F48276BA6F82C3100235F
:100F0000B5F802E0B5F804C0C0684B608B6023639D
:100F1000C6F838712B80616BC6F83C1163636B8037
:100F2000A16BC6F84011A363A6F82EE1A6F830C164
:100F3000C6F83401AB80D8E7A36BC6F82431A063B0
:100F4000A880B2E738B70020216C00205638002076
:100F50005838002084BC002068B70020A42C002052
:100F6000509500205C64002058640020246C002010
:100F70001F85EB5140990020DC2D0020DFF88CC04C
:100F8000DFF884E0C8328CFB02A9C833D217C2EB69
:100F9000E9128CFB03A9DB17C3EBE913C8316B80A3
:100FA0002A808CFB013CA28ACB17C3EBEC139B1A63
:100FB000AB80CEF80C000EF05FFC03F017FC0EF0D7
:100FC00043FCF7F78BFC40462BF096FFB7F8008008
:100FD000D6F8185169E70B2086F8441186F84521A8
:100FE0002BF064FED6F81851074BB6F82C21B6F852
:100FF0002E71B6F83001D6F834112A806F80A8809F
:10100000B6F82821D96070E7409900201F85EB5180
:101010002DE9F04F2DED028BA74BA84A1C7897B015
:1010200000F59C41203181460A911160002C00F0AE
:101030001485A34A1268904240F2E680A14A0792C2
:101040001668A149A14A0691013C1C70A04B04926C
:1010500006F480560993002E40F0E4809D4B1B78E7
:10106000022B00F07387042B00F06287012B00F045
:101070001687994B9945099B9B7800F2BE83002BFC
:1010800040F0BF83954B0893079B1E6816F480576A
:1010900040F0B184DFF87492049BB3F90620069BFC
:1010A0005C8BA242B4BF002401248D4B1B68D90085
:1010B00040F1C280089B1B7813F0010300F0C3804D
:1010C0000699498C914241F35680002C40F0C28031
:1010D000844D95F8D421002A40F0BC80824A83498F
:1010E000106890F82D0000220A604A608A60804AE9
:1010F000002840F0B0801070002B40F0B1807D4B94
:101100001A78002A40F00E810699049D488BB5F9A3
:101110000070898BB5F902508742CCBF802600262B
:1011200046F040038F42A8BF33469B0843F0800639
:101130008542C8BF3346049F43F040068D42B8BF86
:1011400033469B08B7F90450B7F9066043F08007AF
:101150008542C8BF3B4643F040078D42B8BF3B467F
:101160009B0843F080075F4D8642C8BF3B4643F073
:10117000400795F8D6E18E42B8BF3B469E4501F048
:101180003782A5F8D82185F8DA215B4985F8D63170
:101190000E78002E01F049815F2B01F0D3816F2B77
:1011A00001F01282089B1B78DB0700F1BB8095F8E9
:1011B000DA11002940F0B680B5F9D831322B40F36E
:1011C000B18095F8D6210120572A85F8DA0101F07F
:1011D0002685079B1B685C0741F164805A2A41F011
:1011E000618095F84531002B41F0CA8695F8DC31D5
:1011F00083F0010385F8DC31002B41F04B870C2094
:101200002BF054FD01F0B2B92E4B07931E682F4B03
:101210002D4A049306F480562D4B06920993002E16
:101220003FF41CAF00212E4804F0E5FA00287FF4BB
:1012300015AF10F04FFA11E773023FF53BAF089B73
:101240001B7803F00103274D002285F8D421002CE0
:101250003FF444AF264A01211170002B3FF44FAFF9
:10126000F6067FF54CAF254B1B78DD063FF547AF03
:10127000002F7FF444AF1DF0C3FD00287FF43FAF83
:101280001D4B1B78002B01F06B861D4B9B78002CAF
:1012900041F0E0863BB11B4A1B4B12681B689B1A4E
:1012A000002BC1F2F08610200E4D2BF0FFFC012325
:1012B00085F8D53123E700BFDC3400207C330020E3
:1012C000D834002050950020F48B0020DCAD0020A5
:1012D000AC3C0020E43B0020404B4C00105100206F
:1012E0009C970020A42C002084B7002000970020A9
:1012F0007C3000200BB100203723002082B7002073
:1013000060990020E86B0020D4360020943500203E
:101310000F202BF0CBFCB5F8D83185F8DA41FA3B39
:10132000A5F8D831079BB14A1B680592B04C5F07FE
:1013300000F18B840DF1500ADFF8DC820A94002260
:10134000CAF804204546149240F6330B192740F2A0
:101350008336049C02E004354D4520D0A978EB7813
:10136000994217FB0160F6D26978043117FB0363D9
:1013700034F911105945A8BF5946B1F5617FB8BF7E
:101380004FF461718142E6DD9942E4DC2978272936
:10139000E1D85046043504F01FFA4D45DED1954A98
:1013A0000A9C1378944A9AE8030082E80300002B11
:1013B00040F01781914B1F78002F00F0BF8301216F
:1013C0008D4804F018FA002840F04A81099BDB7828
:1013D000002B40F0458123881DB225F00105AEB2F7
:1013E000B342268000F0D785854D02270E204FF0AE
:1013F00014094FF0FF082F7085F8019085F80280DE
:101400002BF054FC39467C48268804F0F4F9002877
:1014100041F0698026F002039BB2B34223800AD0D8
:10142000774B1421FF2202250E201D7059709A70EF
:101430002BF03CFC2688DFF8E4A1DFF8E4B19AF851
:101440000010DBF80400B50708BF81F00201C1F30A
:10145000400102F04DFE2421674804F0CCF930B978
:10146000089A1378590744BF23F004031370059BAF
:101470001B6813F00A0F1DD005215F4804F0BBF96B
:10148000002800F04E8625886F0740F1E3875A4810
:10149000062104F0B0F9002800F030866E0640F115
:1014A000D1870721544804F0A6F9002840F0CE85E2
:1014B000059B1B689D0600F1128326884E480C216F
:1014C00004F099F9002800F0E68046F48073B342F6
:1014D000238009D04A4B02251421FF220E201D70C3
:1014E00059709A702BF0E2FB464B1B78082B00F0EA
:1014F000DE800E2B00F0DB80079B1B685D0548D566
:10150000414B1B79002B00F08F8014213A4804F0E6
:1015100072F9002840F08D802CF04CFC01202BF05B
:10152000CFFA002835D0DFF8FC8000254FF0CC0939
:1015300002E0DDB2022D2CD809FB05F76B1C58F830
:101540000760002EF5D1032290F902300296019235
:10155000C2782E4951F8222000921846324633466E
:1015600001212AF0A3FE034605EB450000EB001025
:10157000069353B1314608EB8000CC2232F049FA91
:10158000069B48F807300135EDB224F0CBFC00286B
:10159000D0D1089B1B78D80740F19C809AF80010A6
:1015A0001B4A1C4DDBF80000012301F00101137000
:1015B0002B7002F09DFD059B1B685A0700F1FE8011
:1015C00017B0BDEC028BBDE8F08F98F8022098F8B8
:1015D00003309A42C0F05B8608F1040845453FF4A9
:1015E000E9AE98F800102329F6D1EEE724B70020E1
:1015F00080B70020205400209C9700204CB0002091
:10160000946F00207099002098BA00208875040813
:10161000E83000201151002044350020B06B00203C
:10162000B46B002064600020089B1B78D9077FF50D
:1016300073AF4FF40F701AF07BFF0028A9D021F090
:1016400069FB4FF40F701AF00BFF0028A1D021F0B6
:1016500061FB4FF40F701AF003FF0028EFD198E7F9
:10166000059B1B689A077FF5B6AE2688F3073FF502
:10167000D1AE46F001039E4223803FF4CBAEB74B80
:101680001421FF2202250E201D7059709A702BF034
:101690000DFB2688BEE626F480739BB2B3422380FE
:1016A0007FF418AFAE4B1B78082B7FF422AF228853
:1016B00022F040039BB29A4223803FF41DAFA74B18
:1016C00002251421FF220E201D7059709A702BF0F4
:1016D000EDFA11E7A34B1E78002E65D1A24B1B68D3
:1016E000002B61D0DFF8CC82DFF8CC9218F8030C25
:1016F00099F804704146A8F103051DF057FB002836
:1017000000F06485002F40F0B58505F10801687987
:101710001DF04CFB002841F007849449A87A1DF085
:1017200045FB002800F06585022F41F005849049B3
:10173000E87B1DF03BFB002841F0FA838D49287DB2
:101740001DF034FB002800F06585042F41F004846F
:101750008949687E1DF02AFB002841F0F9838749FA
:10176000A87F1DF023FB002800F06585062F41F0BF
:10177000EB83834995F823001DF018FB002841F006
:10178000DF83804995F828001DF010FB002800F049
:101790006585082F41F0B0837B4995F82D001DF039
:1017A00005FB002840F06585784B01221A702DF06A
:1017B00051FE059B1B685A077FF502AF03201DF001
:1017C0002DFB002800F02C87238813F008047FF4F9
:1017D000F7AE08200AF0ECFA049E6D486D4D6E4994
:1017E0006E4A6F4BF68800682E80086014601C609B
:1017F00017B0BDEC028BBDE8F08F13B9099A012335
:101800009370684B099A1D7892F8214008931B2029
:101810001DF004FB012C05F00108814600F0AD86A7
:1018200005F00205099A604E92F82030DFF88CA18D
:101830005E4F05959346052B00F2F786DFE813F01F
:10184000C00084000600FE000001F300012C04BF6C
:1018500005238BF82030B8F1000F12D0069B30889A
:10186000B3F918100022134661F30F0260F31F4210
:1018700061F30F03049861F31F4303600323426085
:1018800005934B4DDBF814102A68914280F0BD851A
:1018900047F230510322CBF81C108BF82020022095
:1018A0000AF09EFA0FF016FF2968DBF81C200A44A4
:1018B0000421CBF818208BF82010012C40F0FD8675
:1018C0002A68DBF81810914280F0AF869AF8000081
:1018D00020B91DF0A3FA002840F0A7863A6822F04C
:1018E00002023A602A687388642101FB03234FF4E3
:1018F00080600022CBF810308BF820208BF803207A
:101900000AF03EFA9BF8203095E71DF08DFA012889
:1019100007D1274D72882B68642101FB0233CBF875
:101920001030B9F1000F02D0B379002B7DD1012C1A
:1019300000F07B861E4DDBF810102A689142C0F043
:10194000C98601238BF82030012C6CD0F379012B50
:1019500078D01DF0E9F99BF820306CE7946F0020F7
:10196000709900201151002014510020586F002060
:101970005D6F0020626F0020676F00206C6F002099
:10198000716F0020766F00207B6F0020E830002010
:1019900028B70020C8300020D4300020CC300020F0
:1019A000C430002010510020206A00207CB70020A5
:1019B000E86B00204E6F00207800002037230020C5
:1019C000B8F1000FA1D1059D4FF48060B9F1000F6F
:1019D00000F0FF820AF0ECF9099A00231361002D50
:1019E0003FF452AB28462BF061F9079B1E6816F4B2
:1019F00080573FF44FAB1D21A64803F0FCFE0028A2
:101A00007FF448ABA44B03F1500903E0043399453C
:101A100000F011861A78262AF8D19978DA7891425E
:101A2000F4D2FFF739BB9D4D5CE71DF07DF9032231
:101A30004FF47A738BF82020CBF81C30974D2EE7AB
:101A4000964D3AE71DF070F9032240F6B8338BF853
:101A50002020CBF81C30914D21E7914F3B78002B93
:101A600001F03E818F4BDFF87082DFF870B2DFF853
:101A700070A2069345465E46049099460EE019F81A
:101A800004109847032C28DC88B93B782AF8020F09
:101A900001349C4205F1040580F22A81072CE1B251
:101AA0003046DBF80430EADD984700B2EDE738F85D
:101AB00024206B88801A4FF47A719B1A01FB00F086
:101AC00040F6CA0290FBF3F00844904240F2EE2345
:101AD000A8BF10469842B8BF184600B2D5E7724B6F
:101AE0001B78980704D5714D2B7D042B00F22686B8
:101AF000268816F0300F3FF4E1AC10200AF040F9D0
:101B000020200AF03DF96A4B268800221A70694AA3
:101B100069486A4F6A4D002111606A4A39600023A2
:101B2000296041608161036083604361C361136028
:101B30005160936053619161D361BFE4DFF8A4A168
:101B4000DFF8A481604D0AF15A064FF001095146B1
:101B50001AF8010C1DF02AF9F8B19AF804009AF865
:101B600002309AF803E000EB400105EB8101013BF4
:101B7000D1F8E42103EB4303434493420DD095F89D
:101B8000102281F8E0E109FA00F022EA0000C1F831
:101B9000E431C1F8E87185F810020AF1060A5645E9
:101BA000D5D14A493D4A4A4B09681B78D2F8008092
:101BB000DFF838910B910A934FF0FF3B4FF0000A8A
:101BC000D9F80430002B37D01E78002E34D0D9F845
:101BD0000820A8EB0202002A11DB3B4D012195F8F9
:101BE000102201FA0AF122EA010285F81022394A8C
:101BF00008F5FA704FF0FF31C9F8080011600A9A31
:101C0000D2B199F8002059780432D2B2002940F0BC
:101C1000B88206990498098B30F9122001F1C800A6
:101C2000824240F31A85284D9A7895F8103243FA8B
:101C30000AF3D80740F1C2850AF1010ABAF1040F8C
:101C400009F10C09BCD1FFF7BABB1F4D95F8DC3187
:101C50005BB1089B1B78DE0707D5049BB3F9062010
:101C6000069B5B8B9A4200F398851121094803F08B
:101C7000C2FD002800F06D8295F844312BB995F82B
:101C8000453113B93223A5F82831012385F84431B1
:101C9000FFF750BB9C97002044350020E86B0020E4
:101CA00008360020F48B002082B70020C0570020A7
:101CB000E83E0020D43F0020843F00205030002028
:101CC00044310020AC3F0020A42C002088B7002025
:101CD000A03C0020C00000201C360020ACB000203A
:101CE000EA2D0020656E0020943F0408842E002019
:101CF000DDF81090B84AB94907921268A1FB091B98
:101D000042F2010111404FEA9B1B0F9100F01E822D
:101D1000B34DB448B44CB5492E780078267008709D
:101D20001EB1B2490E7886F00106B14D0F2185F83B
:101D30006C11002B00F0AB83AE4B069C0E93B4F8F5
:101D400024E0B4F826C0069CCDF82CC01846248B9D
:101D50000078A94B1294A94C0D9004940446A3FB5F
:101D600000035B0803EB4303E31ADBB295F86D81D4
:101D7000099302F4805205F5B8700BF5967311952E
:101D800097F800A0DFF8BCC29C4C0C917546DDF8BA
:101D90003CE01392002108930596CDF84090059BF6
:101DA000002B00F0A582964B33F911301FFA83F90E
:101DB000A9454FEA410203D30B9EB14540F2DC82B4
:101DC0005CF821309B4580F09C82A35EBEF1000F41
:101DD00040F0B18201315145A35200F10600DEDB33
:101DE0000C9A119D874B85F86C210F2A0CBF01229C
:101DF0000022DDF8409085F86D811A7000F04E8366
:101E0000814B7849794ADFF840B209931C46042097
:101E100001230B70137009F0E3FFDBF80030A168B9
:101E20006268E3605B1A934284BF002384F8213028
:101E3000079B3C781E68002C00F06987069A734D5A
:101E4000B2F824E0178B6D4916F48056284640F00E
:101E50005B8332460EE0437803EB830303EB83039B
:101E600003F2EE239BB20132A24221F8023B00F1C1
:101E700002000ED015F81230002B00F0B182022BB8
:101E8000E9D001320B8821F8023BA24200F10200A6
:101E9000F0D10E9A137801331370FFF7DCB8544D6C
:101EA000D5F8D031A9EB0303002BFFF6E2A8584A7E
:101EB000584B527C069933F812308A7DDFED566A12
:101EC0009FED566AC97D9BB207EE102A07EE903A45
:101ED000B8EEC77AF8EEE77A27EE267A67EE867ACA
:101EE0000A9AC5F8D021C7EE876A40F2FF32FCEEAD
:101EF000E67ACDED057ABDF81430934228BF13463B
:101F000009B1D31A9BB24648464D0178464C35F884
:101F10001160226825F81130921B13440131434DA2
:101F2000236001F00F021B0902702B80FFF7A1B89C
:101F3000F7F792FC3E4B3F4A1B68C31A93427FF768
:101F400098A83A4B00221A80FFF793B8069A049992
:101F5000537DD27D013B31F913301AB1C3F53B6398
:101F600008331BB2A3F57A7307EE903A9FED327AED
:101F70002E4AF8EEE77A40F2FF3167EE877AFCEE00
:101F8000E77ACDED057ABDF814308B4228BF0B46B9
:101F90001380FFF76EB80221284803F02CFC0028BC
:101FA0003FF438AA2580B7073FF545AA46F002035B
:101FB000B34223803FF43FAA214B02201421FF2289
:101FC00018700E2059709A702AF070FE2688FFF75C
:101FD00032BA09F0D5FEFFE450950020D34D6210CF
:101FE000583300209C000020A03C00209D000020D1
:101FF000A42C0020F9340020ABAAAAAADCAD002052
:10200000EC2D00201AB10020AC3C002050360020FE
:10201000F06B0020106C00200000C84200008044DB
:10202000E53B0020EC3B0020E83B00205442002030
:102030008825002060E316006F12833F9C970020E4
:10204000946F0020FC340020E86B0020CC4AB2F9E9
:102050000030002BB8BF5B42B3F5E17FBFF628AA82
:10206000B2F90230002BB8BF5B42B3F5E17FBFF697
:102070001FAAC44B93ED057AD3ED077AD3ED096A15
:1020800093ED030A77EEA67A30EE070AF7EE000A20
:10209000B0EE007AE7EEC70A30EE000A03F0F8F877
:1020A000B6EE008A20EE488A9FEDB70A38EE000AA5
:1020B000FDEEC07A17EE903A2033402B40F27B833E
:1020C0009FEDB20AB24DDFEDB17A85ED000ABDEEAB
:1020D000C87AC5ED017A17EE103A2033402BC5EDD2
:1020E000027A00F2BB85B0EE480A03F047F80A20F6
:1020F00085ED030A2AF0DAFDFFF7DAB925F040038F
:102100009BB2AB4223803FF4CCA9A24B0225142101
:10211000FF220E201D7059709A702AF0C7FDFFF73C
:10212000C0B9238823F00405ADB2AB4225803FF44B
:10213000AEA9984B02251421FF220E201D70597064
:102140009A702AF0B3FD2588FFF7A1B992490E785D
:10215000E6E595F84531002B3FF4ECA8089B1B7889
:1021600013F001037FF4E6A8012285F8453185F8D4
:102170004621FFF7DFB8894D012285F8D421FFF70A
:1021800069B8012900F02B85BBF1FF3F834D0BD0CF
:102190001B780C2B08D0824B824A03EB8606824BBD
:1021A000C3F800B0736C136095F81022012303FA92
:1021B0000AF30AF1010A1343BAF1040F85F8103249
:1021C00009F10C097FF4FCACFFF7F9B808F105013F
:1021D00068791CF0EBFD00283FF49FAA012F40F026
:1021E000A38605F10D01A87A1CF0E0FD002840F05F
:1021F000A3866E49E87B1CF0D9FD00283FF49EAA17
:10220000032F40F095866A49287D1CF0CFFD0028F9
:1022100040F0A2866749687E1CF0C8FD00283FF4A4
:102220009EAA052F40F094866349A87F1CF0BEFD4E
:10223000002840F08986614995F823001CF0B6FD1E
:1022400000283FF49EAA072F40F07A865C4995F853
:1022500028001CF0ABFD002840F04E86594995F847
:102260002D001CF0A3FD00283FF49EAA092F3FF487
:102270009BAA0926334603EB83031D44524B69781E
:10228000AA7889F8046019705A70FFF78DBA4F4820
:1022900003F0B1FA00283FF48DA814202AF006FDBF
:1022A000FFF788B85D2A00F08E825B2A00F01C855B
:1022B0005E2A00F07485562A00F00586972A00F001
:1022C0002186A72A00F05F85414C23889B0740F0B8
:1022D0002285A2F1B703072B00F29482DFE813F006
:1022E00083029202920292028E0292028C02900269
:1022F000002D3FD05CF821309B454FEA4102FFF4AE
:1023000064AD344B334E9B5C06EB0209002B00F0AE
:10231000DE80022B77D199F8013003EB830303EBC6
:10232000830303F2EE239BB2032963DD1BB2BEF1EC
:10233000000F3FF44FAD099E20F81630B8F1000FA2
:1023400003D10D9E022E7FF645AD0388B0F80290B2
:10235000B0F804804B4498441F4B0FFA88F883FB75
:1023600008631E4EA3EBE87326F802801BB24FF001
:1023700001082FE52B464A00089E4CF8216025E510
:1023800030B700200C010020DB0FC93F0000000027
:1023900084000020946F0020A03C0020A42C00208A
:1023A000943F0408204F0020C00000205D6F0020F3
:1023B000626F0020676F00206C6F0020716F00203B
:1023C000766F00207B6F0020185100209C97002022
:1023D00080B7002050360020565555555C2E002001
:1023E000D3B2022B04D9032B7FF44BAD73463AE5ED
:1023F0003B4638E5012606FA01F90C9E26EA090655
:102400001BB20C96E2E4A35A8EE7B84A1278002A6F
:102410007FF43EAAB8F1000F3FF43AAA012C40F035
:1024200004819BF82030FFF706BA3146B04803F02C
:10243000E2F9002800F0A48085F8DB610FF07AFD56
:10244000FEF7B0BE45F04003AB4223807FF45DAEA3
:10245000FFF727B845F004039D4223800AD0A54B1F
:1024600002251421FF220E201D7059709A702AF047
:102470001DFC2588A04BA14AB3F90430A04982FB7A
:102480000302DB17C3EBA2030B80FFF700B89D4BE1
:102490009D4A0E9201221A709C4B04931B21944872
:1024A00003F0A9F900287FF4ABAC994BDFF888B2B0
:1024B00009931946DBF80030CA688B609B1AC82B59
:1024C00000F21684079B1E6806F48056E1E4CBB246
:1024D000022B40F28183032B95D1129B139E002E79
:1024E00008BF2B4620E726F001039BB2B3422380AE
:1024F0003FF459AD0E202F7085F8019085F80280C9
:102500002AF0D4FB26884EE500220FE0437803EB47
:10251000830303EB830303F2EE239BB20132A24257
:1025200021F8023B00F102003FF4B3AC15F8123081
:102530001BB1022BEAD00B88F0E7D3B2032BFAD8F9
:102540003B46EBE7B2F5FA7FFEF6ECAE95F8DA31F2
:10255000002B7EF4E7AE089B1B78012213EA0204ED
:1025600085F8DA213EF4D4AE0FF0B4F8694B059348
:10257000079B694C1B68FEF7DABE0025FFF752B9CE
:10258000089B664A1B781060D8077EF510AE644B36
:102590001B78002B3EF4C6AE099BDB78002B7EF443
:1025A000C1AE95F8DB310133DBB2032B85F8DB31AB
:1025B0007EF6B8AE5B4B5B7813B9002C7EF4B2AEFE
:1025C0000FF088F8FEF7EEBDB2F5FA7FFEF6AAAE80
:1025D00095F8DA21002A7EF4A5AE089B1B7801212C
:1025E00085F8DA11D90700F154830FF0A3FCBDE799
:1025F0004D4A4E491068B5F9D821C66981FB0601DC
:102600008911F617701A00F5FF407F3082423EF7BD
:10261000BCAD891B0A4412B2A5F8D821FEF7B5BD9E
:10262000082009F0ADFBFEF7CBBF059D002D3EF461
:102630002BADFFF7D7B93E4A069BD488049A1B8B73
:10264000B2F90620191B8A4240F3A48023449A421F
:10265000B4BF00240124FEF728BDC8398A42354D95
:1026600080F289809A7895F8103243FA0AF3D907F4
:102670003FF5E2AA524201200C922AF03DFC731E63
:102680000C9A162B00F27783DFE813F0B401CD012A
:102690005B01880175019D01450144022A02100277
:1026A000E6017503880130019D01450144021701CF
:1026B000FE00E6008D0273025B02AB460999DBF86F
:1026C0000020CB69059D13448B61002D3EF4DCACEA
:1026D000FFF788B91CF028FB032140F6B8328BF8CD
:1026E0002010CBF81C20FFF7DAB800BF6C300020B8
:1026F0009C970020946F002030B7002067666666C4
:10270000F43F00201AB10020F9340020DCAD002095
:10271000AC3C002024B7002080B70020D836002031
:10272000A03C00206099002068B90020D34D6210C1
:10273000046A0020A42C0020E86B00200A201CF072
:102740006DFB26880746002800F08C82F10640F1D8
:10275000C083CE4D95F81872002F7EF4AFAE0D20D9
:102760002AF0A4FA012385F818322688002F7FF476
:10277000CEA9FEF7A3BE95F81032012202FA0AF2A2
:1027800023EA020308F5FA7285F81032C9F8082026
:10279000FFF752BA0124FEF788BC0021BC4803F0C1
:1027A0002AF800287FF461AA322385F8DC01A5F815
:1027B0002831FFF75ABA02F0E1FC83E4002A0CBF8B
:1027C0000120022058E7B34B00220120B249B34C4C
:1027D0000B60B34B227005932AF08EFB079BB14C24
:1027E0001B68FEF7A4BD012010F086F9AC4B0593E1
:1027F000079B1B68FEF79BBD0320F5E70020F3E76E
:102800000220F1E7792A00F013847A2A00F00A8482
:102810009E2A00F0FF839D2A00F0F583AE2A00F087
:10282000EB83AD2A00F0E183EF2A00F0DB83FD2A81
:1028300000F0C683FB2A00F03384FE2A00F02D84CA
:10284000F72A00F004847B2A00F0A383079B944AB4
:102850001B680592FEF76BBDD5F81402924F90F8F5
:1028600002B09344BBF1C80FA8BF4FF0C80B2BEACE
:10287000EB7B80F802B0BB78002B40F014841BF097
:10288000E1FBD9F8043083E4D5F81402864F90F8C0
:1028900001B09344BBF1C80FA8BF4FF0C80B2BEA9F
:1028A000EB7B80F801B0BB78002BE8D013205946B1
:1028B0001CF0FEFAD5F81402E1E7D5F814027A4FBD
:1028C00090F800B09344BBF1C80FA8BF4FF0C80BFD
:1028D0002BEAEB7B80F800B0BB78002BCFD0122026
:1028E00059461CF0E5FAD5F81402C8E76E4F0B996B
:1028F000BB7891F805B09344BBF1640FA8BF4FF0CB
:10290000640B2BEAEB7B81F805B0002B40F0AD8324
:10291000D5F81402B3E7D5F81402634F90F804B069
:10292000B9789344BBF1C80FA8BF4FF0C80B2BEA8E
:10293000EB7B80F804B0002940F0BD83102EA6D1B7
:102940009DE70B99584F91F804B09344BBF1640F85
:10295000A8BF4FF0640B2BEAEB7B81F804B01CF0AE
:10296000C1FABB78002BD3D0032059461CF0A0FA43
:10297000D5F8140283E70B994B4F91F807B0BB7859
:1029800093448BF3080B81F807B0002BC0D00520CF
:1029900059461CF08DFAD5F8140270E70B98424F97
:1029A00090F806B0B9789344BBF1640FA8BF4FF01C
:1029B000640B2BEAEB7B80F806B0002940F05C83C7
:1029C0000D2E94D1A4E7D5F81402374F90F803B038
:1029D000B9789344BBF1C80FA8BF4FF0C80B2BEADE
:1029E000EB7B80F803B0002940F028830F2E7FF4A2
:1029F00067AF44E70B992C4F91F800B09344BBF1BB
:102A0000FA0FA8BF4FF0FA0B2BEAEB7B81F800B06E
:102A1000BB78002B3FF47CAF012059461CF048FAEC
:102A2000D5F814022BE70B991F4F91F802B093448D
:102A3000BBF1640FA8BF4FF0640B2BEAEB7B81F86E
:102A400002B0BB78002B3FF463AF022059461CF064
:102A50002FFAD5F8140212E7D5F81402124F90F8A5
:102A600008B0BB789344BBF1C80FA8BF4FF0C80BA8
:102A70002BEAEB7B80F808B0002B3FF400AF0B2073
:102A800059461CF015FAD5F81402F8E6A42C0020DB
:102A90009C970020C499002084B700206C8C0020F3
:102AA00024B7002080B70020304F0020D5F8140252
:102AB000C44F90F807B0BB789344BBF1C80FA8BFD0
:102AC0004FF0C80B2BEAEB7B80F807B0002B3FF4EC
:102AD000D6AE0A2059461CF0EBF9D5F81402CEE622
:102AE000D5F81402B74F90F806B0BB789344BBF109
:102AF000C80FA8BF4FF0C80B2BEAEB7B80F806B0DD
:102B0000002B3FF4BCAE092059461CF0D1F9D5F892
:102B10001402B4E6D5F81402AA4F90F805B0B978BB
:102B20009344BBF1C80FA8BF4FF0C80B2BEAEB7B57
:102B300080F805B0002940F0CA82112E7FF48FAED4
:102B40009DE6D5F814029F4F90F836B0BB789344B9
:102B5000BBF1640FA8BF4FF0640B2BEAEB7B80F84E
:102B600036B0002B3FF48BAE594617201CF0A0F96D
:102B7000CEE6D5F81402934F90F837B0BB78934463
:102B8000BBF1FE0FA8BF4FF0FE0B2BEAEB7B80F8EA
:102B900037B0002B3FF473AE162059461CF088F96D
:102BA000D5F814026BE60B99864F91F801B0934467
:102BB000BBF5967FA8BF4FF4967B2BEAEB7B81F8A1
:102BC00001B0BB78002B3FF4A3AE152059461CF092
:102BD0006FF9D5F8140252E6129BFFF7A5BB0499D2
:102BE00093F802B031F91220B2F5617F4FF496618B
:102BF00091FBFBF156DB40F6330B9345A8BF9346A0
:102C00000C2EABF5617B9BFBF1FB5FFA8BFB00F0BD
:102C10007781182E00F06B816B4DFFF7B9BA6B4BC3
:102C20006B491A684FF47A73B3FBF2F3C3EB4312A8
:102C300003EB8202079B1B68D2001F06A1F8A820A5
:102C400000F1B180634A0592126855077EF56EABBC
:102C5000614A624C0A211180FEF769BBB0EE670A37
:102C6000FFF745BAF20600F103810B201CF0D6F8FD
:102C7000002840F0C780B30600F14F81524D95F80F
:102C80001832002B3FF46BAD002F7EF440AFFEF7FF
:102C900015BC5349079B0A604E4A1B6805924F4C6E
:102CA000FEF745BB0C2E40F0EB800025AB464D4AAD
:102CB0005278AA42B0D0434F28460FF01DFFBB7890
:102CC0001BB159460C201CF0F3F86B1C3E4DDBB2D7
:102CD00013B118462AF010F9D9F80430FFF758BAA2
:102CE000414A0692FFF706B8404B012202206DE5EB
:102CF0003F4A079B1E68136823F004031360099A78
:102D0000012306F4805682F82130FFF7C2B806F49A
:102D10008056FFF7BEB80023BB2A149300F04D8104
:102D2000B72A00F04681BE2A00F04181BD2A7FF417
:102D300069AD4FF6FE712F4A2648D68905909089D5
:102D4000334401449181D3810CF096FD01F04EFD96
:102D50000CF07AFDF5F7C2FD01202AF0CDF8B5F8A8
:102D6000D821079BFA3A00211B68A5F8D82185F8DD
:102D7000DA11FEF7DCBAD5F814021BF063F94FF054
:102D8000FF3BFFF711BA1C49079B0A7811481B68E3
:102D9000059042F004020A70104CFEF7C8BA174BB7
:102DA0000222032012E5144A127896077FF54AAFF3
:102DB000134A127D042A7FF645AF12F037FF079BB6
:102DC0001B683FE7304F0020A42C002040950020D6
:102DD000648D002024B7002082BC002080B7002032
:102DE000D83600206C8C0020F48B0020129A002032
:102DF0007CB700204099002082B70020609A002014
:102E0000C0570020B64AB74B528993ED007A07EEBF
:102E1000902AF8EEE77AB0EEC77AB4EEE77AF1EEF0
:102E200010FA7FF528AF93ED017AB0EEC77AF4EE91
:102E3000C77AF1EE10FA7FF71EAFB3063FF51EAF6B
:102E4000202008F0B5FF95E80C00A7490A60084665
:102E500041F8043F21F012FBA44B01221A70A44D4B
:102E600095F81832002B00F02F812688FEF74FBE10
:102E7000102008F085FF9D4B26881F700127F4E67F
:102E8000182E40F091804FF0000B5A46984DD5F81F
:102E9000141291F817E0D0B270453FF479A9B2EB63
:102EA0000E02944FC87548BF0732D210B978531C30
:102EB000DBB200293FF40CAF594618200C931BF0ED
:102EC000F7FF0C9B04E7F5F7A9FE95F8D621FFF76D
:102ED000F5B9102008F06CFF202008F051FF86495A
:102EE000081F21F0CBFA814B02221A70B7E75A462D
:102EF000C82AA8BFC822C9E708263346FFF7BBB9CE
:102F00005D46D4E67D497E4A079B05914FF4C87122
:102F10001B6811807B4CFEF70ABA202008F030FFB6
:102F2000724B00221A709AE701263346FFF7A3B9C5
:102F300003263346FFF79FB902263346FFF79BB9B6
:102F400007263346FFF797B906263346FFF793B9AE
:102F500005263346FFF78FB904263346FFF78BB9B2
:102F6000002C3EF4A0A9624D95F8D531002B3EF41B
:102F7000C6A829F07FFE002385F8D531FEF7BFB83B
:102F80005E4B85F8451185F8460105935D4CFEF7CB
:102F90005DBE4FF4FA6102200FF0D8FC574B059349
:102FA000079B1B68FEF7C3B94FF0000B34E6022104
:102FB000C1E619464FF6FE73BDE619460223BAE68E
:102FC000002101200FF0C2FCB5F8D821079B4B4926
:102FD0001B680591963AA5F8D821002285F8DA21D8
:102FE000FEF7A5B900210846ECE7FF21002016F006
:102FF000ACFB95F8D62117E40121002016F0A5FBC3
:1030000095F8D6210DE40021FF2016F09EFB95F8DF
:10301000D62103E40021012016F097FB95F8D62174
:10302000FFF7F9BB384A137A43F0010313720DE43A
:10303000354A137A23F00103137207E40F2059462F
:103040000C921BF035FFD5F814020C9ACEE4002147
:103050000420B7E7002B86D02C492D4A09684FF48D
:103060007A7000FB031313607DE70E2059461BF0B6
:103070001FFFD5F8140202E459460D200C921BF0F4
:1030800017FF0C9A9CE41A4D0EF024FB85F8D541ED
:10309000FEF735B80B20FEF7B3B80021032091E707
:1030A000002102208EE7142059461BF001FFD5F8BD
:1030B0001402FFF7E4BB102059460C921BF0F8FEF7
:1030C000D5F814020C9A39E40127FFF748BB112008
:1030D00059460C921BF0ECFED5F814020C9A2CE524
:1030E000783F0020A8BA00206C250020E83E002090
:1030F000A42C0020304F0020E03E002024B7002008
:1031000084BC002080B7002000400020E86B002035
:10311000D43600202DE9F0478C4B1B78DB0707469F
:1031200044D58B4B8B4D1C788B4E012C59D01CD326
:10313000022C07D189498A4A09881288914201D90B
:1031400001241C70EB7AE3B12B89D3B1854B1B783A
:10315000BBB11FF01DFA002800F09B802B7B83423F
:103160002CBF0121002131700CE07C497E4A098886
:1031700010886A7B801A8842E2DAEB7A0024002BFE
:10318000E2D131782A79632A06D8022C774E00F0F2
:10319000BA803378002B5DD1754AAB7A8C4238BF48
:1031A0000C461470002B4CD1BDE8F0876B4B694D79
:1031B00019885B88E878CB1A83EAE3728142A2EB34
:1031C000E3721DD32B788B421AD3614B1C78E01E1F
:1031D000012861D96749097802294FD0012C5E4E38
:1031E000A5D15F4A5D491288687B0988121A91420D
:1031F00039DD5D4A12888A42A4D200241C70A1E7FE
:10320000B1EB400FE1DC524B1C78E11E012940F28A
:103210009480022ADEDC57494F4E0878DFF844815B
:10322000DFF844C1DFF838E10021032402283470BC
:103230001C7088F80010ACF80010AEF8001081D1B6
:103240001FE0012C71D0022C0BD10720BDE8F04704
:1032500029F02CBD7068381A474B984258DD7270BF
:103260009AE7BDE8F08702241C706BE7022AD2DDE2
:103270004049097802294FF0040464D13949364E97
:1032800009783E48022ACCBF00220122C2808180F8
:103290004BE70221317075E7022A9BDC95F800C0EC
:1032A00091FBFCFC0CF1010CBCF1080FDFF8B4A0A1
:1032B000304EA87895F801E096F800802A4CDFF8A7
:1032C000A090254EA8BF4FF0080C8AF800C01FFA46
:1032D0008CFA10FB0AF01EFB0AFE80B2DFF88CA00D
:1032E0002080A9F800E000244FF0640EB8F1020F2E
:1032F00034701C70CAF804408AF801E07FF439AFDA
:103300000FFA8CF1BDE73078A0B9012377603370F4
:10331000C2F164021A4B00FB02F083FB0023C017CA
:10332000A0EBA3506430707036E70820BDE8F0478A
:1033300029F0BCBC7368F81A8EE7032C96D10D49AE
:10334000097802299AD0044EFCE600BF10510020F3
:103350008070002014B700208670002090BA0020F2
:1033600084700020A6BA002082700020AC300020BB
:103370008C400020216C00207F969800246C002057
:103380006BCA5F6B10B5084B03F10C0193F9002079
:103390005C78845402449C78D470DC789471043353
:1033A0008B42F3D110BD00BF3C400408002870B52B
:1033B0001EDB0928044620DD012303EB83035B00A9
:1033C000B0FBF3F2092AF8D87BB10E4EB4FBF3F050
:1033D0000928CCBF57223022A6FB03E5024403FB99
:1033E0001044EB0801F8012BF0D100230B7070BDE5
:1033F0002D230B7040420131DBE7303001F8010B27
:10340000F3E700BFCDCCCCCC884230B44FF0010400
:103410002ED301FB04F4B0FBF4F58D42F9D284B154
:10342000AAB901E0B0FBF4F5092DCCBF5722302238
:103430002A4404FB150003F8012BB4FBF1F4002C23
:10344000F0D100221A7030BC7047B0FBF4F5092DA2
:10345000CCBF372230222A4404FB150003F8012B8D
:10346000B4FBF1F4002CF0D100221A7030BC70478C
:103470000546002AEBD1D7E72DE9F04714461D4653
:10348000064600234FF47A72204629462EF09AFE13
:10349000DFF848814B4A4C4F88FB00310144C31789
:1034A00082FB002EC3EB611188FB012887FB0027FC
:1034B0008644464AC3EBEE2EC1EB011C82FB0E296B
:1034C000A0EB8C0C0744424A86F806C0C3EB2747A2
:1034D0004FEAEE7C08EB010ACCEBA90C82FB0782D9
:1034E0004FEAE1780CEB4C0CC8EB6A18AEEBCC0E53
:1034F000C8EB0818DFF8E8C086F804E0A1EB880103
:1035000071718CFB0010F917C1EBE21240F2B5515A
:1035100001FB1272C3EBE050B2F5896F4FEA8007EE
:103520003FDA40F2DA239A4243DCB2F5B77FB4BF08
:103530004FF0000C4FF0010C4FEA4C08254B08EB04
:103540000C0103EBC1031FFA8CFE588C224908EBD7
:103550000C0301EBC30116310B2301E031F8020D1E
:1035600082421BDA013BF9D11A4BC44403EBCC0C69
:103570000123BCF80C00B37007F2B2770132121AC3
:10358000BE44F270A6F800E0204629464FF47A7255
:1035900000232EF017FE3281BDE8F0870133DBB245
:1035A000E9E74FF0030EF44640F296504FF006085C
:1035B000CCE74FF0020EF44640F229404FF00408E9
:1035C000C4E700BFC5B3A29107452EC2ABAAAA2A81
:1035D00073B06D163C400408484004088988888808
:1035E000792D031103685A1C0260197070472DE988
:1035F000F047089C2578002B804689460CBF4FF089
:10360000200A4FF0300A661C35B3002A29DD334604
:1036100001E0024698B113F8011B501E0029F8D1B1
:10362000971E60B13D46013D51464046C8476B1C60
:10363000002BF8DC257827EAE770013055B1041B30
:1036400029464046C847301916F8015B002DF7D1CE
:10365000BDE8F087BDE8F087002A04DC2846BDE815
:10366000F0870020EBE7571EDCE783684268D0ED67
:10367000037A00EB83010133934281ED040A8360F6
:1036800004BF0023836000EB830393ED047A036897
:1036900070EE277A9A42C0ED037A77EEC77AC0EDD2
:1036A000037A0CDA013307EE103AF8EEC76AB7EE88
:1036B000007A87EEA60A036030EE070A704707EE2D
:1036C000102AB8EEC77A87EE870A704790ED057A20
:1036D00090ED004AD0ED066AD0ED014AD0ED047AB3
:1036E00090ED035AD0ED025AA4EE007AB0EE406A93
:1036F000B0EE470AB0EE667AA6EE247A67EEC07A9C
:10370000A0EE457AE6EE257A80ED057AC0ED067AE0
:103710007047D0ED057A90ED013AD0ED003AD0ED4A
:10372000064A90ED024A90ED077A90ED035A90ED2B
:10373000086AD0ED045AC0ED067AF0EE406A27EE32
:10374000830AC0ED056AA3EEA60A80ED087AA4EE0E
:10375000240AA5EE470AA5EEC60A80ED070A7047BF
:10376000D0ED007A90ED017A30EE670AE7EE007A4C
:10377000B0EE670AC0ED007A704770470A44914284
:1037800014D030B40139551E41F2210211F8014F15
:10379000082380EA042004044CBF82EA4000400071
:1037A000013B80B2F7D18D42F0D130BC704700238D
:1037B000012243600360836043700371C2718372AE
:1037C0007047F8B50468C4F30D0405460E4604B30B
:1037D0002F6815F0ADFE092840F08880454C23691C
:1037E00023F440732361236943F400732361236945
:1037F00043F0010323613E6015F09AFE2369092816
:1038000023F00103236171D12B6804332B60002066
:10381000F8BD394B394A93422BD902F58042934285
:1038200026D902F5804293422AD902F5804293427A
:1038300028D902F58032934226D902F5003293420C
:1038400024D902F50032934222D902F50032934284
:1038500020D902F5003293421ED902F5802293420C
:103860001CD9B3F1016F1BD30520F4F767FEFBE70A
:10387000082415F05DFE092814D04FF0FF30F8BD84
:103880001024F6E71824F4E72024F2E72824F0E7D0
:103890003024EEE73824ECE74024EAE74824E8E760
:1038A0005824E6E7134F3B6923F440733B613B69BF
:1038B00043F400733B613B6923F0F8033B613B69D0
:1038C00043F002031C433C613B6943F480333B619A
:1038D00015F02EFE3B6923F002033B613B6909288A
:1038E00023F0F8033B613FF473AFC6E76FF00100CC
:1038F000F8BD00BF003C024000400008FF3F000848
:10390000F8B504460D468E180027B54201D120694E
:10391000F8BDE368591CE160234415F8012B1A72C5
:103920000429F2D1206918B9A1682046FFF749FFA0
:103930002061E760E9E7024B1868F6F7CBBA00BFF1
:103940001825002003682DE9F04F03F13F4404F5EA
:103950007E04604EA40A0125345D04F01F0664094C
:10396000032C05FA06F500F0AF80042C00F0A780C8
:10397000022C54D08588B5FA85F0C0F11F0080B2C2
:10398000C40803EB840400F00700266A80000F27B8
:10399000874026EA07062662276A01F0030602FA34
:1039A00000F0721E3843012AC1F3810CC1F30018E4
:1039B0002062C1F3411137D90024224601274FF07C
:1039C000030E03E0102A04F1020426D007FA02F0E5
:1039D000A84302F10102F5D1D3F800C00EFA04F0B9
:1039E000C04300EA0C0CC3F800C0D3F8008006FA0C
:1039F00004FC4CEA080CC3F800C0D3F80CC000EA81
:103A00000C00D860D3F80CC001FA04F040EA0C00B6
:103A1000102AD86004F10204D8D1BDE8F08F2E4CF2
:103A2000666C35436564A5E7002002464FF0010E41
:103A30004FF0030904E00132102A00F102003CD0EB
:103A40000EFA02F737EA0504F5D1D3F800A009FA17
:103A500000F4E4430AEA040AC3F800A0D3F800B073
:103A600006FA00FA4AEA0B0AC3F800A0D3F808A045
:103A700004EA0A0AC3F808A0D3F808B00CFA00FA5E
:103A80004AEA0B0AC3F808A0D3F804A02AEA0707F9
:103A90005F60D3F804A008FA02F747EA0A075F60FC
:103AA000DF683C40DC60DF6801FA00F401323C432F
:103AB000102ADC6000F10200C2D1BDE8F08F064C94
:103AC000266B3543256355E7034C266C3543256447
:103AD00050E700BF1C64040800380240026802F18D
:103AE0003F4303F57E032DE9F04F9B0A544DEB5CF9
:103AF00003F01F055B090124032B04FA05F400F011
:103B00009980042B00F09180022B3ED001F0030637
:103B1000731E012BC1F3810CC1F300188588C1F31A
:103B2000411137D90024234601274FF0030E03E04B
:103B3000102B04F1020426D007FA03F0A84303F186
:103B40000103F5D1D2F800C00EFA04F0C04300EA38
:103B50000C0CC2F800C0D2F8008006FA04FC4CEA53
:103B6000080CC2F800C0D2F80CC000EA0C00D0600B
:103B7000D2F80CC001FA04F040EA0C00102BD0601F
:103B800004F10204D8D1BDE8F08F2E4B5D6C2C43BC
:103B90005C64BBE7002003464FF0010E4FF00309C1
:103BA00004E00133102B00F102003CD00EFA03F7C1
:103BB00037EA0504F5D1D2F800A009FA00F4E4438D
:103BC0000AEA040AC2F800A0D2F800B006FA00FA25
:103BD0004AEA0B0AC2F800A0D2F808A004EA0A0ACE
:103BE000C2F808A0D2F808B00CFA00FA4AEA0B0AA8
:103BF000C2F808A0D2F804A02AEA07075760D2F852
:103C000004A008FA03F747EA0A075760D7683C4060
:103C1000D460D76801FA00F401333C43102BD46020
:103C200000F10200C2D1BDE8F08F064B1D6B2C43A2
:103C30001C636BE7034B1D6C2C431C6466E700BFE1
:103C40001C6404080038024010B50409013C032C30
:103C500017D80D4B33F8142000F00F0042FA00F390
:103C600013F001030DD0012303FA00F001381040D6
:103C70002EF0F8FA054A064B125D104403EBC00023
:103C800010BD002010BD00BF7865040874650408ED
:103C9000506A00202DE9F04F4A484B494B4B4C4CA1
:103CA0004FF0010A4FF002094FF004084FF0080CE2
:103CB0004FF0100E20274026802530F8022B12F0FE
:103CC000010F03D01960A3F804A0083312F0020F0B
:103CD00003D01960A3F80490083312F0040F03D046
:103CE0001960A3F80480083312F0080F03D019609C
:103CF000A3F804C0083312F0100F03D01960A3F822
:103D000004E0083312F0200F02D019609F800833BE
:103D100012F0400F02D019609E80083312F0800F1D
:103D200002D019609D80083312F4807F05D04FF4D3
:103D3000807B1960A3F804B0083312F4007F05D02B
:103D40004FF4007B1960A3F804B0083312F4806FBD
:103D500005D04FF4806B1960A3F804B0083312F457
:103D6000006F05D04FF4006B1960A3F804B008335E
:103D700012F4805F05D04FF4805B1960A3F804B0A3
:103D8000083312F4005F05D04FF4005B1960A3F80C
:103D900004B0083312F4804F05D04FF4804B196003
:103DA000A3F804B00833D20B04D04FF400421960DA
:103DB0009A80083301F58061A1427FF47EAFBDE8AF
:103DC000F08F00BF7865040800000240506A0020B0
:103DD0000010024000286AD003682DE9F04F03F17B
:103DE0003F4404F57E045F4EA40A0125345D04F0CF
:103DF0001F066409032C05FA06F559D0042C00F0BF
:103E0000AC80022C59D08588B5FA85F0C0F11F002E
:103E100080B2C40803EB840400F00700266A800027
:103E20000F27874026EA07062662276A01F0030665
:103E30008240701E3A430128C1F3810CC1F300187F
:103E40002262C1F341113DD90024224601274FF0DF
:103E5000030E03E0102A04F1020426D007FA02F050
:103E6000A84302F10102F5D1D3F800C00EFA04F024
:103E7000C04300EA0C0CC3F800C0D3F8008006FA77
:103E800004FC4CEA080CC3F800C0D3F80CC000EAEC
:103E90000C00D860D3F80CC001FA04F040EA0C0022
:103EA000102AD86004F10204D8D1BDE8F08F704721
:103EB0002D4C266C35432564A5E72B4C666C3543A9
:103EC0006564A0E7002002464FF0010E4FF00309A1
:103ED00004E00132102A00F102003CD00EFA02F791
:103EE00037EA0504F5D1D3F800A009FA00F4E44359
:103EF0000AEA040AC3F800A0D3F800B006FA00FAF0
:103F00004AEA0B0AC3F800A0D3F808A004EA0A0A98
:103F1000C3F808A0D3F808B00CFA00FA4AEA0B0A72
:103F2000C3F808A0D3F804A02AEA07075F60D3F813
:103F300004A008FA02F747EA0A075F60DF683C401E
:103F4000DC60DF6801FA00F401323C43102ADC60D7
:103F500000F10200C2D1BDE8F08F034C266B35435F
:103F6000256350E71C64040800380240002855D03F
:103F7000026802F13F4303F57E032DE9F04F9B0AEF
:103F8000544DEB5C03F01F055B090124032B04FA7D
:103F900005F444D0042B00F09780022B44D001F0AC
:103FA0000306731E012BC1F3810CC1F30018858831
:103FB000C1F341113DD90024234601274FF0030EE0
:103FC00003E0102B04F1020426D007FA03F0A84303
:103FD00003F10103F5D1D2F800C00EFA04F0C0439A
:103FE00000EA0C0CC2F800C0D2F8008006FA04FC0B
:103FF0004CEA080CC2F800C0D2F80CC000EA0C0071
:10400000D060D2F80CC001FA04F040EA0C00102B8A
:10401000D06004F10204D8D1BDE8F08F70472E4B78
:104020001D6C2C431C64BAE72B4B5D6C2C435C6409
:10403000B5E7002003464FF0010E4FF0030904E0FE
:104040000133102B00F102003CD00EFA03F737EADF
:104050000504F5D1D2F800A009FA00F4E4430AEA15
:10406000040AC2F800A0D2F800B006FA00FA4AEA40
:104070000B0AC2F800A0D2F808A004EA0A0AC2F8A3
:1040800008A0D2F808B00CFA00FA4AEA0B0AC2F803
:1040900008A0D2F804A02AEA07075760D2F804A0C3
:1040A00008FA03F747EA0A075760D7683C40D4602C
:1040B000D76801FA00F401333C43102BD46000F1BF
:1040C0000200C2D1BDE8F08F034B1D6B2C431C6373
:1040D00065E700BF1C6404080038024010B10368A3
:1040E00082885A83704710B1036882881A837047A8
:1040F00018B10368828809B95A8370471A837047D8
:1041000030B1036882881B691A4214BF0120002065
:1041100070472DE9F0410B4E346873691C400FD095
:10412000DFF824800127B4FA84F3C3F11F0307FAF0
:1041300003F558F8230003689847AC437561F2D142
:10414000BDE8F081003C0140C02E00202DE9F04187
:104150000B4E346873691C400FD0DFF828800127AC
:10416000B4FA84F3C3F11F0307FA03F558F82300E8
:1041700003689847AC437561F2D1BDE8F08100BF98
:10418000003C0140C02E00202DE9F0410B4E346868
:1041900073691C400FD0DFF828800127B4FA84F33C
:1041A000C3F11F0307FA03F558F823000368984783
:1041B000AC437561F2D1BDE8F08100BF003C014025
:1041C000C02E00202DE9F0410B4E346873691C406D
:1041D0000FD0DFF828800127B4FA84F3C3F11F035E
:1041E00007FA03F558F8230003689847AC43756154
:1041F000F2D1BDE8F08100BF003C0140C02E00209C
:104200002DE9F0410B4E346873691C400FD0DFF884
:1042100028800127B4FA84F3C3F11F0307FA03F5DA
:1042200058F8230003689847AC437561F2D1BDE8A4
:10423000F08100BF003C0140C02E00202DE9F0417C
:104240000B4E346873691C400FD0DFF828800127BB
:10425000B4FA84F3C3F11F0307FA03F558F82300F7
:1042600003689847AC437561F2D1BDE8F08100BFA7
:10427000003C0140C02E00202DE9F0410B4E346877
:1042800073691C400FD0DFF828800127B4FA84F34B
:10429000C3F11F0307FA03F558F823000368984792
:1042A000AC437561F2D1BDE8F08100BF003C014034
:1042B000C02E0020084A536C10B5084C43F48043CC
:1042C00053642046402200212FF0A3FB4FF0FF3320
:1042D0002364C4F8433010BD00380240C02E0020D3
:1042E00010B58B680160044698470022FF23012126
:1042F000A2736373217310BD03685B6A1847036878
:104300001B6A184770B44E1C0568C2728672AC698D
:10431000A44670BC60472DE9F041044618460D469E
:10432000164698462DF083FA2768E6722844A07254
:1043300029467D69434632462046AC46BDE8F041F9
:104340006047036810B504461B68984723682046F9
:104350009B689847A37B0133A37310BD03681B6957
:10436000184710B5036804469B689847FF2301224D
:104370006373227310BD08B5FFF766FC38B12D22B8
:1043800082710022C2712021BDE80840EEE508BD1F
:104390000E4B98420AD0A3F57843984211D003F50A
:1043A000806398420FD04FF0FF3070470022084BD7
:1043B00003EB02135A89013292B25A81588980B2B2
:1043C00070470122F3E70222F1E700BF003001400D
:1043D0004C6C00202DE9F0410578012D82B0064695
:1043E0002FD0022D35D1806841F0800110B10468D2
:1043F00080886083706840F2E93401E0002C70D05E
:104400000589013C15F0020FA4B2F7D089B2818171
:1044100040F2E93101E0002963D00489013914F048
:10442000010F89B2F7D0818900212CF0B7FDB36864
:10443000002B68D01A689B881383012002B0BDE866
:10444000F08190F904E0BEF1FF3F02D0BEF1030F0E
:1044500003DD002002B0BDE8F0814FEACE08DFF8AE
:10446000B0C008EB0E070CEB870778680028F1D086
:1044700074793A6264000026E4B2BC75F9757E7600
:10448000BD763B767D753E758388FA61990514D4B7
:104490000388DA050CD44FF4805401E0013C28D0A5
:1044A00003889B05FAD403889BB243F4807303808E
:1044B00083889BB243F440738380F0440CEB880202
:1044C0004FF4805401E0013C13D0537D002BFAD10E
:1044D0000CEB880898F8144084F0010002B0BDE8A5
:1044E000F0818DE80C00FFF753FF70689DE80C0029
:1044F0009AE7064A1388013370469BB213802BF06B
:104500004BFC2046A6E70120A4E700BF583100205D
:10451000D48200200378012B46D0022B42D12DE912
:10452000F041836801F07F0113B11C689B886383AD
:1045300005461746406840F2E93401E0002C3AD0C5
:104540000689013C16F0020FA4B2F7D089B281812E
:1045500040F2E93100E071B30389013913F0010F32
:1045600089B2F8D0838940F2E93100E039B3048997
:10457000013914F0020F89B2F8D0BFB2878140F23E
:10458000E93300E0DBB10289013B12F0010F9BB27D
:10459000F8D08389AB68ABB11A689B88138301207C
:1045A000BDE8F0810020704713460A46417990F932
:1045B00004002CF07DBBFFF7EBFE6868D3E7FFF744
:1045C000E7FEE7E70120BDE8F081427A02B97047D3
:1045D00010B504460368406804F10A0198470023B7
:1045E000637210BD437A5A1C0344D2B2427299726C
:1045F000037A934200D802B9704710B504460368A5
:10460000406804F10A0198470023637210BD50B35B
:104610000123302803FA01F122D0312820D032289A
:104620001ED033281CD034281ED035281CD020287A
:104630001AD0212818D0102812D0112810D01228F2
:104640000ED013280CD014280ED015280CD0162804
:1046500001D0172806D111F0030018BF01207047C0
:104660004A0703D1002070478B07FBD00120704719
:10467000302829D0312829D0322829D0332829D0F0
:10468000342829D0352829D0202829D0212829D0FC
:10469000102829D0112829D0122829D0132829D050
:1046A000142829D0152829D0162805D0172808BF86
:1046B0000F2302D0002070470E23114A03EB43035F
:1046C000134493F86E0070470023F6E70123F4E7E4
:1046D0000223F2E70323F0E70423EEE70523ECE7E8
:1046E0000623EAE70723E8E70823E6E70923E4E7E8
:1046F0000A23E2E70B23E0E70C23DEE70D23DCE7E8
:104700003C40040870B5448806460D46C4F30B04CB
:104710002246002128462FF07CF93369094A93424A
:1047200009D3094A934206D2224628461946BDE8D3
:1047300070402DF0DBBF23B121462846BDE8704014
:10474000184770BD6806000867070008064B074950
:104750008B4202D30023184670471A88C2F30B021B
:104760009042F8D01433F3E790010008680600087F
:10477000024A136823EA000010607047F49A002090
:10478000F8B5174D2B78A52B28D16B78BE2B25D1EA
:10479000022229464FF6FF70FEF7F0FF114FAC1CC6
:1047A00022884AB1A618BE4218D2052A16D9214637
:1047B000FEF7E4FF3446F3E721460222FEF7DEFF70
:1047C0000222A118FEF7DAFF0634074B641B1C8097
:1047D00041F60F53C31A58425841F8BD0020F8BDA6
:1047E00000400008008000085A3100202DE9F04FF9
:1047F000DFF84C914D4F8BB00326A7EB0907182229
:10480000002104A82FF005F9494BCDF81090059729
:104810001A69002A04DA474A5A6002F188325A605B
:1048200001228DF82420F322DA60434B434C1B888D
:10483000ADF800300222694604A8FFF761F80222B1
:1048400069464FF6FF70FEF799FFDFF8F8A0804643
:104850004FF0000B544539D30AAC002524F8245DF1
:104860000222214604A8FFF74BF8022221464046C7
:10487000FEF784FF40BAC043ADF80800022202A947
:1048800004A8FFF73DF8079878B106ABC0F1040221
:10489000294618442FF0BDF8089818B9069904A8BD
:1048A000FEF78FFF0023089007939DF82430089AA5
:1048B00023B11F490B6943F000430B61013E2DD02A
:1048C000002A9CD1FFF75CFF50B32CE065888DF87F
:1048D0000DB0C5F30B05AB1DADF808302388C3F34D
:1048E0000B02ADF80A201B0B062202A904A88DF8C2
:1048F0000C30FFF705F8062202A94046FEF73EFFFE
:10490000616880462A4604A8FEF7FAFF61684046BF
:104910002A46FEF733FF143480469BE7002AD1D0A5
:104920000520F3F70BFE0BB0BDE8F08F0080000808
:10493000003C024023016745D8400408900100086C
:1049400000400008680600080378202B024600F1AA
:104950000100F9D0092BF7D02D2B2CD02B2B03BF26
:104960005378B7EE000A0246B7EE000AA3F1300111
:10497000C8B209289FED467A10D8F2EE046A07EE15
:10498000901AF8EEE77A12F8013FE7EE267AA3F1E3
:104990003001C8B20928B0EE677AF0D92E2B4CD07E
:1049A00003F0DF03452B0BD0F7EE007A67EE276AA2
:1049B00020EE260A70475378BFEE000A0246D5E77C
:1049C00010B451782D2959D02B290ABF9178501C49
:1049D000901C0024A1F13003092B53D8002303EBD2
:1049E000830301EB430310F8011FA1F13002092AF0
:1049F000A3F13003F3D9B3F59A7F28BF4FF49A732C
:104A0000072B42D9DFED236A1A46F7EE007A083AFF
:104A1000072A67EEA67AFAD803F007032BB1F2EE65
:104A2000046A013B67EEA67AFBD124B3C7EE276A7E
:104A30005DF8044B20EE260A70475378A3F130014D
:104A4000C8B2092802F10102AAD8F2EE046AF0EE17
:104A5000665A07EE901AF8EEE77A12F8013F87EEF1
:104A6000A66AA3F13001C8B2092866EEA56A37EE3E
:104A7000067AEED994E767EE276AD9E7901C917819
:104A80000124A7E7F7EE007ACFE7F7EE007AC5E753
:104A90000000000020BCBE4CB5EEC00ADFED317A4C
:104AA000F1EE10FACCBF30EE270A30EE670ADFEDE8
:104AB0002E7A20EE270A30B5FDEEC07A87B017EEC9
:104AC000904A054684EAE470002303A9A0EBE47051
:104AD00001930093029317F08DFB002CACBF2023B1
:104AE0002D2303A88DF800302CF0A1FE012803A986
:104AF00024D002282DD0032805BF302368466846FD
:104B00008DF801302EF08DFF68462CF090FE0338B2
:104B1000C4B22246694628462EF0BAFF00232B5520
:104B200028462CF084FE2E22431C2A540DEB04014F
:104B3000E8182EF093FF284607B030BD30236846B2
:104B40008DF801308DF802308DF803302EF069FFBA
:104B5000DAE7302368468DF801308DF802302EF008
:104B600060FFD1E76F12033A00007A442DE9F0416B
:104B7000064615460846B6FBF2F43CB905FB14643C
:104B8000124B1B5D00F8013BBDE8F081B4FBF2F76E
:104B900067B90E4B05FB174705FB1464DA5D00F897
:104BA000012B1B5D00F8013BBDE8F081B7FBF2F87B
:104BB000B8F1000F02D04046FFF7D8FF05FB187888
:104BC000024B13F8082000F8012BE3E7647804088F
:104BD000104B2DE93048D3E9004554EA05020BD1CA
:104BE0000346012200201871587198719A70DA708A
:104BF00018801881BDE83088074B1A6814EB020B47
:104C000045F1000C5A466346FEF736FC0120BDE82C
:104C1000308800BF80250020E86B0020F0B40288B7
:104C20008578164FC37804794179A2F2B27202F006
:104C3000030606EB4606013D05EB860507EB450539
:104C4000013BAE898579008940F2B557920807FB90
:104C50000232931903EB430304EBC303C3EB0313C7
:104C600001EB8303C3EB031305EB830300214FF434
:104C70007A72C2FB0301F0BC704700BF3C400408DD
:104C8000FAB170B48E18044603E0101A14D1B14280
:104C900014D014F8012BA2F14103192B11F8013B98
:104CA000A3F1410598BF2032192D03F12000ECD962
:104CB000D01A01D1002BEAD170BC7047002070BC23
:104CC0007047104670474FF0FF32FFF7D9BFA0F191
:104CD0006103192B98BF20387047A0F14103192BAD
:104CE00098BF20307047202805D0093804288CBF91
:104CF00000200120704701207047613819288CBFBF
:104D0000002001207047413819288CBF0020012065
:104D10007047303809288CBF002001207047A0F16F
:104D20003003092B07D920F02000413819288CBF07
:104D30000020012070470120704730B402681146FE
:104D4000531C036011F8024B0160D31C51780360BF
:104D50009378151D05601B0443EA0123D078234393
:104D600043EA006030BC70470368591C1A46016072
:104D700012F8021B0260587841EA0020704703686D
:104D80005A1C02601878704738B50446006815460A
:104D90002DF0ACFC22682A44226038BD036810B4B0
:104DA0000A0E5C1C04601A7003680A0C5C1C046028
:104DB0001A7003680A0A5C1C04601A7003685A1CA3
:104DC000026019705DF8044B7047036810B40A0A5A
:104DD0005C1C04601A7003685A1C026019705DF84C
:104DE000044B704703685A1C026010B419700368C2
:104DF0000A0A5C1C04601A7003680A0C5C1C0460DC
:104E00001A700368090E5A1C026019705DF8044B91
:104E1000704703685A1C026019700368090A5A1C1B
:104E20000260197070472DE9F047002488B0804671
:104E30000F461E46A14605AD531C0393117839B3A6
:104E4000252933D1931CCDF8109003935078302846
:104E50004ED04FF0000AA0F13003DBB2092B42D94B
:104E60006C2819D0642800F0938024D825281CD001
:104E700063D9582876D063281BD131784046B8478B
:104E8000039A531C03931178043601340029D7D1B7
:104E9000204608B0BDE8F087039B5A1C03921B789C
:104EA000642B7CD02AD8252B54D1252140460134AF
:104EB000B847039AC0E7732833D044D975284FD137
:104EC00006F1040E30682B4600220A217646FEF7D2
:104ED0009BFA049A0095534639464046FEF787FBF5
:104EE000039A0444A8E704AA03A920F0DFFFB7E768
:104EF000D31C039390784FF0010AACE7732B10D0CA
:104F00005BD9752B3AD0782B96D1A3F15802B2FA1F
:104F100082F2306852092B4610210436FEF774FAEB
:104F2000D7E73368049A0093394600234046FEF7DA
:104F30005EFB04360444039A7EE70028B9D120467C
:104F400008B0BDE8F0876E28B3D1039A3368043601
:104F50001C6071E72AD9582BD7D0632B8DD06BE713
:104F60007828A6D1A0F15802B2FA82F2306852092C
:104F70002B461021FEF748FA0436AAE706F1040E84
:104F800030682B4600220A217646FEF73DFAA0E75C
:104F9000331D306829461E46FEF708FA99E7331D8F
:104FA000306829461E46FEF701FA92E7002B7FF48F
:104FB00043AF204608B0BDE8F0876E2BC6D03BE774
:104FC0000EB400B584B005AB019053F8042B06492C
:104FD000039301A8FFF727FF019B00221A7004B07A
:104FE0005DF804EB03B07047E53501082DE9F047A3
:104FF00007468CB01E469246002A6AD115461446D2
:105000000A8840F2B1739A423AD98B78581E0B281D
:1050100036D891F803E00EF1FF301E2830D891F811
:1050200004C0BCF1170F2BD891F80590B9F13B0FD4
:1050300026D888793B2823D8B1F80880B8F57A7F3C
:105040001ED24FF00108002E34D109890491002CA2
:10505000B4BF2D212B21002CB8BF644203900591D1
:105060000795CDF80890CDF804C0CDF800E038469B
:1050700006942F49FFF7A4FF40460CB0BDE8F08727
:105080000023012118468E46ADF824308DF82830D3
:105090008DF829308DF82A30ADF82C3099469C4691
:1050A0001A4698468DF826108DF827100B4609A948
:1050B000002ECAD00390CDF80890CDF804C0CDF8EA
:1050C00000E038461B49FFF77BFF40460CB0BDE8C7
:1050D000F087194C84FB0234A318D417C4EB631473
:1050E000C4EB0415A2EB85052DB2002D0846B8BF10
:1050F0006D42FFF793FD4FF47A7200238046894694
:105100002DF060F83C230AFB030A4FF47A72002367
:10511000404649462DF056F84FF47A7192B200237A
:10512000C1FB0A2309A8FEF7A7F924B209A967E77A
:10513000AC7804088C780408898888880FB430B566
:1051400083B006AB0A490B4853F8042B0968006882
:105150000193FFF768FE084C05462068F4F7A6FEA9
:105160000028FAD0284603B0BDE8304004B07047AC
:10517000988200209C82002018250020DFED2B7AE9
:10518000B4EEE70AF1EE10FA4ADDDFED296A9FED91
:10519000297A01E0B0EE670AB4EEC70AF1EE10FA20
:1051A00070EE667AF6DC9FED247AF4EEC77AF1EEC3
:1051B00010FA38D5DFED1E6A9FED207A01E0F0EE9F
:1051C000407AF4EEC77AF1EE10FA37EEA60AF6D47A
:1051D000DFED1B7AB4EEE70AF1EE10FA14DDDFED35
:1051E000137A37EEC00A60EE006A9FED166A9FEDF3
:1051F000167ADFED167AA6EE867A20EE266AE6EEBD
:10520000877AA6EE270A7047DFED117AB4EEE70A37
:10521000F1EE10FA44BFDFED087A37EEC00AE2E79C
:10522000F0EE407ABFE7B0EE670AD1E7DB0F494006
:10523000DB0FC940E4CB1641DB0F49C0E4CB16C1FC
:10524000DB0FC93F92E741B99730083C15A82ABE49
:10525000DB0FC9BF80EAE073A3EBE0738B4205DB91
:10526000002801DD401A704702D1704700207047C6
:105270000844704709B909E0194690FBF1F301FBB6
:1052800013030846002BF7D1084670470146FBE799
:10529000F0EEC07AB0EEE07AB4EEE77AF1EE10FA12
:1052A000B4BFB0EE676AB0EE476AB5EE406AF1EEA1
:1052B00010FA46D0B4EEE77AF1EE10FA8CBFF0EEB9
:1052C000675AF0EE475AC5EE866A9FED1F3A9FED8A
:1052D0001F6A9FED1F4A9FED1F5ADFED1F3ADFED5A
:1052E0001F4ADFED1F5AA6EEC36AE6EEA34AA6EEFA
:1052F000864AB7EE006AA6EE845AA6EEA46AE6EEE7
:10530000855AC5EE866AB4EEE77AF1EE10FA48BF28
:10531000DFED147AF5EEC00A48BF77EEE66AF1EEEB
:1053200010FA48BFDFED107AB5EEC00A48BF77EE3D
:10533000E66AF1EE10FA48BFF1EE666AB0EE660A70
:105340007047DFED076ADEE739094E3DE3B59E3E63
:1053500088FA163E45FE7F3F99FB243F69A2163E20
:10536000A7DFA834DB0FC93FDB0F4940DFED317AFF
:1053700030EE277AFDEEC76A16EE903A2033402BC6
:1053800002D99FED2D0A7047B4EEE70AF1EE10FA4C
:105390004DDD9FED2A6ADFED2A6A01E0B0EE677A03
:1053A000B4EEE67AF1EE10FA77EE467AF6DC9FED8F
:1053B000257AF4EEC77AF1EE10FA35D5DFED1F6AE3
:1053C0009FED217A01E0F0EE407AF4EEC77AF1EE3B
:1053D00010FA37EEA60AF6D4DFED167AB4EEE70A35
:1053E000F1EE10FA1BDCDFED197AB4EEE70AF1EE0C
:1053F00010FA44BFDFED137A37EEC00A60EE006AA0
:105400009FED136A9FED137ADFED137AA6EE867A8D
:1054100020EE266AE6EE877AA6EE270A7047DFEDD1
:105420000F7A37EEC00AE9E7B0EE670AD4E7F0EE8C
:10543000477ABCE7DB0FC93F00000000DB0FC94023
:10544000E4CB1641DB0F49C0E4CB16C1DB0FC9BF6B
:1054500092E741B99730083C15A82ABEDB0F4940B6
:10546000FDEEC07A17EE903A2033402B51D8DFED95
:105470002D7AB4EEE70AF1EE10FA50DDDFED2A6A7C
:105480009FED2A7A01E0B0EE670AB4EEC70AF1EEAA
:1054900010FA70EE667AF6DC9FED257AF4EEC77AA4
:1054A000F1EE10FA38D5DFED206A9FED227A01E0A7
:1054B000F0EE407AF4EEC77AF1EE10FA37EEA60A73
:1054C000F6D4DFED1D7AB4EEE70AF1EE10FA1BDC3C
:1054D000DFED1A7AB4EEE70AF1EE10FA44BFDFED21
:1054E000147A37EEC00A60EE006A9FED156A9FEDF0
:1054F000157ADFED157AA6EE867A20EE266AE6EEBC
:10550000877AA6EE270A7047DFED067A37EEC00AE3
:10551000E9E79FED0E0A7047B0EE670AD1E7F0EEBB
:10552000407AB9E7DB0F4940DB0FC940E4CB1641B5
:10553000DB0F49C0E4CB16C1DB0FC93FDB0FC9BF8E
:1055400092E741B99730083C15A82ABE0000000038
:1055500007EE901AF8EE677A9FED837A27EE800ABD
:1055600020EE070AFDEEC07A17EE903A2033402B6A
:1055700000F28C80DFED7D7AB4EEE70AF1EE10FAEE
:1055800040F3E880B0EE407A9FED796ADFED796A0A
:1055900001E0B0EE677AB4EEE67AF1EE10FA77EE5B
:1055A000467AF6DC9FED747AF4EEC77AF1EE10FAE3
:1055B00040F1CD809FED6E6ADFED706A01E0F0EEA4
:1055C000477AF4EEE67AF1EE10FA37EE867AF6D400
:1055D000DFED6B7AB4EEE77AF1EE10FA51DCDFED35
:1055E000697AB4EEE77AF1EE10FA44BFDFED627A41
:1055F00037EEC77A27EE076ADFED635ADFED637A8D
:10560000DFED636A9FED635AE6EE257A67EE065A90
:10561000E6EE276AF7EE007AA5EEA67AF0EE675A74
:10562000E7EE055AE7EE457A87EEA55ADFED547AA4
:1056300030EE277AFDEEC76A16EE903A2033402B03
:1056400029D99FED557AF6EE006AB7EE006AF7EEBB
:10565000004AC4EEA57A0023836143610362C361FB
:1056600080ED045A67EEA66A27EE866A27EE877AEF
:10567000C0ED006AC0ED026A80ED016A80ED037A38
:105680007047DFED3A7A37EEC77AB3E7B7EE005AE4
:10569000F0EE455ACAE7B4EEE70AF1EE10FA5FDD24
:1056A0009FED336ADFED336A01E0B0EE677AB4EE66
:1056B000E67AF1EE10FA77EE467AF6DC9FED2E7A76
:1056C000F4EEC77AF1EE10FA47D59FED296ADFEDC7
:1056D0002B6A01E0F0EE477AF4EEE67AF1EE10FA8A
:1056E00037EE867AF6D4DFED267AB4EEE77AF1EE7D
:1056F00010FA27DCDFED237AB4EEE77AF1EE10FA48
:1057000044BFDFED1D7A37EEC77A27EE076ADFED7B
:105710001E4ADFED1E6ADFED1E7AE6EE246A67EEB2
:10572000064AE6EE267AB7EE006AA4EEA77AF6EE0F
:10573000006A36EE476AF8EE007A27EE277A66EEC0
:10574000266A84E7DFED097A37EEC77ADDE7B0EE47
:10575000677A3DE7F0EE407A24E7B0EE677AC2E779
:10576000F0EE477AAAE700BF27D4D236DB0F4940D4
:10577000DB0FC940E4CB1641DB0F49C0E4CB16C1B7
:10578000DB0FC93FDB0FC9BF92E741B99730083C37
:1057900015A82ABEF304353F0000008070B40668E7
:1057A0008E4217D90139751E002311F8014F0822C6
:1057B000634013F0800F4FEA430318BF83F0D50313
:1057C000013ADBB2F5D18D42EFD1721C0260337029
:1057D00070BC70470023F8E710B44C09012250F860
:1057E000243001F01F0102FA01F10B4340F824308C
:1057F0005DF8044B70474B0901F01F0150F823205E
:10580000012303FA01F1114214BF1846002070472A
:10581000074A084B10781B78074A834296BFC31A81
:10582000C3F180030020126818441044704700BF81
:10583000289C0020A59B00206C990020064A074B5D
:1058400010781B7883428ABFC3F18003C01AC01846
:10585000C0F17F00704700BF289C0020A59B00205E
:1058600030B5134C237883B01BB90120237003B0EB
:1058700030BD1049052200230D688DF804208DF8F5
:10588000053000BFA868FEF729FC6A4601A902237B
:1058900068682BF083FBA868FEF725FC00BF9DF825
:1058A000013003F0010383F00100237003B030BD29
:1058B0007D6C0020386C002070B5064C06462568CB
:1058C00003E023685B1BB34203D8FFF7C9FF00283E
:1058D000F7D070BDE86B00202DE9F04F89B0B2F130
:1058E000000A02900491039340F3C5800B46002206
:1058F00001EB8A0153F8040B8B420244FAD1039B5B
:105900000592002B00F0AF80059B002B7CD05E4BF6
:10591000059A1B68DFF8889100920099DAB2511855
:10592000B1F5807F8CBFC2F58072009A0192574A10
:1059300092689A4240F28280554A1178002206927B
:105940008DF81C2002228DF81820002960D01A0E34
:105950008DF819200DF11A021C0C190A937014709D
:1059600051700620FFF7A8FF0621D9F80000F9F7CB
:1059700047FC484A0123137000BFD9F800309868EB
:10598000FEF7ACFB424BD9F800201B785068002B87
:1059900006A90CBF0423052300222BF0FFFA0024E4
:1059A000049D029E019FA34629684FEA84080022B5
:1059B0000B46013471B1B9422DD2D9F800003168DB
:1059C00040682BF0EBFA2A68336813443360BF1A3F
:1059D000C5F800B0A24505F1040506F10406E3D1BF
:1059E000D9F800309868FEF77EFB00BF264B01997E
:1059F00000981B68421A0092234A0B441360039AD2
:105A00004AB3009A002A88D1059809B0BDE8F08F02
:105A10000DF11902A0E7029CD9F8003054F80810E3
:105A2000586800223B462BF0B9FA54F808202B683E
:105A30003A44DF1B44F808202F60D1E70598009C0A
:105A40001549164A001B0590059800230B7013702A
:105A500009B0BDE8F08F059B009A9B1A0593059845
:105A600009B0BDE8F08FFFF7FBFE00287FF44CAFD4
:105A7000039B0593C8E7039C1CB9FFF7F1FE05944F
:105A8000C2E700230593BFE76C99002008030020BC
:105A90007C6C00207D6C0020289C0020A59B0020B1
:105AA000386C002070B5104D104E2B7831788B4239
:105AB00084B016D00E4A03921A4402928CBF0C4650
:105AC000CA1A04A98CBFC3F180020024012341F843
:105AD000102D02A802220194FFF7FEFE002333706E
:105AE0002B7004B070BD00BFA59B0020289C002037
:105AF000A89B002070B5194C194D2378297899423C
:105B000084B027D0174A03921A44029234BF0E463B
:105B1000CA1A04A934BFC3F180020026002341F849
:105B2000102D02A802220196FFF7D6FE2378184412
:105B3000C0B203062B7848BF80F0800083422070FB
:105B400002D0002004B070BD002301202B70237010
:105B500004B070BD012004B070BD00BFA59B002043
:105B6000289C0020A89B002010B50C4C45F2082072
:105B7000FFF7A2FE20680621F9F742FB084B2068D8
:105B80000122C7211A70F9F73BFB06480649074A6C
:105B9000002303700B70136010BD00BF386C002031
:105BA0007D6C0020289C0020A59B00206C99002083
:105BB000F0B51F4C83B0277800234FF0030E0093FD
:105BC0000E4615468DF804308DF800E06FB3030ED5
:105BD0008DF801300DF10203010C020A9870197062
:105BE00006205A70FFF768FEE8B100BF114F3B680E
:105BF0009868FEF773FA23783A68002B14BF0523E0
:105C000004236946506800222BF0C8F93B683246ED
:105C1000002158682B462BF0C1F93B689868FEF7C5
:105C200062FA00BF284603B0F0BD0DF10103D3E7CF
:105C30007C6C0020386C0020F0B5124B9D6885B05C
:105C40000DB905B0F0BDED0A14D0002704AE7C19E3
:105C50006410E00210226946FFF7AAFF0F2809DD51
:105C60006B4653F8042B01320AD1B342F9D12546D1
:105C7000AF42ECDBFFF716FF034BED021D60E0E7E0
:105C8000671CF5E7080300206C9900202DE9F04F10
:105C90002DED0C8B364C99B06368069020469847E2
:105CA000002800F07D82B4F8A870002284F851200A
:105CB000002F67D1B4F93860206AA16AB4F93A209C
:105CC000656AB4F93C30DFF8B4A0301A5B1A521B95
:105CD000E06294F85210636304F12C0022630EF02A
:105CE000B3FCDAF80030990042F19E81D4ED0C5AF1
:105CF000DFF88CB0D4ED0B7A1E4A9BED406ADBEDE9
:105D0000416A9BED427ADBF80C311268B8EEE58A05
:105D1000D4ED0D5AF8EEE77AF8EEE58A013377EE26
:105D2000867A38EE268A78EE878A9342CBED407ADF
:105D30008BED418ACBED428ACBF80C3101F00A851C
:105D40000D4B049393F800C0BCF1140F03F05B8675
:105D5000DBF814210025062A01F2FA85DFE812F0AB
:105D60006C19D8189917EB1806188418D90D00BFAC
:105D7000648D0020CC380020216C0020509500203C
:105D8000082F0020D44BD549079391F801901B6848
:105D9000D348DFF8A08304904FF47A71B1FBF3F39A
:105DA000C3EB431603EB8603DE00B6B2B7420578B9
:105DB000B8F9060003F02C83D4F87CE0B4F938205D
:105DC000236E0EF1010107EE902A13440129E167C9
:105DD0002366F8EEE77A03F02583D4ED1B5AD4ED61
:105DE0001D6A07EE101A37EEE56AB8EEC75A012FA2
:105DF00086EE057A37EE257A77EEC77A84ED1C7A3F
:105E0000E7EE866A84ED1B7AF0EE667AC4ED1E6AD0
:105E1000C4ED1D6A03F05387D4F890E0B4F93A203A
:105E2000636E0EF1010107EE902A13440129C4F8B4
:105E300090106366F8EEE77A03F00C83D4ED205AF5
:105E4000D4ED226A07EE101A37EEE56AB8EEC75AAB
:105E5000012F86EE057A37EE257A77EEC77A84ED44
:105E6000217AE7EE866A84ED207AF0EE667AC4ED58
:105E7000236AC4ED226A03F04A87D4F8A4E0B4F997
:105E80003C20A36E0EF1010107EE902A1344012974
:105E9000C4F8A410A366F8EEE77A03F0F482D4ED18
:105EA000255AD4ED276A07EE101A37EEE56AB8EEE8
:105EB000C75A012F86EE057A37EE257A77EEC77A34
:105EC00084ED267AE6EE276A84ED257AF0EE667A8E
:105ED000C4ED286AC4ED276A03F0E486DFF858B2FF
:105EE000A8F80600B4F8A830049A013B1578A4F885
:105EF000A83007990023072D4B608B60CB6040F0E2
:105F00005781F3F7A9FC049BDFF828821D78069BD4
:105F1000C01A9BF82131A8F800000993002B40F02B
:105F20004D816E4B5B79002B01F008836D4B1B7824
:105F3000013BDBB2072D8BF8213102F0688400238E
:105F40000A93694ADBF82C31D2ED006A674A9FED6B
:105F5000686AD2F800A0604A0792069ADBED4AAA66
:105F6000DFF8D8819BED499A9FED62AADFED62BA16
:105F70009FED62CA9FED62BADFF8C491614FCBF822
:105F80002C21D31A07EE903AF8EE677AB7EE007A32
:105F9000C6EE279A08F11C03002508935A4B059377
:105FA0002E4677EE6A8A68EEA68AF4EEC78AF1EE8C
:105FB00010FA88BFF0EE478A544B98ED008A2B44C4
:105FC000D3ED007AF5EE407AF1EE10FA17D0504B8F
:105FD0002B4493ED007A78EE476AB0EEE66AF4EE71
:105FE000C67AF1EE10FA08D5F5EEC06AF1EE10FAB5
:105FF000CCBF37EE878A37EE678A83ED008A454B40
:106000001A8893073FD0022E3DD0434B9AF82E10AA
:1060100033F9163007EE103A089B07EE901A2B441E
:10602000F8EEE76AB8EEC77AD3ED007A4B42A6EEF7
:10603000A77A700007EE903AF8EEE77AB4EEE77AC6
:10604000F1EE10FA0AD407EE901AF8EE677AF4EE41
:10605000C77AF1EE10FA88BFF0EE477A2F4B30493D
:106060000344085EB3F90C30C01A07EE100AB8EE0C
:10607000C77AD007E7EE4A7A41F1F681294B93EDD2
:10608000008A27EE888A079B9BF864212B4493EDB6
:1060900001DA78EE4DCA002A00F0E780224BDBF8E7
:1060A000682106991B688A1A9A4240F3DE809AF8A2
:1060B0004830022B02F0F283022E04F0F2841B4BD4
:1060C0001B68990700F19280194B87ED00CA1B6885
:1060D0009342C0F2C48035E040950020508D0020EE
:1060E000216C0020349900205069002084B70020E2
:1060F00000247449CDCCCC3DAE47813F0000000068
:106100000000C84200970020F49600204469002057
:106110004430002080B700205030002040990020FB
:1061200030B700202C6900205869002024B70020D7
:1061300054690020246C0020082F002038300020F3
:106140000C970020F7EE007AF4EEE7AAF1EE10FAD1
:1061500040F18B8007991F4BD1ED017A93ED007AC6
:10616000F0EEE77AF4EEC77AF1EE10FA7DD5D1EDD4
:10617000027AF0EEE77AB4EEE77AF1EE10FA74DD27
:10618000D1ED037AF0EEE77AB4EEE77AF1EE10FAA9
:106190006BDD114B1B689A0761D51049104B45E028
:1061A000104BDFF844B01D780493072D3FF4A9AEDF
:1061B0009BF821310993002B3FF4B3AE581E8BF8A6
:1061C0002101012D01F0168419B0BDEC0C8BBDE846
:1061D000F08F00BF6069002024B7002030B7002096
:1061E00040990020216C0020082F0020D74BD8496F
:1061F000DFF8CCE331F916C09EED008ADFF8C4E386
:1062000087ED00CA03EB460028EE0A8AB0F90C00BD
:10621000A0EB0C0007EE900AF8EEE77ADEF800003B
:1062200027EE888A904278EE4DCA8BDAB3F90C20BB
:10623000B1F900E0C748AEEB020E00688EEAEE72DC
:10624000A2EBEE72824210DAB3F90E30B1F90220FD
:10625000D21A82EAE273A3EBE273984205DD0023CF
:1062600018468BF86431F3F755FCBB4B2B4493ED88
:10627000000A059B29EE000A022E20EE2C0AA3EC50
:10628000010A059304F05B84B44BD7ED006A93EDEB
:10629000007AB34BD3ED007AB24B93ED006AB24B68
:1062A00067EE277A2B4427EEA87AD3ED007A67EEC3
:1062B000277AF0EE665AECEEA75AB1EE467AF4EE83
:1062C000C75AF1EE10FA08D4F4EEC65AF1EE10FAFD
:1062D0008CBFB0EE467AB0EE657A9BED4A6AF7EE77
:1062E000007AB4EEE76AF1EE10FAACBF01230023A6
:1062F00043B1F0EEE66AF0EEC77AF4EEE67AF1EE3C
:1063000010FA01D587ED007A022E04F0B483974A83
:10631000974B52F826001B68B0EE4D0A9847954AF5
:10632000954B52F826001B6898479AF8373023B1EE
:10633000924B1B88002B01F00481B0EE4C8A904BED
:1063400038EE400A2B4493ED008A83ED000A9AF858
:10635000483030EE480A20EE298A53B3894B1B7827
:10636000DB0741F17480F7EE007AF4EEE7AAF1EE74
:1063700010FA9BF86431C1F24687002B01F0868148
:10638000DBF86831069AD31A7F4A12689A4210DD08
:106390007E4BD3ED007AF0EEECCAF4EEE7CAF1EEF4
:1063A00010FA42F18482002318468BF86431F3F727
:1063B000B1FB774B9BF874212B4493ED000A29EE37
:1063C000000A20EE088A89ED008A32B9059B87ED24
:1063D00000CA03ED01CA89ED00CA0136032E08F197
:1063E000040809F1040907F1040705F104057FF425
:1063F000E3AD049B1B78072B01F00A87012B02F009
:10640000F381002308939BF87C31002B41F0FF823D
:10641000604BDFF8B4A11E68DAF8003096F82C70F3
:10642000D90401F1A9805C4B5C4A059319465C4B89
:10643000498B5C4D92ED006AD3ED004A5A4A5B4BA2
:10644000D5ED036AD3ED005AD2ED007A92ED014A00
:1064500092ED025A8BED636A07EE101AB8EEC77A16
:1064600074EEC63A012336EEC77A8BED616ACBED46
:10647000603ACBED644A8BF89431C7EE258A338DB0
:106480005A4206EE102A4A4ADFED4A6AD2ED005A15
:10649000494AD2ED004AB7EE007AF4EEC78A75EEAB
:1064A000A45AF1EE10FA88BFF0EE478A75EEA75AAB
:1064B000B8EEC66AF4EEE68AF1EE10FA07EE903A0C
:1064C000F4EEC65AB8BFF0EE668AF1EE10FACBEDE4
:1064D000678AB8EE677A01F19084F4EEC75AF1EE5C
:1064E00010FA88BFF0EE475A314BDFED346AD3ED36
:1064F000017A314BD3ED014A77EEA47A65EEA65AC4
:1065000077EE847AB4EEE76AF1EE10FA08DCB4EEC6
:10651000E77AF1EE10FA8CBFB0EE676AB0EE476A28
:10652000234A738DD2ED027A9FED247A5A4204EE0B
:10653000902A75EE277AF8EEE44A26EE076AF4EE22
:10654000E47AF1EE10FA4CD440E000BF409900200C
:1065500030B700205C690020006900208000002026
:10656000A4640020746900200C690020AC64002041
:10657000A864002000650020FC64002080B7002093
:1065800074300020105100205869002064690020F8
:106590001869002084B70020F48B0020B4970020F5
:1065A00024990020A8BA0020009700200C6A00203F
:1065B000F4960020000000000C9700206F12833A30
:1065C0002C690020546900205095002007EE103AF5
:1065D000F8EE474AF4EEE74AF1EE10FA88BFF0EE23
:1065E000674AEB4BDFEDEB7A5B7864EEA74A0BB9B9
:1065F000F1EE644A002F42F03D80F7EE003AE64F9C
:106600003E78002E03F0DB81E44BDFEDE57A93ED7D
:10661000025AD3ED016A93ED037A26EE055AA5EEF0
:10662000A65AA4EE875A23EE855AB4EEE75AF1EE45
:1066300010FAB4BFB0EE674AB0EE454A98BFF0EE2C
:10664000457A012E8DED105A03F0F08193ED067A14
:1066500093ED053AD3ED076A26EE077AA5EE837A25
:10666000A4EEA67A23EE877AB4EEE77AF1EE10FA7A
:10667000B4EEC47A8CBFF0EE676AF0EE476AF1EED2
:1066800010FA88BFF0EE676AB4BFF0EE447AF0EE1D
:10669000477A022E8DED117A00F0DE8093ED0A7AB2
:1066A00093ED093A93ED0B4A26EE077AA5EE837A2D
:1066B000A4EE847A23EE877AB4EEE67AF1EE10FA4D
:1066C000B4EEE77A8CBFB0EE664AB0EE474AF1EE20
:1066D00010FA98BFF0EE446AA8BFF0EE477A032E96
:1066E0008DED127A00F0B88093ED0E7A93ED0D3AAD
:1066F00093ED0F4A26EE077AA5EE837AA4EE847A0C
:1067000023EE877AB4EEE67AF1EE10FAB4EEE77A89
:106710008CBFB0EE664AB0EE474AF1EE10FA98BF71
:10672000F0EE446AA8BFF0EE477A042E8DED137A9E
:1067300000F0928093ED124A93ED113A93ED137AA3
:1067400026EE044AA5EE834AA4EE874A23EE844A45
:10675000B4EEE64AF1EE10FAB4EEE74A8CBFB0EEC2
:10676000667AB0EE447AF1EE10FA98BFF0EE476A1E
:10677000A8BFF0EE447A052E8DED144A6CD093ED4F
:10678000164A93ED153A93ED177A26EE044AA5EED4
:10679000834AA4EE874A23EE844AB4EEE64AF1EE39
:1067A00010FAB4EEE74A8CBFB0EE667AB0EE447AE7
:1067B000F1EE10FA98BFF0EE476AA8BFF0EE447A07
:1067C000062E8DED154A47D093ED1A4A93ED193AEE
:1067D00093ED1B7A26EE044AA5EE834AA4EE874A7F
:1067E00023EE844AB4EEE64AF1EE10FAB4EEE74A3C
:1067F0008CBFB0EE667AB0EE447AF1EE10FA98BF34
:10680000F0EE476AA8BFF0EE447A072E8DED164AE7
:1068100022D093ED1E7A93ED1D3A93ED1F4A26EE9A
:10682000077AA5EE837AA4EE247A27EE237AB4EED3
:10683000E67AF1EE10FAB4EEE77A8CBFB0EE666A53
:10684000B0EE476AF1EE10FA8DED177A98BFF0EED0
:10685000466AA8BFF0EE477A77EEE67AF7EE006A6E
:10686000F4EEE67AF1EE10FACBED4A7A43F3F587CF
:1068700086EEA77A022EDDED117A27EE055A67EE35
:10688000877A8DED105ACDED117A2DD0DDED127A8B
:1068900067EE877A032ECDED127A25D0DDED137ADF
:1068A00067EE877A042ECDED137A1DD0DDED147AD4
:1068B00067EE877A052ECDED147A15D0DDED157AC9
:1068C00067EE877A062ECDED157A0DD0DDED167ABE
:1068D00067EE877A072ECDED167A05D0DDED177AB3
:1068E00027EE877A8DED177A2E4B1B68DA0041F17F
:1068F0001684F6EE008ACBED678A002E03F05680F0
:10690000294B9BF99421D878284BDBED647A93F8D6
:1069100000E0274B9BED63AA079309EE102AB3F919
:106920000630244A0A93FDEEE77A059BDAF800C0A8
:106930002149D2ED00AA5B8B91F800900B9317EEE2
:10694000902AFDEECA7A0CF010010CF48053DBEDB6
:10695000609A9BED618AB8EEC99A0EF0010C17EEB1
:10696000908A002841F0AE80002941F05B850B49F8
:106970009DED107AD1ED007A104B68EEA77AE7EE24
:10698000097AB0EE487AA7EEA97AFDEEC77A17E049
:10699000709900206F12833AA1B900207C69002011
:1069A000000000009C970020AC3C0020105100200B
:1069B000DCAD00207869002020540020549700208E
:1069C00017EE90EA17EE900A9645A8BF1046F045DC
:1069D000C8BF404607EE900AF8EEE77A012EC3EDF5
:1069E000007A00F0DC80D1ED047A9DED117A68EE3A
:1069F000A77AE7EE097AB0EE487AA7EEA97AFDEE1B
:106A0000C77A17EE90EA17EE900A9645A8BF10468F
:106A1000F045C8BF404607EE900AF8EEE77A022E2E
:106A2000C3ED017A00F0BB80D1ED087A9DED127ABA
:106A300068EEA77AE7EE097AB0EE487AA7EEA97A6F
:106A4000FDEEC77A17EE90EA17EE900A9645A8BFBA
:106A50001046F045C8BF404607EE900AF8EEE77AC8
:106A6000032EC3ED027A00F09A80D1ED0C7A9DEDF1
:106A7000137A68EEA77AE7EE097AB0EE487AA7EEC5
:106A8000A97AFDEEC77A17EE90EA17EE900A9645BE
:106A9000A8BF1046F045C8BF404607EE900AF8EE82
:106AA000E77A042EC3ED037A79D0D1ED107A9DED0B
:106AB000147A68EEA77AE7EE097AB0EE487AA7EE84
:106AC000A97AFDEEC77A17EE90EA17EE900A96457E
:106AD000A8BF1046F045C8BF404607EE900AF8EE42
:106AE000E77A052EC3ED047A59D0D1ED147A9DEDE5
:106AF000157A68EEA77AE7EE097AB0EE487AA7EE43
:106B0000A97AFDEEC77A17EE90EA17EE900A96453D
:106B1000A8BF1046F045C8BF404607EE900AF8EE01
:106B2000E77A062EC3ED057A39D0D1ED187A9DEDBE
:106B3000167A68EEA77AE7EE097AB0EE487AA7EE01
:106B4000A97AFDEEC77A17EE90EA17EE900A9645FD
:106B5000A8BF1046F045C8BF404607EE900AF8EEC1
:106B6000E77A072EC3ED067A19D0D1ED1C7A9DED98
:106B7000177A68EEA78AE9EE078AA9EEA88AFDEEE1
:106B8000C87A17EE901A8A42A8BF0A468845D8BF2D
:106B9000904607EE908AF8EEE77AC3ED077ABCF1EB
:106BA000000F01F09D80E14B1B68002B41F0A58098
:106BB000DF4B1B789BB1387870B1DFF8A083DFF82A
:106BC000A0930026F0B2D9F80030B8EC010A98473B
:106BD000387801368642F5DBD64B1B689847049B14
:106BE0001B78072B01F0298300230B93DAF8003080
:106BF0000A935E0501F17481CF4B1F683C0701F1D8
:106C00001181CE4BB3F80090CD4B0893CD4B079A32
:106C10001C68B2F906806289904580F25F864FF069
:106C20007E53CBF824310599089A0E8B079992F977
:106C30000430B1F9000092F801E01178002BA0EBCC
:106C4000060383EAE37CACEBE37C14BF01224FF044
:106C5000FF32BCF5FA7FA8BF4FF4FA7C614580F2A1
:106C60003986ACEB010307EE903AF8EEE77AB042D2
:106C7000C5ED007A03DAF1EE677AC5ED007A079B7D
:106C8000B3F90200831B83EAE37CACEBE37CBCF545
:106C9000FA7FA8BF4FF4FA7C614580F21786ACEB0F
:106CA000010307EE903AF8EEE77AB042C5ED017ABB
:106CB00003DAF1EE677AC5ED017A079BB3F90410A8
:106CC0008B1B83EAE370A0EBE370B0F5FA7FA8BFFB
:106CD0004FF4FA707045CCBFA0EB0E0E4FF0000ED3
:106CE00002FB0EFE07EE90EAF8EEE77AB1420A9B4D
:106CF000C5ED027ABCBFF1EE677AC5ED027A13F4F6
:106D00008053079300F0BD85B8F5FA6F4246A8BFDF
:106D10004FF4FA62B2F57A7F9BF8A431B8BF4FF412
:106D20007A72A2F57A72002B40F0C4858649DFF8AA
:106D300034E281FB0230D317C3EB6013581C6FF0B1
:106D4000630C3EF910003EF913E00CFB0323A0EBAB
:106D50000E0003FB00F381FB0321DB17C3EB611380
:106D60009E440FFA8EFE07EE90EA079BB8EEE78A84
:106D700085ED038A002B41F0C08019F040030C938D
:106D800000F0FD80714B724993ED019A93ED026A18
:106D900091ED020A91ED043AD3ED030AD3ED003AE6
:106DA000D1ED038AD1ED015AD5ED011A95ED002AF6
:106DB000684B30EE435A39EE467A73EEA07A25EEF0
:106DC000077A75EEE84A73EEE09A35EEA8AA24EE4B
:106DD000A71AB0EE474AAAEE294A19F00302B0EE0C
:106DE000415A79EE067A70EE036AAAEE295AA6EEA7
:106DF000A74AA6EEE75AF0EE474AD6EEA74A34EE87
:106E0000014AF6EE006A73EE89AA26EEC44A35EE10
:106E1000475A35EE807AF0EE647AEAEE694AA7EED8
:106E20002A4A77EEC17A36EE607A73EE68AA25EECA
:106E3000265AEAEE297AAAEE875A74EE814A24EE9F
:106E4000047A73EEC93A33EE283A64EEA64A67EE46
:106E5000A66AF0EE477AE3EE234A75EEC05A36EEA4
:106E6000206AD5EE057AA5EE057AE5EE866AF1EEA2
:106E7000648AB0EE476AB0EE677AA8EEA47AF1EEC3
:106E8000663A26EEA43AA3EEA66A64EE260AF0EE6F
:106E9000665AB1EE450AA6EEA67AB0EE431AF0EEB7
:106EA000606AE3EEA57A64EE243AE5EE246AA0EE89
:106EB000041AA8EEA46AF0EE638A71EEA19AE0EEDD
:106EC000240AE5EE258A27EE217A32EE029AA5EE13
:106ED000043A61EE211A66EEA96AE4EEA47AE0EEC5
:106EE000253A0CBFD5ED022ADFED1B2A83ED005AAF
:106EF000E2EE066AA9EE207AE2EE281A33EE033AB1
:106F000067EEA27A73EEA33AB0EE006AA2EE837A3D
:106F1000E2EEA36AE1EE867A8BED6C7A85ED017A7A
:106F2000CBED6B6AC5ED006A1EE000BFE8520020A1
:106F3000485700201C54002024B7002080B70020B0
:106F40003899002088B700201F85EB51FC000020F5
:106F50008000002034010020000000005497002031
:106F600014540020286A0020CBED6D7A83ED014A8D
:106F7000C3ED025AC3ED034A0AB9C5ED027A17F010
